 Brackets

 Timestamp is 5e7d7d80 (Fri Mar 27 04:13:52 2020)

 Preferred load address is 0000000180000000

 Start         Length     Name                   Class
 0001:00000000 00000008H .CRT$XCA                CODE
 0001:00000008 00000008H .CRT$XCZ                CODE
 0001:00000010 00000008H .CRT$XIA                CODE
 0001:00000018 00000018H .CRT$XIC                CODE
 0001:00000030 00000008H .CRT$XIZ                CODE
 0001:00000038 00000008H .CRT$XPA                CODE
 0001:00000040 00000010H .CRT$XPX                CODE
 0001:00000050 00000008H .CRT$XPXA               CODE
 0001:00000058 00000008H .CRT$XPZ                CODE
 0001:00000060 00000008H .CRT$XTA                CODE
 0001:00000068 00000008H .CRT$XTZ                CODE
 0001:00000070 00000000H .gfids$y                CODE
 0001:00000070 00007848H .rdata                  CODE
 0001:000078b8 000001f4H .rdata$r                CODE
 0001:00007aac 000002c4H .rdata$zzzdbg           CODE
 0001:00007d70 00000008H .rtc$IAA                CODE
 0001:00007d78 00000008H .rtc$IZZ                CODE
 0001:00007d80 00000008H .rtc$TAA                CODE
 0001:00007d88 00000008H .rtc$TZZ                CODE
 0001:00007d90 0000f630H .text$mn                CODE
 0001:000173c0 00000020H .text$mn$00             CODE
 0001:000173e0 000002e0H .text$x                 CODE
 0001:000176c0 00000c48H .xdata                  CODE
 0001:00018308 000000f8H .xdata$x                CODE
 0001:00018400 000000a6H .edata                  CODE
 0002:00000000 00000a60H .data                   DATA
 0002:00000a60 000000a0H .data$r                 DATA
 0002:00000b00 000013b0H .bss                    DATA
 0003:00000000 00000f48H .pdata                  DATA
 0004:00000000 00000248H .idata$5                DATA
 0004:00000248 00000010H .00cfg                  DATA
 0004:00000258 00000028H .idata$2                DATA
 0004:00000280 00000018H .idata$3                DATA
 0004:00000298 00000248H .idata$4                DATA
 0004:000004e0 00000534H .idata$6                DATA
 0005:00000000 00000094H _RDATA                  DATA
 0006:00000000 00000060H .rsrc$01                DATA
 0006:00000060 00000380H .rsrc$02                DATA

  Address         Publics by Value              Rva+Base               Lib:Object

 0000:00000000       __hybrid_code_map_count    0000000000000000     <absolute>
 0000:00000000       __hybrid_code_map          0000000000000000     <absolute>
 0000:00000000       __guard_iat_count          0000000000000000     <absolute>
 0000:00000000       __volatile_metadata        0000000000000000     <absolute>
 0000:00000000       __guard_longjmp_count      0000000000000000     <absolute>
 0000:00000000       __guard_longjmp_table      0000000000000000     <absolute>
 0000:00000000       __guard_iat_table          0000000000000000     <absolute>
 0000:00000000       __guard_fids_count         0000000000000000     <absolute>
 0000:00000000       ___safe_se_handler_count   0000000000000000     <absolute>
 0000:00000000       __enclave_config           0000000000000000     <absolute>
 0000:00000000       __AbsoluteZero             0000000000000000     <absolute>
 0000:00000000       ___safe_se_handler_table   0000000000000000     <absolute>
 0000:00000000       __guard_fids_table         0000000000000000     <absolute>
 0000:00000000       __dynamic_value_reloc_table 0000000000000000     <absolute>
 0000:00000000       __hybrid_auxiliary_iat     0000000000000000     <absolute>
 0000:00000100       __guard_flags              0000000000000100     <absolute>
 0000:00000000       __ImageBase                0000000180000000     <linker-defined>
 0001:00000000       __xc_a                     0000000180001000     LIBCMT:initializers.obj
 0001:00000008       __xc_z                     0000000180001008     LIBCMT:initializers.obj
 0001:00000010       __xi_a                     0000000180001010     LIBCMT:initializers.obj
 0001:00000018       __acrt_multibyte_initializer 0000000180001018     libucrt:multibyte_initializer.obj
 0001:00000020       __acrt_stdio_initializer   0000000180001020     libucrt:stdio_initializer.obj
 0001:00000028       __acrt_tran_fma3_initializer 0000000180001028     libucrt:fma3_initializer.obj
 0001:00000030       __xi_z                     0000000180001030     LIBCMT:initializers.obj
 0001:00000038       __xp_a                     0000000180001038     LIBCMT:initializers.obj
 0001:00000040       __acrt_locale_terminator   0000000180001040     libucrt:locale_initializer.obj
 0001:00000048       __dcrt_console_output_terminator 0000000180001048     libucrt:console_output_initializer.obj
 0001:00000050       __acrt_stdio_terminator    0000000180001050     libucrt:stdio_initializer.obj
 0001:00000058       __xp_z                     0000000180001058     LIBCMT:initializers.obj
 0001:00000060       __xt_a                     0000000180001060     LIBCMT:initializers.obj
 0001:00000068       __xt_z                     0000000180001068     LIBCMT:initializers.obj
 0001:00000070       MainGuid                   0000000180001070     Brackets.obj
 0001:00000080       MenuGuid                   0000000180001080     Brackets.obj
 0001:00000090       DialogGuid                 0000000180001090     Brackets.obj
 0001:000000a0       ??_7?$DialogItemBinding@UFarDialogItem@@@@6B@ 00000001800010a0     Brackets.obj
 0001:000000b0       ??_7PluginCheckBoxBinding@@6B@ 00000001800010b0     Brackets.obj
 0001:000000c0       ??_7PluginRadioButtonBinding@@6B@ 00000001800010c0     Brackets.obj
 0001:000000d0       ??_7PluginEditFieldBinding@@6B@ 00000001800010d0     Brackets.obj
 0001:000000e0       ??_7PluginIntEditFieldBinding@@6B@ 00000001800010e0     Brackets.obj
 0001:000000f0       ??_C@_15EFLNJKHH@?$AA?$CF?$AAu@ 00000001800010f0     Brackets.obj
 0001:000000f8       ??_7PluginUIntEditFieldBinding@@6B@ 00000001800010f8     Brackets.obj
 0001:00000108       ??_7?$DialogBuilderBase@UFarDialogItem@@@@6B@ 0000000180001108     Brackets.obj
 0001:00000150       ??_7PluginDialogBuilder@@6B@ 0000000180001150     Brackets.obj
 0001:00000198       ??_C@_11LOCGONAA@@         0000000180001198     Brackets.obj
 0001:000001a0       ??_C@_1BC@GJFAHMHB@?$AAB?$AAr?$AAa?$AAc?$AAk?$AAe?$AAt?$AAs@ 00000001800011a0     Brackets.obj
 0001:000001c0       ??_C@_1EE@CJLEEDHO@?$AAB?$AAr?$AAa?$AAc?$AAk?$AAe?$AAt?$AAs?$AA?5?$AAm?$AAa?$AAt?$AAc?$AAh?$AAi@ 00000001800011c0     Brackets.obj
 0001:00000208       ??_C@_1DE@BGKMIKPD@?$AAE?$AAu?$AAg?$AAe?$AAn?$AAe?$AA?5?$AAR?$AAo?$AAs?$AAh?$AAa?$AAl?$AA?5?$AA?$CG@ 0000000180001208     Brackets.obj
 0001:00000240       ??_C@_1BK@LFBLPBJM@?$AAI?$AAg?$AAn?$AAo?$AAr?$AAe?$AAQ?$AAu?$AAo?$AAt?$AAe?$AAs@ 0000000180001240     Brackets.obj
 0001:00000260       ??_C@_1BI@LPBIFPPH@?$AAI?$AAg?$AAn?$AAo?$AAr?$AAe?$AAA?$AAf?$AAt?$AAe?$AAr@ 0000000180001260     Brackets.obj
 0001:00000278       ??_C@_1BK@LJLNAEDP@?$AAB?$AAr?$AAa?$AAc?$AAk?$AAe?$AAt?$AAP?$AAr?$AAi?$AAo?$AAr@ 0000000180001278     Brackets.obj
 0001:00000298       ??_C@_1BG@KDMBKMK@?$AAJ?$AAu?$AAm?$AAp?$AAT?$AAo?$AAP?$AAa?$AAi?$AAr@ 0000000180001298     Brackets.obj
 0001:000002b0       ??_C@_19CNDHNALO@?$AAB?$AAe?$AAe?$AAp@ 00000001800012b0     Brackets.obj
 0001:000002c0       ??_C@_1BG@KHOAFHB@?$AA?8?$AA?8?$AA?$CC?$AA?$CC?$AA?$GA?$AA?8?$AA?$GA?$AA?$GA?$AA?$BO?$AA?$BN@ 00000001800012c0     Brackets.obj
 0001:000002d8       ??_C@_1BG@ICHMEPOB@?$AAQ?$AAu?$AAo?$AAt?$AAe?$AAs?$AAT?$AAy?$AAp?$AAe@ 00000001800012d8     Brackets.obj
 0001:000002f0       ??_C@_1CC@FLEKOJBB@?$AA?$DM?$AA?$DO?$AA?$HL?$AA?$HN?$AA?$FL?$AA?$FN?$AA?$CI?$AA?$CJ?$AA?$CC?$AA?$CC?$AA?8?$AA?8?$AA?$CF?$AA?$CF?$PP?$KL@ 00000001800012f0     Brackets.obj
 0001:00000318       ??_C@_1BE@CHAAIDDE@?$AAB?$AAr?$AAa?$AAc?$AAk?$AAe?$AAt?$AAs?$AA1@ 0000000180001318     Brackets.obj
 0001:00000330       ??_C@_1BK@EKFLELHE@?$AA?1?$AA?$CK?$AA?$CK?$AA?1?$AA?$DM?$AA?$DP?$AA?$DP?$AA?$DO?$AA?$DM?$AA?$CF?$AA?$CF?$AA?$DO@ 0000000180001330     Brackets.obj
 0001:00000350       ??_C@_1BE@DFLFCMNK@?$AAB?$AAr?$AAa?$AAc?$AAk?$AAe?$AAt?$AAs?$AA2@ 0000000180001350     Brackets.obj
 0001:00000368       ??_C@_19MGMPFFIA@?$AAF?$AAi?$AAn?$AAd@ 0000000180001368     Brackets.obj
 0001:00000378       ??_C@_1O@MDCABJAO@?$AAD?$AAi?$AAr?$AAe?$AAc?$AAt@ 0000000180001378     Brackets.obj
 0001:00000388       ??_C@_1BE@LCCGEFEM@?$AAS?$AAE?$AAA?$AAR?$AAC?$AAH?$AAF?$AAW?$AAD@ 0000000180001388     Brackets.obj
 0001:000003a0       ??_C@_1BG@LIFFHAGC@?$AAS?$AAE?$AAA?$AAR?$AAC?$AAH?$AAB?$AAA?$AAC?$AAK@ 00000001800013a0     Brackets.obj
 0001:000003b8       ??_C@_1BE@IFIBPANP@?$AAS?$AAE?$AAL?$AAE?$AAC?$AAT?$AAF?$AAW?$AAD@ 00000001800013b8     Brackets.obj
 0001:000003d0       ??_C@_1BG@FJDCNJBP@?$AAS?$AAE?$AAL?$AAE?$AAC?$AAT?$AAB?$AAA?$AAC?$AAK@ 00000001800013d0     Brackets.obj
 0001:000003e8       ??_C@_1O@BAHOLLMK@?$AAC?$AAO?$AAN?$AAF?$AAI?$AAG@ 00000001800013e8     Brackets.obj
 0001:00000400       __xmm@ffffffffffffffff0000000000000002 0000000180001400     Brackets.obj
 0001:00000410       __xmm@ffffffffffffffffffffffffffffffff 0000000180001410     Brackets.obj
 0001:00000420       _pRawDllMain               0000000180001420     LIBCMT:dll_dllmain.obj
 0001:00000420       _pDefaultRawDllMain        0000000180001420     LIBCMT:dll_dllmain.obj
 0001:00000430       ??_7exception@std@@6B@     0000000180001430     LIBCMT:throw_bad_alloc.obj
 0001:00000440       ??_C@_0BC@EOODALEL@Unknown?5exception@ 0000000180001440     LIBCMT:throw_bad_alloc.obj
 0001:00000460       ??_7bad_alloc@std@@6B@     0000000180001460     LIBCMT:throw_bad_alloc.obj
 0001:00000470       ??_C@_0P@GHFPNOJB@bad?5allocation@ 0000000180001470     LIBCMT:throw_bad_alloc.obj
 0001:00000488       ??_7bad_array_new_length@std@@6B@ 0000000180001488     LIBCMT:throw_bad_alloc.obj
 0001:00000498       ??_C@_0BF@KINCDENJ@bad?5array?5new?5length@ 0000000180001498     LIBCMT:throw_bad_alloc.obj
 0001:000004b8       ??_7type_info@@6B@         00000001800014b8     LIBCMT:std_type_info_static.obj
 0001:000004c0       _pDestructExceptionObject  00000001800014c0     libvcruntime:ehhelpers.obj
 0001:00000bd0       ??_C@_08EHJDFFNH@__based?$CI@ 0000000180001bd0     libvcruntime:undname.obj
 0001:00000be0       ??_C@_07KOLFKCDI@__cdecl@  0000000180001be0     libvcruntime:undname.obj
 0001:00000be8       ??_C@_08GHMPAG@__pascal@   0000000180001be8     libvcruntime:undname.obj
 0001:00000bf8       ??_C@_09IFJBGAPI@__stdcall@ 0000000180001bf8     libvcruntime:undname.obj
 0001:00000c08       ??_C@_0L@NPHFGOKO@__thiscall@ 0000000180001c08     libvcruntime:undname.obj
 0001:00000c18       ??_C@_0L@JMKHOMEK@__fastcall@ 0000000180001c18     libvcruntime:undname.obj
 0001:00000c28       ??_C@_0N@BCKKPABJ@__vectorcall@ 0000000180001c28     libvcruntime:undname.obj
 0001:00000c38       ??_C@_09HIJEGCPM@__clrcall@ 0000000180001c38     libvcruntime:undname.obj
 0001:00000c44       ??_C@_06GHPCKEAG@__eabi@   0000000180001c44     libvcruntime:undname.obj
 0001:00000c50       ??_C@_09IOPIDJLG@__swift_1@ 0000000180001c50     libvcruntime:undname.obj
 0001:00000c60       ??_C@_09KFNFGKHF@__swift_2@ 0000000180001c60     libvcruntime:undname.obj
 0001:00000c70       ??_C@_07JOMMBBKO@__ptr64@  0000000180001c70     libvcruntime:undname.obj
 0001:00000c78       ??_C@_0L@PILCLIHE@__restrict@ 0000000180001c78     libvcruntime:undname.obj
 0001:00000c88       ??_C@_0M@GFIIJFMG@__unaligned@ 0000000180001c88     libvcruntime:undname.obj
 0001:00000c98       ??_C@_09DHDLOLLB@restrict?$CI@ 0000000180001c98     libvcruntime:undname.obj
 0001:00000ca2       ??_C@_00CNPNBAHC@@         0000000180001ca2     libvcruntime:undname.obj
 0001:00000ca4       ??_C@_04NIHEBCM@?5new@     0000000180001ca4     libvcruntime:undname.obj
 0001:00000cb0       ??_C@_07FPCDHGMM@?5delete@ 0000000180001cb0     libvcruntime:undname.obj
 0001:00000cb8       ??_C@_01NEMOKFLO@?$DN@     0000000180001cb8     libvcruntime:undname.obj
 0001:00000cbc       ??_C@_02GPIOPFAK@?$DO?$DO@ 0000000180001cbc     libvcruntime:undname.obj
 0001:00000cc0       ??_C@_02FODMEDOG@?$DM?$DM@ 0000000180001cc0     libvcruntime:undname.obj
 0001:00000cc4       ??_C@_01DCLJPIOD@?$CB@     0000000180001cc4     libvcruntime:undname.obj
 0001:00000cc8       ??_C@_02EGOFBIJA@?$DN?$DN@ 0000000180001cc8     libvcruntime:undname.obj
 0001:00000ccc       ??_C@_02FDNJECIE@?$CB?$DN@ 0000000180001ccc     libvcruntime:undname.obj
 0001:00000cd0       ??_C@_02GPECMEKF@?$FL?$FN@ 0000000180001cd0     libvcruntime:undname.obj
 0001:00000cd8       ??_C@_08LHJFAFGD@operator@ 0000000180001cd8     libvcruntime:undname.obj
 0001:00000ce4       ??_C@_02HBOOOICD@?9?$DO@   0000000180001ce4     libvcruntime:undname.obj
 0001:00000ce8       ??_C@_01NBENCBCI@?$CK@     0000000180001ce8     libvcruntime:undname.obj
 0001:00000cec       ??_C@_02ECNGHCIF@?$CL?$CL@ 0000000180001cec     libvcruntime:undname.obj
 0001:00000cf0       ??_C@_02BAABKJLB@?9?9@     0000000180001cf0     libvcruntime:undname.obj
 0001:00000cf4       ??_C@_01JOAMLHOP@?9@       0000000180001cf4     libvcruntime:undname.obj
 0001:00000cf8       ??_C@_01MIFGBAGJ@?$CL@     0000000180001cf8     libvcruntime:undname.obj
 0001:00000cfc       ??_C@_01HNPIGOCE@?$CG@     0000000180001cfc     libvcruntime:undname.obj
 0001:00000d00       ??_C@_03MNHNFDLC@?9?$DO?$CK@ 0000000180001d00     libvcruntime:undname.obj
 0001:00000d04       ??_C@_01KMDKNFGN@?1@       0000000180001d04     libvcruntime:undname.obj
 0001:00000d08       ??_C@_01FGNFDNOH@?$CF@     0000000180001d08     libvcruntime:undname.obj
 0001:00000d0c       ??_C@_01MNNFJEPP@?$DM@     0000000180001d0c     libvcruntime:undname.obj
 0001:00000d10       ??_C@_02EHCHHCKH@?$DM?$DN@ 0000000180001d10     libvcruntime:undname.obj
 0001:00000d14       ??_C@_01PPODPGHN@?$DO@     0000000180001d14     libvcruntime:undname.obj
 0001:00000d18       ??_C@_02EEKDKGMJ@?$DO?$DN@ 0000000180001d18     libvcruntime:undname.obj
 0001:00000d1c       ??_C@_01IHBHIGKO@?0@       0000000180001d1c     libvcruntime:undname.obj
 0001:00000d20       ??_C@_02HCKGKOFO@?$CI?$CJ@ 0000000180001d20     libvcruntime:undname.obj
 0001:00000d24       ??_C@_01PJKLJHI@?$HO@      0000000180001d24     libvcruntime:undname.obj
 0001:00000d28       ??_C@_01JKBOJNNK@?$FO@     0000000180001d28     libvcruntime:undname.obj
 0001:00000d2c       ??_C@_01DNKMNLPK@?$HM@     0000000180001d2c     libvcruntime:undname.obj
 0001:00000d30       ??_C@_02PPKAJPJL@?$CG?$CG@ 0000000180001d30     libvcruntime:undname.obj
 0001:00000d34       ??_C@_02NONPIBCD@?$HM?$HM@ 0000000180001d34     libvcruntime:undname.obj
 0001:00000d38       ??_C@_02FPIMKNGF@?$CK?$DN@ 0000000180001d38     libvcruntime:undname.obj
 0001:00000d3c       ??_C@_02FOEOMHFC@?$CL?$DN@ 0000000180001d3c     libvcruntime:undname.obj
 0001:00000d40       ??_C@_02FKMDLLOA@?9?$DN@   0000000180001d40     libvcruntime:undname.obj
 0001:00000d44       ??_C@_02FJEHGPIO@?1?$DN@   0000000180001d44     libvcruntime:undname.obj
 0001:00000d48       ??_C@_02FENAOKFI@?$CF?$DN@ 0000000180001d48     libvcruntime:undname.obj
 0001:00000d4c       ??_C@_03IKFCCPFF@?$DO?$DO?$DN@ 0000000180001d4c     libvcruntime:undname.obj
 0001:00000d50       ??_C@_03CDNPDDLA@?$DM?$DM?$DN@ 0000000180001d50     libvcruntime:undname.obj
 0001:00000d54       ??_C@_02FGJGFEAB@?$CG?$DN@ 0000000180001d54     libvcruntime:undname.obj
 0001:00000d58       ??_C@_02DHLNPPGH@?$HM?$DN@ 0000000180001d58     libvcruntime:undname.obj
 0001:00000d5c       ??_C@_02MHEGNOJ@?$FO?$DN@  0000000180001d5c     libvcruntime:undname.obj
 0001:00000d60       ??_C@_09IFPLHPGF@?$GAvftable?8@ 0000000180001d60     libvcruntime:undname.obj
 0001:00000d70       ??_C@_09BLBHBJP@?$GAvbtable?8@ 0000000180001d70     libvcruntime:undname.obj
 0001:00000d80       ??_C@_07FEEIOKP@?$GAvcall?8@ 0000000180001d80     libvcruntime:undname.obj
 0001:00000d88       ??_C@_08LLFFHHDJ@?$GAtypeof?8@ 0000000180001d88     libvcruntime:undname.obj
 0001:00000d98       ??_C@_0BF@KDPPACIK@?$GAlocal?5static?5guard?8@ 0000000180001d98     libvcruntime:undname.obj
 0001:00000db0       ??_C@_08OBABFOLI@?$GAstring?8@ 0000000180001db0     libvcruntime:undname.obj
 0001:00000dc0       ??_C@_0BD@JDLKDPAB@?$GAvbase?5destructor?8@ 0000000180001dc0     libvcruntime:undname.obj
 0001:00000dd8       ??_C@_0BN@DEGPLNFK@?$GAvector?5deleting?5destructor?8@ 0000000180001dd8     libvcruntime:undname.obj
 0001:00000df8       ??_C@_0BO@OBMKPJIG@?$GAdefault?5constructor?5closure?8@ 0000000180001df8     libvcruntime:undname.obj
 0001:00000e18       ??_C@_0BN@IMDCHIKM@?$GAscalar?5deleting?5destructor?8@ 0000000180001e18     libvcruntime:undname.obj
 0001:00000e38       ??_C@_0BO@PFGOCPJJ@?$GAvector?5constructor?5iterator?8@ 0000000180001e38     libvcruntime:undname.obj
 0001:00000e58       ??_C@_0BN@LFPFMEDL@?$GAvector?5destructor?5iterator?8@ 0000000180001e58     libvcruntime:undname.obj
 0001:00000e78       ??_C@_0CE@IKBNEHA@?$GAvector?5vbase?5constructor?5itera@ 0000000180001e78     libvcruntime:undname.obj
 0001:00000ea0       ??_C@_0BL@NILFHHPC@?$GAvirtual?5displacement?5map?8@ 0000000180001ea0     libvcruntime:undname.obj
 0001:00000ec0       ??_C@_0CB@JONCMFFK@?$GAeh?5vector?5constructor?5iterator@ 0000000180001ec0     libvcruntime:undname.obj
 0001:00000ee8       ??_C@_0CA@GCEOPDGL@?$GAeh?5vector?5destructor?5iterator?8@ 0000000180001ee8     libvcruntime:undname.obj
 0001:00000f08       ??_C@_0CH@OOJPLCPH@?$GAeh?5vector?5vbase?5constructor?5it@ 0000000180001f08     libvcruntime:undname.obj
 0001:00000f30       ??_C@_0BL@LLKPOHJI@?$GAcopy?5constructor?5closure?8@ 0000000180001f30     libvcruntime:undname.obj
 0001:00000f50       ??_C@_0BA@KBCDOMBN@?$GAudt?5returning?8@ 0000000180001f50     libvcruntime:undname.obj
 0001:00000f60       ??_C@_03KLGMFNMG@?$GAEH@   0000000180001f60     libvcruntime:undname.obj
 0001:00000f64       ??_C@_05KHLCHHI@?$GARTTI@  0000000180001f64     libvcruntime:undname.obj
 0001:00000f70       ??_C@_0BA@KKLDJDLB@?$GAlocal?5vftable?8@ 0000000180001f70     libvcruntime:undname.obj
 0001:00000f80       ??_C@_0CE@IIHCMGGL@?$GAlocal?5vftable?5constructor?5clos@ 0000000180001f80     libvcruntime:undname.obj
 0001:00000fa4       ??_C@_06FHBGPFGH@?5new?$FL?$FN@ 0000000180001fa4     libvcruntime:undname.obj
 0001:00000fb0       ??_C@_09LBNFPBCA@?5delete?$FL?$FN@ 0000000180001fb0     libvcruntime:undname.obj
 0001:00000fc0       ??_C@_0P@HJKNJFNN@?$GAomni?5callsig?8@ 0000000180001fc0     libvcruntime:undname.obj
 0001:00000fd0       ??_C@_0BL@CNOONJFP@?$GAplacement?5delete?5closure?8@ 0000000180001fd0     libvcruntime:undname.obj
 0001:00000ff0       ??_C@_0BN@CKNJLHMB@?$GAplacement?5delete?$FL?$FN?5closure?8@ 0000000180001ff0     libvcruntime:undname.obj
 0001:00001010       ??_C@_0CG@CFDHKGGD@?$GAmanaged?5vector?5constructor?5ite@ 0000000180002010     libvcruntime:undname.obj
 0001:00001038       ??_C@_0CF@IMGKMJNO@?$GAmanaged?5vector?5destructor?5iter@ 0000000180002038     libvcruntime:undname.obj
 0001:00001060       ??_C@_0CG@HLDDJMAG@?$GAeh?5vector?5copy?5constructor?5ite@ 0000000180002060     libvcruntime:undname.obj
 0001:00001088       ??_C@_0CM@FCBBDIGB@?$GAeh?5vector?5vbase?5copy?5construct@ 0000000180002088     libvcruntime:undname.obj
 0001:000010b8       ??_C@_0BL@CLIPGLGB@?$GAdynamic?5initializer?5for?5?8@ 00000001800020b8     libvcruntime:undname.obj
 0001:000010d8       ??_C@_0CB@PDBIFEP@?$GAdynamic?5atexit?5destructor?5for?5@ 00000001800020d8     libvcruntime:undname.obj
 0001:00001100       ??_C@_0CD@CGAJBKEJ@?$GAvector?5copy?5constructor?5iterat@ 0000000180002100     libvcruntime:undname.obj
 0001:00001128       ??_C@_0CJ@GJELGAMM@?$GAvector?5vbase?5copy?5constructor?5@ 0000000180002128     libvcruntime:undname.obj
 0001:00001158       ??_C@_0CL@FGIJHLCE@?$GAmanaged?5vector?5copy?5constructo@ 0000000180002158     libvcruntime:undname.obj
 0001:00001188       ??_C@_0BM@PMGGMLDN@?$GAlocal?5static?5thread?5guard?8@ 0000000180002188     libvcruntime:undname.obj
 0001:000011a8       ??_C@_0N@BDNMDMOL@operator?5?$CC?$CC?5@ 00000001800021a8     libvcruntime:undname.obj
 0001:000011b8       ??_C@_0BC@GGEBGALA@operator?5co_await@ 00000001800021b8     libvcruntime:undname.obj
 0001:000011d0       ??_C@_0M@GAAIMMOH@operator?$DM?$DN?$DO@ 00000001800021d0     libvcruntime:undname.obj
 0001:000011e0       ??_C@_0BC@DAFEJGAK@?5Type?5Descriptor?8@ 00000001800021e0     libvcruntime:undname.obj
 0001:000011f8       ??_C@_0BM@LDKODKLH@?5Base?5Class?5Descriptor?5at?5?$CI@ 00000001800021f8     libvcruntime:undname.obj
 0001:00001218       ??_C@_0BD@LGICGFMM@?5Base?5Class?5Array?8@ 0000000180002218     libvcruntime:undname.obj
 0001:00001230       ??_C@_0BN@MECKDCOJ@?5Class?5Hierarchy?5Descriptor?8@ 0000000180002230     libvcruntime:undname.obj
 0001:00001250       ??_C@_0BK@CFCOFLF@?5Complete?5Object?5Locator?8@ 0000000180002250     libvcruntime:undname.obj
 0001:00001270       ??_C@_0BG@JNJLAMPM@?$GAanonymous?5namespace?8@ 0000000180002270     libvcruntime:undname.obj
 0001:000012a0       ??_C@_1DM@KHCHBNEB@?$AAa?$AAp?$AAi?$AA?9?$AAm?$AAs?$AA?9?$AAw?$AAi?$AAn?$AA?9?$AAc?$AAo?$AAr?$AAe@ 00000001800022a0     libvcruntime:winapi_downlevel.obj
 0001:000012e0       ??_C@_1DK@LPPGFMPP@?$AAa?$AAp?$AAi?$AA?9?$AAm?$AAs?$AA?9?$AAw?$AAi?$AAn?$AA?9?$AAc?$AAo?$AAr?$AAe@ 00000001800022e0     libvcruntime:winapi_downlevel.obj
 0001:00001320       ??_C@_1BC@GDMECMAK@?$AAk?$AAe?$AAr?$AAn?$AAe?$AAl?$AA3?$AA2@ 0000000180002320     libvcruntime:winapi_downlevel.obj
 0001:00001338       ??_C@_1BA@PFFKHIOG@?$AAa?$AAp?$AAi?$AA?9?$AAm?$AAs?$AA?9@ 0000000180002338     libvcruntime:winapi_downlevel.obj
 0001:00001350       ??_C@_08KNHFBNJ@FlsAlloc@  0000000180002350     libvcruntime:winapi_downlevel.obj
 0001:00001368       ??_C@_07PEJMOBNF@FlsFree@  0000000180002368     libvcruntime:winapi_downlevel.obj
 0001:00001378       ??_C@_0M@GDNOONDI@FlsGetValue@ 0000000180002378     libvcruntime:winapi_downlevel.obj
 0001:00001390       ??_C@_0M@JCPCPOEF@FlsSetValue@ 0000000180002390     libvcruntime:winapi_downlevel.obj
 0001:000013a8       ??_C@_0BM@HCFOFFN@InitializeCriticalSectionEx@ 00000001800023a8     libvcruntime:winapi_downlevel.obj
 0001:000013d0       __acrt_exception_action_table 00000001800023d0     libucrt:exception_filter.obj
 0001:00001490       __acrt_signal_action_table_count 0000000180002490     libucrt:exception_filter.obj
 0001:00001498       __acrt_signal_action_first_fpe_index 0000000180002498     libucrt:exception_filter.obj
 0001:000014a0       __acrt_signal_action_fpe_count 00000001800024a0     libucrt:exception_filter.obj
 0001:000014a8       ??_C@_1BI@BGOHAHKC@?$AAm?$AAs?$AAc?$AAo?$AAr?$AAe?$AAe?$AA?4?$AAd?$AAl?$AAl@ 00000001800024a8     libucrt:exit.obj
 0001:000014c0       ??_C@_0P@MIGLKIOC@CorExitProcess@ 00000001800024c0     libucrt:exit.obj
 0001:00001758       ??_C@_1M@HPNHIDJI@?$AAj?$AAa?$AA?9?$AAJ?$AAP@ 0000000180002758     libucrt:mbctype.obj
 0001:00001768       ??_C@_1M@BIBDDEMK@?$AAz?$AAh?$AA?9?$AAC?$AAN@ 0000000180002768     libucrt:mbctype.obj
 0001:00001778       ??_C@_1M@JLOOOEGK@?$AAk?$AAo?$AA?9?$AAK?$AAR@ 0000000180002778     libucrt:mbctype.obj
 0001:00001788       ??_C@_1M@CLNBBOPM@?$AAz?$AAh?$AA?9?$AAT?$AAW@ 0000000180002788     libucrt:mbctype.obj
 0001:00001840       ??_C@_1EA@JGEFHKEI@?$AAa?$AAp?$AAi?$AA?9?$AAm?$AAs?$AA?9?$AAw?$AAi?$AAn?$AA?9?$AAc?$AAo?$AAr?$AAe@ 0000000180002840     libucrt:winapi_thunks.obj
 0001:00001880       ??_C@_1DI@IJCEHOCB@?$AAa?$AAp?$AAi?$AA?9?$AAm?$AAs?$AA?9?$AAw?$AAi?$AAn?$AA?9?$AAc?$AAo?$AAr?$AAe@ 0000000180002880     libucrt:winapi_thunks.obj
 0001:000018c0       ??_C@_1EI@MPIAOHOC@?$AAa?$AAp?$AAi?$AA?9?$AAm?$AAs?$AA?9?$AAw?$AAi?$AAn?$AA?9?$AAc?$AAo?$AAr?$AAe@ 00000001800028c0     libucrt:winapi_thunks.obj
 0001:00001910       ??_C@_1FK@FPHCKFIE@?$AAa?$AAp?$AAi?$AA?9?$AAm?$AAs?$AA?9?$AAw?$AAi?$AAn?$AA?9?$AAc?$AAo?$AAr?$AAe@ 0000000180002910     libucrt:winapi_thunks.obj
 0001:00001970       ??_C@_1EM@DILCGIIO@?$AAa?$AAp?$AAi?$AA?9?$AAm?$AAs?$AA?9?$AAw?$AAi?$AAn?$AA?9?$AAc?$AAo?$AAr?$AAe@ 0000000180002970     libucrt:winapi_thunks.obj
 0001:000019c0       ??_C@_1DM@LNCGDDPN@?$AAa?$AAp?$AAi?$AA?9?$AAm?$AAs?$AA?9?$AAw?$AAi?$AAn?$AA?9?$AAc?$AAo?$AAr?$AAe@ 00000001800029c0     libucrt:winapi_thunks.obj
 0001:00001a00       ??_C@_1DO@FPAPJEMD@?$AAa?$AAp?$AAi?$AA?9?$AAm?$AAs?$AA?9?$AAw?$AAi?$AAn?$AA?9?$AAc?$AAo?$AAr?$AAe@ 0000000180002a00     libucrt:winapi_thunks.obj
 0001:00001a40       ??_C@_1DK@NDHNAHIO@?$AAa?$AAp?$AAi?$AA?9?$AAm?$AAs?$AA?9?$AAw?$AAi?$AAn?$AA?9?$AAc?$AAo?$AAr?$AAe@ 0000000180002a40     libucrt:winapi_thunks.obj
 0001:00001a80       ??_C@_1DM@KGHDGBCM@?$AAa?$AAp?$AAi?$AA?9?$AAm?$AAs?$AA?9?$AAw?$AAi?$AAn?$AA?9?$AAc?$AAo?$AAr?$AAe@ 0000000180002a80     libucrt:winapi_thunks.obj
 0001:00001ac0       ??_C@_1EO@IJIOEFOH@?$AAa?$AAp?$AAi?$AA?9?$AAm?$AAs?$AA?9?$AAw?$AAi?$AAn?$AA?9?$AAr?$AAt?$AAc?$AAo@ 0000000180002ac0     libucrt:winapi_thunks.obj
 0001:00001b10       ??_C@_1FG@HHGEKANL@?$AAa?$AAp?$AAi?$AA?9?$AAm?$AAs?$AA?9?$AAw?$AAi?$AAn?$AA?9?$AAs?$AAe?$AAc?$AAu@ 0000000180002b10     libucrt:winapi_thunks.obj
 0001:00001b70       ??_C@_1EG@DBIOJECG@?$AAe?$AAx?$AAt?$AA?9?$AAm?$AAs?$AA?9?$AAw?$AAi?$AAn?$AA?9?$AAn?$AAt?$AAu?$AAs@ 0000000180002b70     libucrt:winapi_thunks.obj
 0001:00001bc0       ??_C@_1EO@FIHMJCLF@?$AAe?$AAx?$AAt?$AA?9?$AAm?$AAs?$AA?9?$AAw?$AAi?$AAn?$AA?9?$AAn?$AAt?$AAu?$AAs@ 0000000180002bc0     libucrt:winapi_thunks.obj
 0001:00001c10       ??_C@_1BC@DNHGCMLG@?$AAa?$AAd?$AAv?$AAa?$AAp?$AAi?$AA3?$AA2@ 0000000180002c10     libucrt:winapi_thunks.obj
 0001:00001c28       ??_C@_1M@OAIMIKLP@?$AAn?$AAt?$AAd?$AAl?$AAl@ 0000000180002c28     libucrt:winapi_thunks.obj
 0001:00001c40       ??_C@_1EG@DPGNFKGC@?$AAa?$AAp?$AAi?$AA?9?$AAm?$AAs?$AA?9?$AAw?$AAi?$AAn?$AA?9?$AAa?$AAp?$AAp?$AAm@ 0000000180002c40     libucrt:winapi_thunks.obj
 0001:00001c88       ??_C@_1O@BCCLBEOE@?$AAu?$AAs?$AAe?$AAr?$AA3?$AA2@ 0000000180002c88     libucrt:winapi_thunks.obj
 0001:00001c98       ??_C@_1BA@IAIFMGEF@?$AAe?$AAx?$AAt?$AA?9?$AAm?$AAs?$AA?9@ 0000000180002c98     libucrt:winapi_thunks.obj
 0001:00001cb0       ??_C@_0BA@FHFNEAED@AreFileApisANSI@ 0000000180002cb0     libucrt:winapi_thunks.obj
 0001:00001cf0       ??_C@_0O@KKBNKAPF@LCMapStringEx@ 0000000180002cf0     libucrt:winapi_thunks.obj
 0001:00001d08       ??_C@_0BB@HBDEELFH@LocaleNameToLCID@ 0000000180002d08     libucrt:winapi_thunks.obj
 0001:00001d20       ??_C@_0CF@OJOFEIGO@AppPolicyGetProcessTerminationM@ 0000000180002d20     libucrt:winapi_thunks.obj
 0001:00001d50       __lc_time_c                0000000180002d50     libucrt:nlsdata.obj
 0001:00002010       ??_C@_03KOEHGMDN@Sun@      0000000180003010     libucrt:nlsdata.obj
 0001:00002014       ??_C@_03PDAGKDH@Mon@       0000000180003014     libucrt:nlsdata.obj
 0001:00002018       ??_C@_03NAGEINEP@Tue@      0000000180003018     libucrt:nlsdata.obj
 0001:0000201c       ??_C@_03MHOMLAJA@Wed@      000000018000301c     libucrt:nlsdata.obj
 0001:00002020       ??_C@_03IOFIKPDN@Thu@      0000000180003020     libucrt:nlsdata.obj
 0001:00002024       ??_C@_03IDIOELNC@Fri@      0000000180003024     libucrt:nlsdata.obj
 0001:00002028       ??_C@_03FEFJNEK@Sat@       0000000180003028     libucrt:nlsdata.obj
 0001:0000202c       ??_C@_06OOPIFAJ@Sunday@    000000018000302c     libucrt:nlsdata.obj
 0001:00002034       ??_C@_06JLEDEDGH@Monday@   0000000180003034     libucrt:nlsdata.obj
 0001:00002040       ??_C@_07BAAGCFCM@Tuesday@  0000000180003040     libucrt:nlsdata.obj
 0001:00002048       ??_C@_09DLIGFAKA@Wednesday@ 0000000180003048     libucrt:nlsdata.obj
 0001:00002058       ??_C@_08HACCIKIA@Thursday@ 0000000180003058     libucrt:nlsdata.obj
 0001:00002064       ??_C@_06JECMNKMI@Friday@   0000000180003064     libucrt:nlsdata.obj
 0001:00002070       ??_C@_08INBOOONO@Saturday@ 0000000180003070     libucrt:nlsdata.obj
 0001:0000207c       ??_C@_03JIHJHPIE@Jan@      000000018000307c     libucrt:nlsdata.obj
 0001:00002080       ??_C@_03HJBDCHOM@Feb@      0000000180003080     libucrt:nlsdata.obj
 0001:00002084       ??_C@_03ODNJBKGA@Mar@      0000000180003084     libucrt:nlsdata.obj
 0001:00002088       ??_C@_03LEOLGMJP@Apr@      0000000180003088     libucrt:nlsdata.obj
 0001:0000208c       ??_C@_03CNMDKL@May@        000000018000308c     libucrt:nlsdata.obj
 0001:00002090       ??_C@_03IDFGHECI@Jun@      0000000180003090     libucrt:nlsdata.obj
 0001:00002094       ??_C@_03LBGABGKK@Jul@      0000000180003094     libucrt:nlsdata.obj
 0001:00002098       ??_C@_03IFJFEIGA@Aug@      0000000180003098     libucrt:nlsdata.obj
 0001:0000209c       ??_C@_03GGCAPAJC@Sep@      000000018000309c     libucrt:nlsdata.obj
 0001:000020a0       ??_C@_03BMAOKBAD@Oct@      00000001800030a0     libucrt:nlsdata.obj
 0001:000020a4       ??_C@_03JPJOFNIA@Nov@      00000001800030a4     libucrt:nlsdata.obj
 0001:000020a8       ??_C@_03MKABNOCG@Dec@      00000001800030a8     libucrt:nlsdata.obj
 0001:000020b0       ??_C@_07CGJPFGJA@January@  00000001800030b0     libucrt:nlsdata.obj
 0001:000020b8       ??_C@_08GNJGEPFN@February@ 00000001800030b8     libucrt:nlsdata.obj
 0001:000020c4       ??_C@_05HPCKOFNC@March@    00000001800030c4     libucrt:nlsdata.obj
 0001:000020cc       ??_C@_05DMJDNLEJ@April@    00000001800030cc     libucrt:nlsdata.obj
 0001:000020d4       ??_C@_04CNLMGBGM@June@     00000001800030d4     libucrt:nlsdata.obj
 0001:000020dc       ??_C@_04MIEPOIFP@July@     00000001800030dc     libucrt:nlsdata.obj
 0001:000020e4       ??_C@_06LBBHFDDG@August@   00000001800030e4     libucrt:nlsdata.obj
 0001:000020f0       ??_C@_09BHHEALKD@September@ 00000001800030f0     libucrt:nlsdata.obj
 0001:00002100       ??_C@_07JJNFCEND@October@  0000000180003100     libucrt:nlsdata.obj
 0001:00002108       ??_C@_08HCHEGEOA@November@ 0000000180003108     libucrt:nlsdata.obj
 0001:00002118       ??_C@_08EDHMEBNP@December@ 0000000180003118     libucrt:nlsdata.obj
 0001:00002124       ??_C@_02DEDBPAFC@AM@       0000000180003124     libucrt:nlsdata.obj
 0001:00002128       ??_C@_02CJNFDJBF@PM@       0000000180003128     libucrt:nlsdata.obj
 0001:00002130       ??_C@_08BPBNCDIB@MM?1dd?1yy@ 0000000180003130     libucrt:nlsdata.obj
 0001:00002140       ??_C@_0BE@CKGJFCPC@dddd?0?5MMMM?5dd?0?5yyyy@ 0000000180003140     libucrt:nlsdata.obj
 0001:00002158       ??_C@_08JCCMCCIL@HH?3mm?3ss@ 0000000180003158     libucrt:nlsdata.obj
 0001:00002168       ??_C@_17MBGCMIPB@?$AAS?$AAu?$AAn@ 0000000180003168     libucrt:nlsdata.obj
 0001:00002170       ??_C@_17KBOMKBF@?$AAM?$AAo?$AAn@ 0000000180003170     libucrt:nlsdata.obj
 0001:00002178       ??_C@_17BMKGEGOJ@?$AAT?$AAu?$AAe@ 0000000180003178     libucrt:nlsdata.obj
 0001:00002180       ??_C@_17CJEDCEPE@?$AAW?$AAe?$AAd@ 0000000180003180     libucrt:nlsdata.obj
 0001:00002188       ??_C@_17PDPHAADD@?$AAT?$AAh?$AAu@ 0000000180003188     libucrt:nlsdata.obj
 0001:00002190       ??_C@_17HFOLPPLP@?$AAF?$AAr?$AAi@ 0000000180003190     libucrt:nlsdata.obj
 0001:00002198       ??_C@_17GGIBDPIH@?$AAS?$AAa?$AAt@ 0000000180003198     libucrt:nlsdata.obj
 0001:000021a0       ??_C@_1O@IHNHDHPB@?$AAS?$AAu?$AAn?$AAd?$AAa?$AAy@ 00000001800031a0     libucrt:nlsdata.obj
 0001:000021b0       ??_C@_1O@MMNBFLIA@?$AAM?$AAo?$AAn?$AAd?$AAa?$AAy@ 00000001800031b0     libucrt:nlsdata.obj
 0001:000021c0       ??_C@_1BA@ENFBFFEK@?$AAT?$AAu?$AAe?$AAs?$AAd?$AAa?$AAy@ 00000001800031c0     libucrt:nlsdata.obj
 0001:000021d0       ??_C@_1BE@EBOGMDOH@?$AAW?$AAe?$AAd?$AAn?$AAe?$AAs?$AAd?$AAa?$AAy@ 00000001800031d0     libucrt:nlsdata.obj
 0001:000021e8       ??_C@_1BC@HHMNLIHE@?$AAT?$AAh?$AAu?$AAr?$AAs?$AAd?$AAa?$AAy@ 00000001800031e8     libucrt:nlsdata.obj
 0001:00002200       ??_C@_1O@PDICJHAG@?$AAF?$AAr?$AAi?$AAd?$AAa?$AAy@ 0000000180003200     libucrt:nlsdata.obj
 0001:00002210       ??_C@_1BC@ENMNNPAJ@?$AAS?$AAa?$AAt?$AAu?$AAr?$AAd?$AAa?$AAy@ 0000000180003210     libucrt:nlsdata.obj
 0001:00002228       ??_C@_17DKNBKCHM@?$AAJ?$AAa?$AAn@ 0000000180003228     libucrt:nlsdata.obj
 0001:00002230       ??_C@_17LMDJEKJN@?$AAF?$AAe?$AAb@ 0000000180003230     libucrt:nlsdata.obj
 0001:00002238       ??_C@_17CKNLEDEC@?$AAM?$AAa?$AAr@ 0000000180003238     libucrt:nlsdata.obj
 0001:00002240       ??_C@_17LFPOIHDD@?$AAA?$AAp?$AAr@ 0000000180003240     libucrt:nlsdata.obj
 0001:00002248       ??_C@_17PNNKMEED@?$AAM?$AAa?$AAy@ 0000000180003248     libucrt:nlsdata.obj
 0001:00002250       ??_C@_17KCJGOCPB@?$AAJ?$AAu?$AAn@ 0000000180003250     libucrt:nlsdata.obj
 0001:00002258       ??_C@_17IJPCKHK@?$AAJ?$AAu?$AAl@ 0000000180003258     libucrt:nlsdata.obj
 0001:00002260       ??_C@_17ICPELBCN@?$AAA?$AAu?$AAg@ 0000000180003260     libucrt:nlsdata.obj
 0001:00002268       ??_C@_17HCHCOKMG@?$AAS?$AAe?$AAp@ 0000000180003268     libucrt:nlsdata.obj
 0001:00002270       ??_C@_17FNLKOI@?$AAO?$AAc?$AAt@ 0000000180003270     libucrt:nlsdata.obj
 0001:00002278       ??_C@_17BBDMLCIG@?$AAN?$AAo?$AAv@ 0000000180003278     libucrt:nlsdata.obj
 0001:00002280       ??_C@_17EGKACKIF@?$AAD?$AAe?$AAc@ 0000000180003280     libucrt:nlsdata.obj
 0001:00002288       ??_C@_1BA@EFMEIEBA@?$AAJ?$AAa?$AAn?$AAu?$AAa?$AAr?$AAy@ 0000000180003288     libucrt:nlsdata.obj
 0001:00002298       ??_C@_1BC@JGDDFFAM@?$AAF?$AAe?$AAb?$AAr?$AAu?$AAa?$AAr?$AAy@ 0000000180003298     libucrt:nlsdata.obj
 0001:000022b0       ??_C@_1M@IKEENEDF@?$AAM?$AAa?$AAr?$AAc?$AAh@ 00000001800032b0     libucrt:nlsdata.obj
 0001:000022c0       ??_C@_1M@GJNLMHFD@?$AAA?$AAp?$AAr?$AAi?$AAl@ 00000001800032c0     libucrt:nlsdata.obj
 0001:000022d0       ??_C@_19EPFLPGAP@?$AAJ?$AAu?$AAn?$AAe@ 00000001800032d0     libucrt:nlsdata.obj
 0001:000022e0       ??_C@_19BIFMLPCD@?$AAJ?$AAu?$AAl?$AAy@ 00000001800032e0     libucrt:nlsdata.obj
 0001:000022f0       ??_C@_1O@PAHLKOAC@?$AAA?$AAu?$AAg?$AAu?$AAs?$AAt@ 00000001800032f0     libucrt:nlsdata.obj
 0001:00002300       ??_C@_1BE@DKAAMBJL@?$AAS?$AAe?$AAp?$AAt?$AAe?$AAm?$AAb?$AAe?$AAr@ 0000000180003300     libucrt:nlsdata.obj
 0001:00002318       ??_C@_1BA@EPANDLNG@?$AAO?$AAc?$AAt?$AAo?$AAb?$AAe?$AAr@ 0000000180003318     libucrt:nlsdata.obj
 0001:00002328       ??_C@_1BC@BGLIFPF@?$AAN?$AAo?$AAv?$AAe?$AAm?$AAb?$AAe?$AAr@ 0000000180003328     libucrt:nlsdata.obj
 0001:00002340       ??_C@_1BC@FEMKIFH@?$AAD?$AAe?$AAc?$AAe?$AAm?$AAb?$AAe?$AAr@ 0000000180003340     libucrt:nlsdata.obj
 0001:00002354       ??_C@_15ODEHAHHF@?$AAA?$AAM@ 0000000180003354     libucrt:nlsdata.obj
 0001:0000235c       ??_C@_15CLMNNGEL@?$AAP?$AAM@ 000000018000335c     libucrt:nlsdata.obj
 0001:00002368       ??_C@_1BC@IEBCMHCM@?$AAM?$AAM?$AA?1?$AAd?$AAd?$AA?1?$AAy?$AAy@ 0000000180003368     libucrt:nlsdata.obj
 0001:00002380       ??_C@_1CI@KNAKOEBC@?$AAd?$AAd?$AAd?$AAd?$AA?0?$AA?5?$AAM?$AAM?$AAM?$AAM?$AA?5?$AAd?$AAd?$AA?0?$AA?5@ 0000000180003380     libucrt:nlsdata.obj
 0001:000023a8       ??_C@_1BC@GDGBMEMK@?$AAH?$AAH?$AA?3?$AAm?$AAm?$AA?3?$AAs?$AAs@ 00000001800033a8     libucrt:nlsdata.obj
 0001:000023c0       ??_C@_1M@BMHNFIME@?$AAe?$AAn?$AA?9?$AAU?$AAS@ 00000001800033c0     libucrt:nlsdata.obj
 0001:000023d0       __newctype                 00000001800033d0     libucrt:ctype.obj
 0001:000026d0       __newclmap                 00000001800036d0     libucrt:ctype.obj
 0001:00002850       __newcumap                 0000000180003850     libucrt:ctype.obj
 0001:00003810       ??_C@_15EMKDOKLE@?$AAa?$AAr@ 0000000180004810     libucrt:lcidtoname_downlevel.obj
 0001:00003818       ??_C@_15KNPADPLH@?$AAb?$AAg@ 0000000180004818     libucrt:lcidtoname_downlevel.obj
 0001:00003820       ??_C@_15EDMHLDMO@?$AAc?$AAa@ 0000000180004820     libucrt:lcidtoname_downlevel.obj
 0001:00003828       ??_C@_1O@BPEAJADD@?$AAz?$AAh?$AA?9?$AAC?$AAH?$AAS@ 0000000180004828     libucrt:lcidtoname_downlevel.obj
 0001:00003838       ??_C@_15LJNHCMNK@?$AAc?$AAs@ 0000000180004838     libucrt:lcidtoname_downlevel.obj
 0001:00003840       ??_C@_15FOMCIDHG@?$AAd?$AAa@ 0000000180004840     libucrt:lcidtoname_downlevel.obj
 0001:00003848       ??_C@_15NBKABECB@?$AAd?$AAe@ 0000000180004848     libucrt:lcidtoname_downlevel.obj
 0001:00003850       ??_C@_15GHPEIIAO@?$AAe?$AAl@ 0000000180004850     libucrt:lcidtoname_downlevel.obj
 0001:00003858       ??_C@_15MNPNEAIF@?$AAe?$AAn@ 0000000180004858     libucrt:lcidtoname_downlevel.obj
 0001:00003860       ??_C@_15GPIOMPMH@?$AAe?$AAs@ 0000000180004860     libucrt:lcidtoname_downlevel.obj
 0001:00003868       ??_C@_15NGLOAKJC@?$AAf?$AAi@ 0000000180004868     libucrt:lcidtoname_downlevel.obj
 0001:00003870       ??_C@_15FBKGNKAM@?$AAf?$AAr@ 0000000180004870     libucrt:lcidtoname_downlevel.obj
 0001:00003878       ??_C@_15KGGCNEFK@?$AAh?$AAe@ 0000000180004878     libucrt:lcidtoname_downlevel.obj
 0001:00003880       ??_C@_15PGHLIDMF@?$AAh?$AAu@ 0000000180004880     libucrt:lcidtoname_downlevel.obj
 0001:00003888       ??_C@_15BIEMAPLM@?$AAi?$AAs@ 0000000180004888     libucrt:lcidtoname_downlevel.obj
 0001:00003890       ??_C@_15IFJLDHAF@?$AAi?$AAt@ 0000000180004890     libucrt:lcidtoname_downlevel.obj
 0001:00003898       ??_C@_15GEMIOCAG@?$AAj?$AAa@ 0000000180004898     libucrt:lcidtoname_downlevel.obj
 0001:000038a0       ??_C@_15EPELEGJA@?$AAk?$AAo@ 00000001800048a0     libucrt:lcidtoname_downlevel.obj
 0001:000038a8       ??_C@_15NDDHIMN@?$AAn?$AAl@ 00000001800048a8     libucrt:lcidtoname_downlevel.obj
 0001:000038b0       ??_C@_15BPIGNHCD@?$AAn?$AAo@ 00000001800048b0     libucrt:lcidtoname_downlevel.obj
 0001:000038b8       ??_C@_15DEOPBLCG@?$AAp?$AAl@ 00000001800048b8     libucrt:lcidtoname_downlevel.obj
 0001:000038c0       ??_C@_15KBECGEFG@?$AAp?$AAt@ 00000001800048c0     libucrt:lcidtoname_downlevel.obj
 0001:000038c8       ??_C@_15GLJCBFMD@?$AAr?$AAo@ 00000001800048c8     libucrt:lcidtoname_downlevel.obj
 0001:000038d0       ??_C@_15FEDGKCDI@?$AAr?$AAu@ 00000001800048d0     libucrt:lcidtoname_downlevel.obj
 0001:000038d8       ??_C@_15GLKMLLHM@?$AAh?$AAr@ 00000001800048d8     libucrt:lcidtoname_downlevel.obj
 0001:000038e0       ??_C@_15CPKMFBDB@?$AAs?$AAk@ 00000001800048e0     libucrt:lcidtoname_downlevel.obj
 0001:000038e8       ??_C@_15BAAIOGMK@?$AAs?$AAq@ 00000001800048e8     libucrt:lcidtoname_downlevel.obj
 0001:000038f0       ??_C@_15INNPNOHD@?$AAs?$AAv@ 00000001800048f0     libucrt:lcidtoname_downlevel.obj
 0001:000038f8       ??_C@_15CABMMOGH@?$AAt?$AAh@ 00000001800048f8     libucrt:lcidtoname_downlevel.obj
 0001:00003900       ??_C@_15BPLIHJJM@?$AAt?$AAr@ 0000000180004900     libucrt:lcidtoname_downlevel.obj
 0001:00003908       ??_C@_15NEOEKKDJ@?$AAu?$AAr@ 0000000180004908     libucrt:lcidtoname_downlevel.obj
 0001:00003910       ??_C@_15NFICGAJK@?$AAi?$AAd@ 0000000180004910     libucrt:lcidtoname_downlevel.obj
 0001:00003918       ??_C@_15PJPFLCCM@?$AAu?$AAk@ 0000000180004918     libucrt:lcidtoname_downlevel.obj
 0001:00003920       ??_C@_15HPJPHDM@?$AAb?$AAe@ 0000000180004920     libucrt:lcidtoname_downlevel.obj
 0001:00003928       ??_C@_15LCHLGJII@?$AAs?$AAl@ 0000000180004928     libucrt:lcidtoname_downlevel.obj
 0001:00003930       ??_C@_15PCFJPHHO@?$AAe?$AAt@ 0000000180004930     libucrt:lcidtoname_downlevel.obj
 0001:00003938       ??_C@_15HPFPGODN@?$AAl?$AAv@ 0000000180004938     libucrt:lcidtoname_downlevel.obj
 0001:00003940       ??_C@_15NFFGKGLG@?$AAl?$AAt@ 0000000180004940     libucrt:lcidtoname_downlevel.obj
 0001:00003948       ??_C@_15BDAKCCHN@?$AAf?$AAa@ 0000000180004948     libucrt:lcidtoname_downlevel.obj
 0001:00003950       ??_C@_15NFGIAIAJ@?$AAv?$AAi@ 0000000180004950     libucrt:lcidtoname_downlevel.obj
 0001:00003958       ??_C@_15LMKNDMHN@?$AAh?$AAy@ 0000000180004958     libucrt:lcidtoname_downlevel.obj
 0001:00003960       ??_C@_15IJBHMCFL@?$AAa?$AAz@ 0000000180004960     libucrt:lcidtoname_downlevel.obj
 0001:00003968       ??_C@_15EKOFJABL@?$AAe?$AAu@ 0000000180004968     libucrt:lcidtoname_downlevel.obj
 0001:00003970       ??_C@_15BGHADCNK@?$AAm?$AAk@ 0000000180004970     libucrt:lcidtoname_downlevel.obj
 0001:00003978       ??_C@_15JDNICKHM@?$AAa?$AAf@ 0000000180004978     libucrt:lcidtoname_downlevel.obj
 0001:00003980       ??_C@_15KPJEDBKD@?$AAk?$AAa@ 0000000180004980     libucrt:lcidtoname_downlevel.obj
 0001:00003988       ??_C@_15PDNFFFEO@?$AAf?$AAo@ 0000000180004988     libucrt:lcidtoname_downlevel.obj
 0001:00003990       ??_C@_15OMLEGLOC@?$AAh?$AAi@ 0000000180004990     libucrt:lcidtoname_downlevel.obj
 0001:00003998       ??_C@_15IDNNENKK@?$AAm?$AAs@ 0000000180004998     libucrt:lcidtoname_downlevel.obj
 0001:000039a0       ??_C@_15MACJNBMH@?$AAk?$AAk@ 00000001800049a0     libucrt:lcidtoname_downlevel.obj
 0001:000039a8       ??_C@_15DKDJEOND@?$AAk?$AAy@ 00000001800049a8     libucrt:lcidtoname_downlevel.obj
 0001:000039b0       ??_C@_15DFGDLJBG@?$AAs?$AAw@ 00000001800049b0     libucrt:lcidtoname_downlevel.obj
 0001:000039b8       ??_C@_15BBFAICNG@?$AAu?$AAz@ 00000001800049b8     libucrt:lcidtoname_downlevel.obj
 0001:000039c0       ??_C@_15DKNDCGEA@?$AAt?$AAt@ 00000001800049c0     libucrt:lcidtoname_downlevel.obj
 0001:000039c8       ??_C@_15MGIFMDPL@?$AAp?$AAa@ 00000001800049c8     libucrt:lcidtoname_downlevel.obj
 0001:000039d0       ??_C@_15HCNDBBA@?$AAg?$AAu@ 00000001800049d0     libucrt:lcidtoname_downlevel.obj
 0001:000039d8       ??_C@_15FNBEIBON@?$AAt?$AAa@ 00000001800049d8     libucrt:lcidtoname_downlevel.obj
 0001:000039e0       ??_C@_15NCHGBGLK@?$AAt?$AAe@ 00000001800049e0     libucrt:lcidtoname_downlevel.obj
 0001:000039e8       ??_C@_15PHPHCBPF@?$AAk?$AAn@ 00000001800049e8     libucrt:lcidtoname_downlevel.obj
 0001:000039f0       ??_C@_15DLGBCKMP@?$AAm?$AAr@ 00000001800049f0     libucrt:lcidtoname_downlevel.obj
 0001:000039f8       ??_C@_15EABBLBFF@?$AAs?$AAa@ 00000001800049f8     libucrt:lcidtoname_downlevel.obj
 0001:00003a00       ??_C@_15CBKOMCOI@?$AAm?$AAn@ 0000000180004a00     libucrt:lcidtoname_downlevel.obj
 0001:00003a08       ??_C@_15CKDMCJAF@?$AAg?$AAl@ 0000000180004a08     libucrt:lcidtoname_downlevel.obj
 0001:00003a10       ??_C@_17CNJFBPG@?$AAk?$AAo?$AAk@ 0000000180004a10     libucrt:lcidtoname_downlevel.obj
 0001:00003a18       ??_C@_17FFBJICPL@?$AAs?$AAy?$AAr@ 0000000180004a18     libucrt:lcidtoname_downlevel.obj
 0001:00003a20       ??_C@_17KPNDCPAF@?$AAd?$AAi?$AAv@ 0000000180004a20     libucrt:lcidtoname_downlevel.obj
 0001:00003a28       ??_C@_1M@OKAHONE@?$AAa?$AAr?$AA?9?$AAS?$AAA@ 0000000180004a28     libucrt:lcidtoname_downlevel.obj
 0001:00003a38       ??_C@_1M@FFFIGIGK@?$AAb?$AAg?$AA?9?$AAB?$AAG@ 0000000180004a38     libucrt:lcidtoname_downlevel.obj
 0001:00003a48       ??_C@_1M@BJNKEDC@?$AAc?$AAa?$AA?9?$AAE?$AAS@ 0000000180004a48     libucrt:lcidtoname_downlevel.obj
 0001:00003a58       ??_C@_1M@IJJHFJHA@?$AAc?$AAs?$AA?9?$AAC?$AAZ@ 0000000180004a58     libucrt:lcidtoname_downlevel.obj
 0001:00003a68       ??_C@_1M@CLPEOBGI@?$AAd?$AAa?$AA?9?$AAD?$AAK@ 0000000180004a68     libucrt:lcidtoname_downlevel.obj
 0001:00003a78       ??_C@_1M@MCMADGCB@?$AAd?$AAe?$AA?9?$AAD?$AAE@ 0000000180004a78     libucrt:lcidtoname_downlevel.obj
 0001:00003a88       ??_C@_1M@OOCKEMAM@?$AAe?$AAl?$AA?9?$AAG?$AAR@ 0000000180004a88     libucrt:lcidtoname_downlevel.obj
 0001:00003a98       ??_C@_1M@DDNJFGID@?$AAf?$AAi?$AA?9?$AAF?$AAI@ 0000000180004a98     libucrt:lcidtoname_downlevel.obj
 0001:00003aa8       ??_C@_1M@GLIPPMAC@?$AAf?$AAr?$AA?9?$AAF?$AAR@ 0000000180004aa8     libucrt:lcidtoname_downlevel.obj
 0001:00003ab8       ??_C@_1M@GFMCHPE@?$AAh?$AAe?$AA?9?$AAI?$AAL@ 0000000180004ab8     libucrt:lcidtoname_downlevel.obj
 0001:00003ac8       ??_C@_1M@MHLPGNKM@?$AAh?$AAu?$AA?9?$AAH?$AAU@ 0000000180004ac8     libucrt:lcidtoname_downlevel.obj
 0001:00003ad8       ??_C@_1M@LPDDNNPN@?$AAi?$AAs?$AA?9?$AAI?$AAS@ 0000000180004ad8     libucrt:lcidtoname_downlevel.obj
 0001:00003ae8       ??_C@_1M@MADIPODN@?$AAi?$AAt?$AA?9?$AAI?$AAT@ 0000000180004ae8     libucrt:lcidtoname_downlevel.obj
 0001:00003af8       ??_C@_1M@IHBJJGG@?$AAn?$AAl?$AA?9?$AAN?$AAL@ 0000000180004af8     libucrt:lcidtoname_downlevel.obj
 0001:00003b08       ??_C@_1M@EANAGDL@?$AAn?$AAb?$AA?9?$AAN?$AAO@ 0000000180004b08     libucrt:lcidtoname_downlevel.obj
 0001:00003b18       ??_C@_1M@NEIEMEGP@?$AAp?$AAl?$AA?9?$AAP?$AAL@ 0000000180004b18     libucrt:lcidtoname_downlevel.obj
 0001:00003b28       ??_C@_1M@BOCFIGEP@?$AAp?$AAt?$AA?9?$AAB?$AAR@ 0000000180004b28     libucrt:lcidtoname_downlevel.obj
 0001:00003b38       ??_C@_1M@IMPFOPBG@?$AAr?$AAo?$AA?9?$AAR?$AAO@ 0000000180004b38     libucrt:lcidtoname_downlevel.obj
 0001:00003b48       ??_C@_1M@IDNNEJMM@?$AAr?$AAu?$AA?9?$AAR?$AAU@ 0000000180004b48     libucrt:lcidtoname_downlevel.obj
 0001:00003b58       ??_C@_1M@LILEEOGM@?$AAh?$AAr?$AA?9?$AAH?$AAR@ 0000000180004b58     libucrt:lcidtoname_downlevel.obj
 0001:00003b68       ??_C@_1M@FKIFEHPB@?$AAs?$AAk?$AA?9?$AAS?$AAK@ 0000000180004b68     libucrt:lcidtoname_downlevel.obj
 0001:00003b78       ??_C@_1M@LJMAMNPJ@?$AAs?$AAq?$AA?9?$AAA?$AAL@ 0000000180004b78     libucrt:lcidtoname_downlevel.obj
 0001:00003b88       ??_C@_1M@GIAKDKJK@?$AAs?$AAv?$AA?9?$AAS?$AAE@ 0000000180004b88     libucrt:lcidtoname_downlevel.obj
 0001:00003b98       ??_C@_1M@MKJKIKCL@?$AAt?$AAh?$AA?9?$AAT?$AAH@ 0000000180004b98     libucrt:lcidtoname_downlevel.obj
 0001:00003ba8       ??_C@_1M@MFLCCMPB@?$AAt?$AAr?$AA?9?$AAT?$AAR@ 0000000180004ba8     libucrt:lcidtoname_downlevel.obj
 0001:00003bb8       ??_C@_1M@OIJHDKJN@?$AAu?$AAr?$AA?9?$AAP?$AAK@ 0000000180004bb8     libucrt:lcidtoname_downlevel.obj
 0001:00003bc8       ??_C@_1M@LHIPCIEK@?$AAi?$AAd?$AA?9?$AAI?$AAD@ 0000000180004bc8     libucrt:lcidtoname_downlevel.obj
 0001:00003bd8       ??_C@_1M@MFMOBGI@?$AAu?$AAk?$AA?9?$AAU?$AAA@ 0000000180004bd8     libucrt:lcidtoname_downlevel.obj
 0001:00003be8       ??_C@_1M@OBGLJIPL@?$AAb?$AAe?$AA?9?$AAB?$AAY@ 0000000180004be8     libucrt:lcidtoname_downlevel.obj
 0001:00003bf8       ??_C@_1M@BCFAJEAD@?$AAs?$AAl?$AA?9?$AAS?$AAI@ 0000000180004bf8     libucrt:lcidtoname_downlevel.obj
 0001:00003c08       ??_C@_1M@FKFFEDDN@?$AAe?$AAt?$AA?9?$AAE?$AAE@ 0000000180004c08     libucrt:lcidtoname_downlevel.obj
 0001:00003c18       ??_C@_1M@KGKKAACI@?$AAl?$AAv?$AA?9?$AAL?$AAV@ 0000000180004c18     libucrt:lcidtoname_downlevel.obj
 0001:00003c28       ??_C@_1M@IFGBIJO@?$AAl?$AAt?$AA?9?$AAL?$AAT@ 0000000180004c28     libucrt:lcidtoname_downlevel.obj
 0001:00003c38       ??_C@_1M@FGEAHEDM@?$AAf?$AAa?$AA?9?$AAI?$AAR@ 0000000180004c38     libucrt:lcidtoname_downlevel.obj
 0001:00003c48       ??_C@_1M@KBMAIBFN@?$AAv?$AAi?$AA?9?$AAV?$AAN@ 0000000180004c48     libucrt:lcidtoname_downlevel.obj
 0001:00003c58       ??_C@_1M@GPCBKDJK@?$AAh?$AAy?$AA?9?$AAA?$AAM@ 0000000180004c58     libucrt:lcidtoname_downlevel.obj
 0001:00003c68       ??_C@_1BG@BECMDDJB@?$AAa?$AAz?$AA?9?$AAA?$AAZ?$AA?9?$AAL?$AAa?$AAt?$AAn@ 0000000180004c68     libucrt:lcidtoname_downlevel.obj
 0001:00003c80       ??_C@_1M@MAOFCAEA@?$AAe?$AAu?$AA?9?$AAE?$AAS@ 0000000180004c80     libucrt:lcidtoname_downlevel.obj
 0001:00003c90       ??_C@_1M@IGHABKPI@?$AAm?$AAk?$AA?9?$AAM?$AAK@ 0000000180004c90     libucrt:lcidtoname_downlevel.obj
 0001:00003ca0       ??_C@_1M@IAIGNEJG@?$AAt?$AAn?$AA?9?$AAZ?$AAA@ 0000000180004ca0     libucrt:lcidtoname_downlevel.obj
 0001:00003cb0       ??_C@_1M@IIJCOJFA@?$AAx?$AAh?$AA?9?$AAZ?$AAA@ 0000000180004cb0     libucrt:lcidtoname_downlevel.obj
 0001:00003cc0       ??_C@_1M@LGPJHNJH@?$AAz?$AAu?$AA?9?$AAZ?$AAA@ 0000000180004cc0     libucrt:lcidtoname_downlevel.obj
 0001:00003cd0       ??_C@_1M@HOKAOIO@?$AAa?$AAf?$AA?9?$AAZ?$AAA@ 0000000180004cd0     libucrt:lcidtoname_downlevel.obj
 0001:00003ce0       ??_C@_1M@DPCLHLIE@?$AAk?$AAa?$AA?9?$AAG?$AAE@ 0000000180004ce0     libucrt:lcidtoname_downlevel.obj
 0001:00003cf0       ??_C@_1M@BLKMHJBI@?$AAf?$AAo?$AA?9?$AAF?$AAO@ 0000000180004cf0     libucrt:lcidtoname_downlevel.obj
 0001:00003d00       ??_C@_1M@LGGJAPPB@?$AAh?$AAi?$AA?9?$AAI?$AAN@ 0000000180004d00     libucrt:lcidtoname_downlevel.obj
 0001:00003d10       ??_C@_1M@FIKPIHFE@?$AAm?$AAt?$AA?9?$AAM?$AAT@ 0000000180004d10     libucrt:lcidtoname_downlevel.obj
 0001:00003d20       ??_C@_1M@HEGGPBFA@?$AAs?$AAe?$AA?9?$AAN?$AAO@ 0000000180004d20     libucrt:lcidtoname_downlevel.obj
 0001:00003d30       ??_C@_1M@EIBJEEPA@?$AAm?$AAs?$AA?9?$AAM?$AAY@ 0000000180004d30     libucrt:lcidtoname_downlevel.obj
 0001:00003d40       ??_C@_1M@FHLBGMPP@?$AAk?$AAk?$AA?9?$AAK?$AAZ@ 0000000180004d40     libucrt:lcidtoname_downlevel.obj
 0001:00003d50       ??_C@_1M@NGJJLCGI@?$AAk?$AAy?$AA?9?$AAK?$AAG@ 0000000180004d50     libucrt:lcidtoname_downlevel.obj
 0001:00003d60       ??_C@_1M@GIENNBFC@?$AAs?$AAw?$AA?9?$AAK?$AAE@ 0000000180004d60     libucrt:lcidtoname_downlevel.obj
 0001:00003d70       ??_C@_1BG@NDGMJIMJ@?$AAu?$AAz?$AA?9?$AAU?$AAZ?$AA?9?$AAL?$AAa?$AAt?$AAn@ 0000000180004d70     libucrt:lcidtoname_downlevel.obj
 0001:00003d88       ??_C@_1M@IDCCIHBC@?$AAt?$AAt?$AA?9?$AAR?$AAU@ 0000000180004d88     libucrt:lcidtoname_downlevel.obj
 0001:00003d98       ??_C@_1M@LOICPMOJ@?$AAb?$AAn?$AA?9?$AAI?$AAN@ 0000000180004d98     libucrt:lcidtoname_downlevel.obj
 0001:00003da8       ??_C@_1M@KPKKNEAH@?$AAp?$AAa?$AA?9?$AAI?$AAN@ 0000000180004da8     libucrt:lcidtoname_downlevel.obj
 0001:00003db8       ??_C@_1M@PJGPPBOG@?$AAg?$AAu?$AA?9?$AAI?$AAN@ 0000000180004db8     libucrt:lcidtoname_downlevel.obj
 0001:00003dc8       ??_C@_1M@KMKMOPHI@?$AAt?$AAa?$AA?9?$AAI?$AAN@ 0000000180004dc8     libucrt:lcidtoname_downlevel.obj
 0001:00003dd8       ??_C@_1M@KFEHEPAC@?$AAt?$AAe?$AA?9?$AAI?$AAN@ 0000000180004dd8     libucrt:lcidtoname_downlevel.obj
 0001:00003de8       ??_C@_1M@CDCLMGHI@?$AAk?$AAn?$AA?9?$AAI?$AAN@ 0000000180004de8     libucrt:lcidtoname_downlevel.obj
 0001:00003df8       ??_C@_1M@MIODLDKF@?$AAm?$AAl?$AA?9?$AAI?$AAN@ 0000000180004df8     libucrt:lcidtoname_downlevel.obj
 0001:00003e08       ??_C@_1M@PBIEACPO@?$AAm?$AAr?$AA?9?$AAI?$AAN@ 0000000180004e08     libucrt:lcidtoname_downlevel.obj
 0001:00003e18       ??_C@_1M@NIDEAGPH@?$AAs?$AAa?$AA?9?$AAI?$AAN@ 0000000180004e18     libucrt:lcidtoname_downlevel.obj
 0001:00003e28       ??_C@_1M@FHIHCBIO@?$AAm?$AAn?$AA?9?$AAM?$AAN@ 0000000180004e28     libucrt:lcidtoname_downlevel.obj
 0001:00003e38       ??_C@_1M@JAIJPENP@?$AAc?$AAy?$AA?9?$AAG?$AAB@ 0000000180004e38     libucrt:lcidtoname_downlevel.obj
 0001:00003e48       ??_C@_1M@PHGFBEPN@?$AAg?$AAl?$AA?9?$AAE?$AAS@ 0000000180004e48     libucrt:lcidtoname_downlevel.obj
 0001:00003e58       ??_C@_1O@KPIPDNCP@?$AAk?$AAo?$AAk?$AA?9?$AAI?$AAN@ 0000000180004e58     libucrt:lcidtoname_downlevel.obj
 0001:00003e68       ??_C@_1O@KNHJLDJA@?$AAs?$AAy?$AAr?$AA?9?$AAS?$AAY@ 0000000180004e68     libucrt:lcidtoname_downlevel.obj
 0001:00003e78       ??_C@_1O@MKEKBLAH@?$AAd?$AAi?$AAv?$AA?9?$AAM?$AAV@ 0000000180004e78     libucrt:lcidtoname_downlevel.obj
 0001:00003e88       ??_C@_1O@OHDCKDDF@?$AAq?$AAu?$AAz?$AA?9?$AAB?$AAO@ 0000000180004e88     libucrt:lcidtoname_downlevel.obj
 0001:00003e98       ??_C@_1M@LEPJNLFD@?$AAn?$AAs?$AA?9?$AAZ?$AAA@ 0000000180004e98     libucrt:lcidtoname_downlevel.obj
 0001:00003ea8       ??_C@_1M@OMLEIIJB@?$AAm?$AAi?$AA?9?$AAN?$AAZ@ 0000000180004ea8     libucrt:lcidtoname_downlevel.obj
 0001:00003eb8       ??_C@_1M@PMPEAILG@?$AAa?$AAr?$AA?9?$AAI?$AAQ@ 0000000180004eb8     libucrt:lcidtoname_downlevel.obj
 0001:00003ec8       ??_C@_1M@CNKPNOEE@?$AAd?$AAe?$AA?9?$AAC?$AAH@ 0000000180004ec8     libucrt:lcidtoname_downlevel.obj
 0001:00003ed8       ??_C@_1M@LKMGMLKO@?$AAe?$AAn?$AA?9?$AAG?$AAB@ 0000000180004ed8     libucrt:lcidtoname_downlevel.obj
 0001:00003ee8       ??_C@_1M@PGKJFFGL@?$AAe?$AAs?$AA?9?$AAM?$AAX@ 0000000180004ee8     libucrt:lcidtoname_downlevel.obj
 0001:00003ef8       ??_C@_1M@DNNANBDC@?$AAf?$AAr?$AA?9?$AAB?$AAE@ 0000000180004ef8     libucrt:lcidtoname_downlevel.obj
 0001:00003f08       ??_C@_1M@HLGMDFHM@?$AAi?$AAt?$AA?9?$AAC?$AAH@ 0000000180004f08     libucrt:lcidtoname_downlevel.obj
 0001:00003f18       ??_C@_1M@CLLBGJH@?$AAn?$AAl?$AA?9?$AAB?$AAE@ 0000000180004f18     libucrt:lcidtoname_downlevel.obj
 0001:00003f28       ??_C@_1M@BODBOGLF@?$AAn?$AAn?$AA?9?$AAN?$AAO@ 0000000180004f28     libucrt:lcidtoname_downlevel.obj
 0001:00003f38       ??_C@_1M@HFFAHKAD@?$AAp?$AAt?$AA?9?$AAP?$AAT@ 0000000180004f38     libucrt:lcidtoname_downlevel.obj
 0001:00003f48       ??_C@_1BG@LNOAKHIE@?$AAs?$AAr?$AA?9?$AAS?$AAP?$AA?9?$AAL?$AAa?$AAt?$AAn@ 0000000180004f48     libucrt:lcidtoname_downlevel.obj
 0001:00003f60       ??_C@_1M@HBMHBGAK@?$AAs?$AAv?$AA?9?$AAF?$AAI@ 0000000180004f60     libucrt:lcidtoname_downlevel.obj
 0001:00003f70       ??_C@_1BG@DGCJGJBE@?$AAa?$AAz?$AA?9?$AAA?$AAZ?$AA?9?$AAC?$AAy?$AAr?$AAl@ 0000000180004f70     libucrt:lcidtoname_downlevel.obj
 0001:00003f88       ??_C@_1M@KEJDAAHB@?$AAs?$AAe?$AA?9?$AAS?$AAE@ 0000000180004f88     libucrt:lcidtoname_downlevel.obj
 0001:00003f98       ??_C@_1M@HEIBJJAD@?$AAm?$AAs?$AA?9?$AAB?$AAN@ 0000000180004f98     libucrt:lcidtoname_downlevel.obj
 0001:00003fa8       ??_C@_1BG@PBGJMCEM@?$AAu?$AAz?$AA?9?$AAU?$AAZ?$AA?9?$AAC?$AAy?$AAr?$AAl@ 0000000180004fa8     libucrt:lcidtoname_downlevel.obj
 0001:00003fc0       ??_C@_1O@LAOBCMDF@?$AAq?$AAu?$AAz?$AA?9?$AAE?$AAC@ 0000000180004fc0     libucrt:lcidtoname_downlevel.obj
 0001:00003fd0       ??_C@_1M@POEEMAIO@?$AAa?$AAr?$AA?9?$AAE?$AAG@ 0000000180004fd0     libucrt:lcidtoname_downlevel.obj
 0001:00003fe0       ??_C@_1M@EFAKDEDL@?$AAz?$AAh?$AA?9?$AAH?$AAK@ 0000000180004fe0     libucrt:lcidtoname_downlevel.obj
 0001:00003ff0       ??_C@_1M@HKKIJHGI@?$AAd?$AAe?$AA?9?$AAA?$AAT@ 0000000180004ff0     libucrt:lcidtoname_downlevel.obj
 0001:00004000       ??_C@_1M@KBFBEHJF@?$AAe?$AAn?$AA?9?$AAA?$AAU@ 0000000180005000     libucrt:lcidtoname_downlevel.obj
 0001:00004010       ??_C@_1M@MNPLFAAH@?$AAe?$AAs?$AA?9?$AAE?$AAS@ 0000000180005010     libucrt:lcidtoname_downlevel.obj
 0001:00004020       ??_C@_1M@HJOOJFMA@?$AAf?$AAr?$AA?9?$AAC?$AAA@ 0000000180005020     libucrt:lcidtoname_downlevel.obj
 0001:00004030       ??_C@_1BG@JPOFPNAB@?$AAs?$AAr?$AA?9?$AAS?$AAP?$AA?9?$AAC?$AAy?$AAr?$AAl@ 0000000180005030     libucrt:lcidtoname_downlevel.obj
 0001:00004048       ??_C@_1M@LNFOCMOB@?$AAs?$AAe?$AA?9?$AAF?$AAI@ 0000000180005048     libucrt:lcidtoname_downlevel.obj
 0001:00004058       ??_C@_1O@MGJBOAMB@?$AAq?$AAu?$AAz?$AA?9?$AAP?$AAE@ 0000000180005058     libucrt:lcidtoname_downlevel.obj
 0001:00004068       ??_C@_1M@GJINLBOK@?$AAa?$AAr?$AA?9?$AAL?$AAY@ 0000000180005068     libucrt:lcidtoname_downlevel.obj
 0001:00004078       ??_C@_1M@GGMNHJNL@?$AAz?$AAh?$AA?9?$AAS?$AAG@ 0000000180005078     libucrt:lcidtoname_downlevel.obj
 0001:00004088       ??_C@_1M@HOIKODND@?$AAd?$AAe?$AA?9?$AAL?$AAU@ 0000000180005088     libucrt:lcidtoname_downlevel.obj
 0001:00004098       ??_C@_1M@DDOCCGFG@?$AAe?$AAn?$AA?9?$AAC?$AAA@ 0000000180005098     libucrt:lcidtoname_downlevel.obj
 0001:000040a8       ??_C@_1M@BNOEMJLF@?$AAe?$AAs?$AA?9?$AAG?$AAT@ 00000001800050a8     libucrt:lcidtoname_downlevel.obj
 0001:000040b8       ??_C@_1M@EOGNKEK@?$AAf?$AAr?$AA?9?$AAC?$AAH@ 00000001800050b8     libucrt:lcidtoname_downlevel.obj
 0001:000040c8       ??_C@_1M@FLIDJFHL@?$AAh?$AAr?$AA?9?$AAB?$AAA@ 00000001800050c8     libucrt:lcidtoname_downlevel.obj
 0001:000040d8       ??_C@_1O@FMCELNAJ@?$AAs?$AAm?$AAj?$AA?9?$AAN?$AAO@ 00000001800050d8     libucrt:lcidtoname_downlevel.obj
 0001:000040e8       ??_C@_1M@JHGLJMGJ@?$AAa?$AAr?$AA?9?$AAD?$AAZ@ 00000001800050e8     libucrt:lcidtoname_downlevel.obj
 0001:000040f8       ??_C@_1M@JKKFDCNP@?$AAz?$AAh?$AA?9?$AAM?$AAO@ 00000001800050f8     libucrt:lcidtoname_downlevel.obj
 0001:00004108       ??_C@_1M@GEEFALPE@?$AAd?$AAe?$AA?9?$AAL?$AAI@ 0000000180005108     libucrt:lcidtoname_downlevel.obj
 0001:00004118       ??_C@_1M@IGEOFBG@?$AAe?$AAn?$AA?9?$AAN?$AAZ@ 0000000180005118     libucrt:lcidtoname_downlevel.obj
 0001:00004128       ??_C@_1M@KDBONEHP@?$AAe?$AAs?$AA?9?$AAC?$AAR@ 0000000180005128     libucrt:lcidtoname_downlevel.obj
 0001:00004138       ??_C@_1M@FHMDOHNN@?$AAf?$AAr?$AA?9?$AAL?$AAU@ 0000000180005138     libucrt:lcidtoname_downlevel.obj
 0001:00004148       ??_C@_1BG@NFKKMAFG@?$AAb?$AAs?$AA?9?$AAB?$AAA?$AA?9?$AAL?$AAa?$AAt?$AAn@ 0000000180005148     libucrt:lcidtoname_downlevel.obj
 0001:00004160       ??_C@_1O@IMNBEMCI@?$AAs?$AAm?$AAj?$AA?9?$AAS?$AAE@ 0000000180005160     libucrt:lcidtoname_downlevel.obj
 0001:00004170       ??_C@_1M@DHHMBNDP@?$AAa?$AAr?$AA?9?$AAM?$AAA@ 0000000180005170     libucrt:lcidtoname_downlevel.obj
 0001:00004180       ??_C@_1M@BNBLJCGH@?$AAe?$AAn?$AA?9?$AAI?$AAE@ 0000000180005180     libucrt:lcidtoname_downlevel.obj
 0001:00004190       ??_C@_1M@GEPAFMDL@?$AAe?$AAs?$AA?9?$AAP?$AAA@ 0000000180005190     libucrt:lcidtoname_downlevel.obj
 0001:000041a0       ??_C@_1M@OJONDMDL@?$AAf?$AAr?$AA?9?$AAM?$AAC@ 00000001800051a0     libucrt:lcidtoname_downlevel.obj
 0001:000041b0       ??_C@_1BG@OBCNFJB@?$AAs?$AAr?$AA?9?$AAB?$AAA?$AA?9?$AAL?$AAa?$AAt?$AAn@ 00000001800051b0     libucrt:lcidtoname_downlevel.obj
 0001:000041c8       ??_C@_1O@KEMEEGPO@?$AAs?$AAm?$AAa?$AA?9?$AAN?$AAO@ 00000001800051c8     libucrt:lcidtoname_downlevel.obj
 0001:000041d8       ??_C@_1M@ELMGFODK@?$AAa?$AAr?$AA?9?$AAT?$AAN@ 00000001800051d8     libucrt:lcidtoname_downlevel.obj
 0001:000041e8       ??_C@_1M@BHDLHFAF@?$AAe?$AAn?$AA?9?$AAZ?$AAA@ 00000001800051e8     libucrt:lcidtoname_downlevel.obj
 0001:000041f8       ??_C@_1M@BMGIGLIF@?$AAe?$AAs?$AA?9?$AAD?$AAO@ 00000001800051f8     libucrt:lcidtoname_downlevel.obj
 0001:00004208       ??_C@_1BG@CMBHIPBE@?$AAs?$AAr?$AA?9?$AAB?$AAA?$AA?9?$AAC?$AAy?$AAr?$AAl@ 0000000180005208     libucrt:lcidtoname_downlevel.obj
 0001:00004220       ??_C@_1O@HEDBLHNP@?$AAs?$AAm?$AAa?$AA?9?$AAS?$AAE@ 0000000180005220     libucrt:lcidtoname_downlevel.obj
 0001:00004230       ??_C@_1M@DAGCADIM@?$AAa?$AAr?$AA?9?$AAO?$AAM@ 0000000180005230     libucrt:lcidtoname_downlevel.obj
 0001:00004240       ??_C@_1M@FODLMICG@?$AAe?$AAn?$AA?9?$AAJ?$AAM@ 0000000180005240     libucrt:lcidtoname_downlevel.obj
 0001:00004250       ??_C@_1M@DNMLCIHB@?$AAe?$AAs?$AA?9?$AAV?$AAE@ 0000000180005250     libucrt:lcidtoname_downlevel.obj
 0001:00004260       ??_C@_1O@EOKHMKJK@?$AAs?$AAm?$AAs?$AA?9?$AAF?$AAI@ 0000000180005260     libucrt:lcidtoname_downlevel.obj
 0001:00004270       ??_C@_1M@CAFJMKOF@?$AAa?$AAr?$AA?9?$AAY?$AAE@ 0000000180005270     libucrt:lcidtoname_downlevel.obj
 0001:00004280       ??_C@_1M@CBFHIJLI@?$AAe?$AAn?$AA?9?$AAC?$AAB@ 0000000180005280     libucrt:lcidtoname_downlevel.obj
 0001:00004290       ??_C@_1M@BGNFLDN@?$AAe?$AAs?$AA?9?$AAC?$AAO@ 0000000180005290     libucrt:lcidtoname_downlevel.obj
 0001:000042a0       ??_C@_1O@JMPHMAMC@?$AAs?$AAm?$AAn?$AA?9?$AAF?$AAI@ 00000001800052a0     libucrt:lcidtoname_downlevel.obj
 0001:000042b0       ??_C@_1M@JLANABKE@?$AAa?$AAr?$AA?9?$AAS?$AAY@ 00000001800052b0     libucrt:lcidtoname_downlevel.obj
 0001:000042c0       ??_C@_1M@HPKGCFGN@?$AAe?$AAn?$AA?9?$AAB?$AAZ@ 00000001800052c0     libucrt:lcidtoname_downlevel.obj
 0001:000042d0       ??_C@_1M@OLJCMLGM@?$AAe?$AAs?$AA?9?$AAP?$AAE@ 00000001800052d0     libucrt:lcidtoname_downlevel.obj
 0001:000042e0       ??_C@_1M@MKKGFKLE@?$AAa?$AAr?$AA?9?$AAJ?$AAO@ 00000001800052e0     libucrt:lcidtoname_downlevel.obj
 0001:000042f0       ??_C@_1M@EKPGLDNI@?$AAe?$AAn?$AA?9?$AAT?$AAT@ 00000001800052f0     libucrt:lcidtoname_downlevel.obj
 0001:00004300       ??_C@_1M@OONGHFHE@?$AAe?$AAs?$AA?9?$AAA?$AAR@ 0000000180005300     libucrt:lcidtoname_downlevel.obj
 0001:00004310       ??_C@_1M@OOJFGBHE@?$AAa?$AAr?$AA?9?$AAL?$AAB@ 0000000180005310     libucrt:lcidtoname_downlevel.obj
 0001:00004320       ??_C@_1M@GCEJHNEG@?$AAe?$AAn?$AA?9?$AAZ?$AAW@ 0000000180005320     libucrt:lcidtoname_downlevel.obj
 0001:00004330       ??_C@_1M@JNOCAHJI@?$AAe?$AAs?$AA?9?$AAE?$AAC@ 0000000180005330     libucrt:lcidtoname_downlevel.obj
 0001:00004340       ??_C@_1M@JEFHPGGB@?$AAa?$AAr?$AA?9?$AAK?$AAW@ 0000000180005340     libucrt:lcidtoname_downlevel.obj
 0001:00004350       ??_C@_1M@MLKIBJOJ@?$AAe?$AAn?$AA?9?$AAP?$AAH@ 0000000180005350     libucrt:lcidtoname_downlevel.obj
 0001:00004360       ??_C@_1M@BDNIPEND@?$AAe?$AAs?$AA?9?$AAC?$AAL@ 0000000180005360     libucrt:lcidtoname_downlevel.obj
 0001:00004370       ??_C@_1M@MPNMEKBD@?$AAa?$AAr?$AA?9?$AAA?$AAE@ 0000000180005370     libucrt:lcidtoname_downlevel.obj
 0001:00004380       ??_C@_1M@KBJALCPI@?$AAe?$AAs?$AA?9?$AAU?$AAY@ 0000000180005380     libucrt:lcidtoname_downlevel.obj
 0001:00004390       ??_C@_1M@LLCCOAGA@?$AAa?$AAr?$AA?9?$AAB?$AAH@ 0000000180005390     libucrt:lcidtoname_downlevel.obj
 0001:000043a0       ??_C@_1M@PBFNCDEL@?$AAe?$AAs?$AA?9?$AAP?$AAY@ 00000001800053a0     libucrt:lcidtoname_downlevel.obj
 0001:000043b0       ??_C@_1M@EDGINPNP@?$AAa?$AAr?$AA?9?$AAQ?$AAA@ 00000001800053b0     libucrt:lcidtoname_downlevel.obj
 0001:000043c0       ??_C@_1M@MKDBIIJI@?$AAe?$AAs?$AA?9?$AAB?$AAO@ 00000001800053c0     libucrt:lcidtoname_downlevel.obj
 0001:000043d0       ??_C@_1M@CPKKEBLD@?$AAe?$AAs?$AA?9?$AAS?$AAV@ 00000001800053d0     libucrt:lcidtoname_downlevel.obj
 0001:000043e0       ??_C@_1M@NDBGMMJL@?$AAe?$AAs?$AA?9?$AAH?$AAN@ 00000001800053e0     libucrt:lcidtoname_downlevel.obj
 0001:000043f0       ??_C@_1M@JIJIBHDP@?$AAe?$AAs?$AA?9?$AAN?$AAI@ 00000001800053f0     libucrt:lcidtoname_downlevel.obj
 0001:00004400       ??_C@_1M@CGFMKEEK@?$AAe?$AAs?$AA?9?$AAP?$AAR@ 0000000180005400     libucrt:lcidtoname_downlevel.obj
 0001:00004410       ??_C@_1O@ICJHKIIK@?$AAz?$AAh?$AA?9?$AAC?$AAH?$AAT@ 0000000180005410     libucrt:lcidtoname_downlevel.obj
 0001:00004420       ??_C@_15CLNEJCE@?$AAs?$AAr@ 0000000180005420     libucrt:lcidtoname_downlevel.obj
 0001:00005270       ??_C@_1M@KAHEKEIG@?$AAa?$AAf?$AA?9?$AAz?$AAa@ 0000000180006270     libucrt:lcidtoname_downlevel.obj
 0001:00005280       ??_C@_1M@GIECOABL@?$AAa?$AAr?$AA?9?$AAa?$AAe@ 0000000180006280     libucrt:lcidtoname_downlevel.obj
 0001:00005290       ??_C@_1M@BMLMEKGI@?$AAa?$AAr?$AA?9?$AAb?$AAh@ 0000000180006290     libucrt:lcidtoname_downlevel.obj
 0001:000052a0       ??_C@_1M@DAPFDGGB@?$AAa?$AAr?$AA?9?$AAd?$AAz@ 00000001800062a0     libucrt:lcidtoname_downlevel.obj
 0001:000052b0       ??_C@_1M@FJNKGKIG@?$AAa?$AAr?$AA?9?$AAe?$AAg@ 00000001800062b0     libucrt:lcidtoname_downlevel.obj
 0001:000052c0       ??_C@_1M@FLGKKCLO@?$AAa?$AAr?$AA?9?$AAi?$AAq@ 00000001800062c0     libucrt:lcidtoname_downlevel.obj
 0001:000052d0       ??_C@_1M@GNDIPALM@?$AAa?$AAr?$AA?9?$AAj?$AAo@ 00000001800062d0     libucrt:lcidtoname_downlevel.obj
 0001:000052e0       ??_C@_1M@DDMJFMGJ@?$AAa?$AAr?$AA?9?$AAk?$AAw@ 00000001800062e0     libucrt:lcidtoname_downlevel.obj
 0001:000052f0       ??_C@_1M@EJALMLHM@?$AAa?$AAr?$AA?9?$AAl?$AAb@ 00000001800062f0     libucrt:lcidtoname_downlevel.obj
 0001:00005300       ??_C@_1M@MOBDBLOC@?$AAa?$AAr?$AA?9?$AAl?$AAy@ 0000000180006300     libucrt:lcidtoname_downlevel.obj
 0001:00005310       ??_C@_1M@JAOCLHDH@?$AAa?$AAr?$AA?9?$AAm?$AAa@ 0000000180006310     libucrt:lcidtoname_downlevel.obj
 0001:00005320       ??_C@_1M@JHPMKJIE@?$AAa?$AAr?$AA?9?$AAo?$AAm@ 0000000180006320     libucrt:lcidtoname_downlevel.obj
 0001:00005330       ??_C@_1M@OEPGHFNH@?$AAa?$AAr?$AA?9?$AAq?$AAa@ 0000000180006330     libucrt:lcidtoname_downlevel.obj
 0001:00005340       ??_C@_1M@KJDONENM@?$AAa?$AAr?$AA?9?$AAs?$AAa@ 0000000180006340     libucrt:lcidtoname_downlevel.obj
 0001:00005350       ??_C@_1M@DMJDKLKM@?$AAa?$AAr?$AA?9?$AAs?$AAy@ 0000000180006350     libucrt:lcidtoname_downlevel.obj
 0001:00005360       ??_C@_1M@OMFIPEDC@?$AAa?$AAr?$AA?9?$AAt?$AAn@ 0000000180006360     libucrt:lcidtoname_downlevel.obj
 0001:00005370       ??_C@_1M@IHMHGAON@?$AAa?$AAr?$AA?9?$AAy?$AAe@ 0000000180006370     libucrt:lcidtoname_downlevel.obj
 0001:00005380       ??_C@_1BG@KDCPGJGB@?$AAa?$AAz?$AA?9?$AAa?$AAz?$AA?9?$AAc?$AAy?$AAr?$AAl@ 0000000180006380     libucrt:lcidtoname_downlevel.obj
 0001:00005398       ??_C@_1BG@IBCKDDOE@?$AAa?$AAz?$AA?9?$AAa?$AAz?$AA?9?$AAl?$AAa?$AAt?$AAn@ 0000000180006398     libucrt:lcidtoname_downlevel.obj
 0001:000053b0       ??_C@_1M@EGPFDCPD@?$AAb?$AAe?$AA?9?$AAb?$AAy@ 00000001800063b0     libucrt:lcidtoname_downlevel.obj
 0001:000053c0       ??_C@_1M@PCMGMCGC@?$AAb?$AAg?$AA?9?$AAb?$AAg@ 00000001800063c0     libucrt:lcidtoname_downlevel.obj
 0001:000053d0       ??_C@_1M@BJBMFGOB@?$AAb?$AAn?$AA?9?$AAi?$AAn@ 00000001800063d0     libucrt:lcidtoname_downlevel.obj
 0001:000053e0       ??_C@_1BG@EAKMMACD@?$AAb?$AAs?$AA?9?$AAb?$AAa?$AA?9?$AAl?$AAa?$AAt?$AAn@ 00000001800063e0     libucrt:lcidtoname_downlevel.obj
 0001:000053f8       ??_C@_1M@KGADAODK@?$AAc?$AAa?$AA?9?$AAe?$AAs@ 00000001800063f8     libucrt:lcidtoname_downlevel.obj
 0001:00005408       ??_C@_1M@COAJPDHI@?$AAc?$AAs?$AA?9?$AAc?$AAz@ 0000000180006408     libucrt:lcidtoname_downlevel.obj
 0001:00005418       ??_C@_1M@DHBHFONH@?$AAc?$AAy?$AA?9?$AAg?$AAb@ 0000000180006418     libucrt:lcidtoname_downlevel.obj
 0001:00005428       ??_C@_1M@IMGKELGA@?$AAd?$AAa?$AA?9?$AAd?$AAk@ 0000000180006428     libucrt:lcidtoname_downlevel.obj
 0001:00005438       ??_C@_1M@NNDGDNGA@?$AAd?$AAe?$AA?9?$AAa?$AAt@ 0000000180006438     libucrt:lcidtoname_downlevel.obj
 0001:00005448       ??_C@_1M@IKDBHEEM@?$AAd?$AAe?$AA?9?$AAc?$AAh@ 0000000180006448     libucrt:lcidtoname_downlevel.obj
 0001:00005458       ??_C@_1M@GFFOJMCJ@?$AAd?$AAe?$AA?9?$AAd?$AAe@ 0000000180006458     libucrt:lcidtoname_downlevel.obj
 0001:00005468       ??_C@_1M@MDNLKBPM@?$AAd?$AAe?$AA?9?$AAl?$AAi@ 0000000180006468     libucrt:lcidtoname_downlevel.obj
 0001:00005478       ??_C@_1M@NJBEEJNL@?$AAd?$AAe?$AA?9?$AAl?$AAu@ 0000000180006478     libucrt:lcidtoname_downlevel.obj
 0001:00005488       ??_C@_1O@GNNELBAP@?$AAd?$AAi?$AAv?$AA?9?$AAm?$AAv@ 0000000180006488     libucrt:lcidtoname_downlevel.obj
 0001:00005498       ??_C@_1M@EJLEOGAE@?$AAe?$AAl?$AA?9?$AAg?$AAr@ 0000000180006498     libucrt:lcidtoname_downlevel.obj
 0001:000054a8       ??_C@_1M@GMPONJN@?$AAe?$AAn?$AA?9?$AAa?$AAu@ 00000001800064a8     libucrt:lcidtoname_downlevel.obj
 0001:000054b8       ??_C@_1M@NIDIIPGF@?$AAe?$AAn?$AA?9?$AAb?$AAz@ 00000001800064b8     libucrt:lcidtoname_downlevel.obj
 0001:000054c8       ??_C@_1M@JEHMIMFO@?$AAe?$AAn?$AA?9?$AAc?$AAa@ 00000001800064c8     libucrt:lcidtoname_downlevel.obj
 0001:000054d8       ??_C@_1M@IGMJCDLA@?$AAe?$AAn?$AA?9?$AAc?$AAb@ 00000001800064d8     libucrt:lcidtoname_downlevel.obj
 0001:000054e8       ??_C@_1M@BNFIGBKG@?$AAe?$AAn?$AA?9?$AAg?$AAb@ 00000001800064e8     libucrt:lcidtoname_downlevel.obj
 0001:000054f8       ??_C@_1M@LKIFDIGP@?$AAe?$AAn?$AA?9?$AAi?$AAe@ 00000001800064f8     libucrt:lcidtoname_downlevel.obj
 0001:00005508       ??_C@_1M@PJKFGCCO@?$AAe?$AAn?$AA?9?$AAj?$AAm@ 0000000180006508     libucrt:lcidtoname_downlevel.obj
 0001:00005518       ??_C@_1M@KPPKEPBO@?$AAe?$AAn?$AA?9?$AAn?$AAz@ 0000000180006518     libucrt:lcidtoname_downlevel.obj
 0001:00005528       ??_C@_1M@GMDGLDOB@?$AAe?$AAn?$AA?9?$AAp?$AAh@ 0000000180006528     libucrt:lcidtoname_downlevel.obj
 0001:00005538       ??_C@_1M@ONGIBJNA@?$AAe?$AAn?$AA?9?$AAt?$AAt@ 0000000180006538     libucrt:lcidtoname_downlevel.obj
 0001:00005548       ??_C@_1M@LLODPCMM@?$AAe?$AAn?$AA?9?$AAu?$AAs@ 0000000180006548     libucrt:lcidtoname_downlevel.obj
 0001:00005558       ??_C@_1M@LAKFNPAN@?$AAe?$AAn?$AA?9?$AAz?$AAa@ 0000000180006558     libucrt:lcidtoname_downlevel.obj
 0001:00005568       ??_C@_1M@MFNHNHEO@?$AAe?$AAn?$AA?9?$AAz?$AAw@ 0000000180006568     libucrt:lcidtoname_downlevel.obj
 0001:00005578       ??_C@_1M@EJEINPHM@?$AAe?$AAs?$AA?9?$AAa?$AAr@ 0000000180006578     libucrt:lcidtoname_downlevel.obj
 0001:00005588       ??_C@_1M@GNKPCCJA@?$AAe?$AAs?$AA?9?$AAb?$AAo@ 0000000180006588     libucrt:lcidtoname_downlevel.obj
 0001:00005598       ??_C@_1M@LEEGFONL@?$AAe?$AAs?$AA?9?$AAc?$AAl@ 0000000180006598     libucrt:lcidtoname_downlevel.obj
 0001:000055a8       ??_C@_1M@KGPDPBDF@?$AAe?$AAs?$AA?9?$AAc?$AAo@ 00000001800065a8     libucrt:lcidtoname_downlevel.obj
 0001:000055b8       ??_C@_1M@EIAHOHH@?$AAe?$AAs?$AA?9?$AAc?$AAr@ 00000001800065b8     libucrt:lcidtoname_downlevel.obj
 0001:000055c8       ??_C@_1M@LLPGMBIN@?$AAe?$AAs?$AA?9?$AAd?$AAo@ 00000001800065c8     libucrt:lcidtoname_downlevel.obj
 0001:000055d8       ??_C@_1M@DKHMKNJA@?$AAe?$AAs?$AA?9?$AAe?$AAc@ 00000001800065d8     libucrt:lcidtoname_downlevel.obj
 0001:000055e8       ??_C@_1M@GKGFPKAP@?$AAe?$AAs?$AA?9?$AAe?$AAs@ 00000001800065e8     libucrt:lcidtoname_downlevel.obj
 0001:000055f8       ??_C@_1M@LKHKGDLN@?$AAe?$AAs?$AA?9?$AAg?$AAt@ 00000001800065f8     libucrt:lcidtoname_downlevel.obj
 0001:00005608       ??_C@_1M@HEIIGGJD@?$AAe?$AAs?$AA?9?$AAh?$AAn@ 0000000180006608     libucrt:lcidtoname_downlevel.obj
 0001:00005618       ??_C@_1M@FBDHPPGD@?$AAe?$AAs?$AA?9?$AAm?$AAx@ 0000000180006618     libucrt:lcidtoname_downlevel.obj
 0001:00005628       ??_C@_1M@DPAGLNDH@?$AAe?$AAs?$AA?9?$AAn?$AAi@ 0000000180006628     libucrt:lcidtoname_downlevel.obj
 0001:00005638       ??_C@_1M@MDGOPGDD@?$AAe?$AAs?$AA?9?$AAp?$AAa@ 0000000180006638     libucrt:lcidtoname_downlevel.obj
 0001:00005648       ??_C@_1M@EMAMGBGE@?$AAe?$AAs?$AA?9?$AAp?$AAe@ 0000000180006648     libucrt:lcidtoname_downlevel.obj
 0001:00005658       ??_C@_1M@IBMCAOEC@?$AAe?$AAs?$AA?9?$AAp?$AAr@ 0000000180006658     libucrt:lcidtoname_downlevel.obj
 0001:00005668       ??_C@_1M@FGMDIJED@?$AAe?$AAs?$AA?9?$AAp?$AAy@ 0000000180006668     libucrt:lcidtoname_downlevel.obj
 0001:00005678       ??_C@_1M@IIDEOLLL@?$AAe?$AAs?$AA?9?$AAs?$AAv@ 0000000180006678     libucrt:lcidtoname_downlevel.obj
 0001:00005688       ??_C@_1M@GAOBIPA@?$AAe?$AAs?$AA?9?$AAu?$AAy@ 0000000180006688     libucrt:lcidtoname_downlevel.obj
 0001:00005698       ??_C@_1M@JKFFICHJ@?$AAe?$AAs?$AA?9?$AAv?$AAe@ 0000000180006698     libucrt:lcidtoname_downlevel.obj
 0001:000056a8       ??_C@_1M@PNMLOJDF@?$AAe?$AAt?$AA?9?$AAe?$AAe@ 00000001800066a8     libucrt:lcidtoname_downlevel.obj
 0001:000056b8       ??_C@_1M@GHHLIKEI@?$AAe?$AAu?$AA?9?$AAe?$AAs@ 00000001800066b8     libucrt:lcidtoname_downlevel.obj
 0001:000056c8       ??_C@_1M@PBNONODE@?$AAf?$AAa?$AA?9?$AAi?$AAr@ 00000001800066c8     libucrt:lcidtoname_downlevel.obj
 0001:000056d8       ??_C@_1M@JEEHPMIL@?$AAf?$AAi?$AA?9?$AAf?$AAi@ 00000001800066d8     libucrt:lcidtoname_downlevel.obj
 0001:000056e8       ??_C@_1M@LMDCNDBA@?$AAf?$AAo?$AA?9?$AAf?$AAo@ 00000001800066e8     libucrt:lcidtoname_downlevel.obj
 0001:000056f8       ??_C@_1M@JKEOHLDK@?$AAf?$AAr?$AA?9?$AAb?$AAe@ 00000001800066f8     libucrt:lcidtoname_downlevel.obj
 0001:00005708       ??_C@_1M@NOHADPMI@?$AAf?$AAr?$AA?9?$AAc?$AAa@ 0000000180006708     libucrt:lcidtoname_downlevel.obj
 0001:00005718       ??_C@_1M@KDHIHAEC@?$AAf?$AAr?$AA?9?$AAc?$AAh@ 0000000180006718     libucrt:lcidtoname_downlevel.obj
 0001:00005728       ??_C@_1M@MMBBFGAK@?$AAf?$AAr?$AA?9?$AAf?$AAr@ 0000000180006728     libucrt:lcidtoname_downlevel.obj
 0001:00005738       ??_C@_1M@PAFNENNF@?$AAf?$AAr?$AA?9?$AAl?$AAu@ 0000000180006738     libucrt:lcidtoname_downlevel.obj
 0001:00005748       ??_C@_1M@EOHDJGDD@?$AAf?$AAr?$AA?9?$AAm?$AAc@ 0000000180006748     libucrt:lcidtoname_downlevel.obj
 0001:00005758       ??_C@_1M@FAPLLOPF@?$AAg?$AAl?$AA?9?$AAe?$AAs@ 0000000180006758     libucrt:lcidtoname_downlevel.obj
 0001:00005768       ??_C@_1M@FOPBFLOO@?$AAg?$AAu?$AA?9?$AAi?$AAn@ 0000000180006768     libucrt:lcidtoname_downlevel.obj
 0001:00005778       ??_C@_1M@KBMCINPM@?$AAh?$AAe?$AA?9?$AAi?$AAl@ 0000000180006778     libucrt:lcidtoname_downlevel.obj
 0001:00005788       ??_C@_1M@BBPHKFPJ@?$AAh?$AAi?$AA?9?$AAi?$AAn@ 0000000180006788     libucrt:lcidtoname_downlevel.obj
 0001:00005798       ??_C@_1M@PMBNDPHD@?$AAh?$AAr?$AA?9?$AAb?$AAa@ 0000000180006798     libucrt:lcidtoname_downlevel.obj
 0001:000057a8       ??_C@_1M@BPCKOEGE@?$AAh?$AAr?$AA?9?$AAh?$AAr@ 00000001800067a8     libucrt:lcidtoname_downlevel.obj
 0001:000057b8       ??_C@_1M@GACBMHKE@?$AAh?$AAu?$AA?9?$AAh?$AAu@ 00000001800067b8     libucrt:lcidtoname_downlevel.obj
 0001:000057c8       ??_C@_1M@MILPAJJC@?$AAh?$AAy?$AA?9?$AAa?$AAm@ 00000001800067c8     libucrt:lcidtoname_downlevel.obj
 0001:000057d8       ??_C@_1M@BABBICEC@?$AAi?$AAd?$AA?9?$AAi?$AAd@ 00000001800067d8     libucrt:lcidtoname_downlevel.obj
 0001:000057e8       ??_C@_1M@BIKNHHPF@?$AAi?$AAs?$AA?9?$AAi?$AAs@ 00000001800067e8     libucrt:lcidtoname_downlevel.obj
 0001:000057f8       ??_C@_1M@NMPCJPHE@?$AAi?$AAt?$AA?9?$AAc?$AAh@ 00000001800067f8     libucrt:lcidtoname_downlevel.obj
 0001:00005808       ??_C@_1M@GHKGFEDF@?$AAi?$AAt?$AA?9?$AAi?$AAt@ 0000000180006808     libucrt:lcidtoname_downlevel.obj
 0001:00005818       ??_C@_1M@NIEJCJJA@?$AAj?$AAa?$AA?9?$AAj?$AAp@ 0000000180006818     libucrt:lcidtoname_downlevel.obj
 0001:00005828       ??_C@_1M@JILFNBIM@?$AAk?$AAa?$AA?9?$AAg?$AAe@ 0000000180006828     libucrt:lcidtoname_downlevel.obj
 0001:00005838       ??_C@_1M@PACPMGPH@?$AAk?$AAk?$AA?9?$AAk?$AAz@ 0000000180006838     libucrt:lcidtoname_downlevel.obj
 0001:00005848       ??_C@_1M@IELFGMHA@?$AAk?$AAn?$AA?9?$AAi?$AAn@ 0000000180006848     libucrt:lcidtoname_downlevel.obj
 0001:00005858       ??_C@_1O@IBBJHCH@?$AAk?$AAo?$AAk?$AA?9?$AAi?$AAn@ 0000000180006858     libucrt:lcidtoname_downlevel.obj
 0001:00005868       ??_C@_1M@DMHAEOGC@?$AAk?$AAo?$AA?9?$AAk?$AAr@ 0000000180006868     libucrt:lcidtoname_downlevel.obj
 0001:00005878       ??_C@_1M@HBAHBIGA@?$AAk?$AAy?$AA?9?$AAk?$AAg@ 0000000180006878     libucrt:lcidtoname_downlevel.obj
 0001:00005888       ??_C@_1M@KPMILCJG@?$AAl?$AAt?$AA?9?$AAl?$AAt@ 0000000180006888     libucrt:lcidtoname_downlevel.obj
 0001:00005898       ??_C@_1M@BDEKKCA@?$AAl?$AAv?$AA?9?$AAl?$AAv@ 0000000180006898     libucrt:lcidtoname_downlevel.obj
 0001:000058a8       ??_C@_1M@ELCKCCJJ@?$AAm?$AAi?$AA?9?$AAn?$AAz@ 00000001800068a8     libucrt:lcidtoname_downlevel.obj
 0001:000058b8       ??_C@_1M@CBOOLAPA@?$AAm?$AAk?$AA?9?$AAm?$AAk@ 00000001800068b8     libucrt:lcidtoname_downlevel.obj
 0001:000058c8       ??_C@_1M@GPHNBJKN@?$AAm?$AAl?$AA?9?$AAi?$AAn@ 00000001800068c8     libucrt:lcidtoname_downlevel.obj
 0001:000058d8       ??_C@_1M@PABJILIG@?$AAm?$AAn?$AA?9?$AAm?$AAn@ 00000001800068d8     libucrt:lcidtoname_downlevel.obj
 0001:000058e8       ??_C@_1M@FGBKKIPG@?$AAm?$AAr?$AA?9?$AAi?$AAn@ 00000001800068e8     libucrt:lcidtoname_downlevel.obj
 0001:000058f8       ??_C@_1M@NDBPDDAL@?$AAm?$AAs?$AA?9?$AAb?$AAn@ 00000001800068f8     libucrt:lcidtoname_downlevel.obj
 0001:00005908       ??_C@_1M@OPIHOOPI@?$AAm?$AAs?$AA?9?$AAm?$AAy@ 0000000180006908     libucrt:lcidtoname_downlevel.obj
 0001:00005918       ??_C@_1M@PPDBCNFM@?$AAm?$AAt?$AA?9?$AAm?$AAt@ 0000000180006918     libucrt:lcidtoname_downlevel.obj
 0001:00005928       ??_C@_1M@KDJDKMDD@?$AAn?$AAb?$AA?9?$AAn?$AAo@ 0000000180006928     libucrt:lcidtoname_downlevel.obj
 0001:00005938       ??_C@_1M@KFCFLMJP@?$AAn?$AAl?$AA?9?$AAb?$AAe@ 0000000180006938     libucrt:lcidtoname_downlevel.obj
 0001:00005948       ??_C@_1M@KPOPDDGO@?$AAn?$AAl?$AA?9?$AAn?$AAl@ 0000000180006948     libucrt:lcidtoname_downlevel.obj
 0001:00005958       ??_C@_1M@LJKPEMLN@?$AAn?$AAn?$AA?9?$AAn?$AAo@ 0000000180006958     libucrt:lcidtoname_downlevel.obj
 0001:00005968       ??_C@_1M@BDGHHBFL@?$AAn?$AAs?$AA?9?$AAz?$AAa@ 0000000180006968     libucrt:lcidtoname_downlevel.obj
 0001:00005978       ??_C@_1M@IDEHOAP@?$AAp?$AAa?$AA?9?$AAi?$AAn@ 0000000180006978     libucrt:lcidtoname_downlevel.obj
 0001:00005988       ??_C@_1M@HDBKGOGH@?$AAp?$AAl?$AA?9?$AAp?$AAl@ 0000000180006988     libucrt:lcidtoname_downlevel.obj
 0001:00005998       ??_C@_1M@LJLLCMEH@?$AAp?$AAt?$AA?9?$AAb?$AAr@ 0000000180006998     libucrt:lcidtoname_downlevel.obj
 0001:000059a8       ??_C@_1M@NCMONAAL@?$AAp?$AAt?$AA?9?$AAp?$AAt@ 00000001800069a8     libucrt:lcidtoname_downlevel.obj
 0001:000059b8       ??_C@_1O@EAKMAJDN@?$AAq?$AAu?$AAz?$AA?9?$AAb?$AAo@ 00000001800069b8     libucrt:lcidtoname_downlevel.obj
 0001:000059c8       ??_C@_1O@BHHPIGDN@?$AAq?$AAu?$AAz?$AA?9?$AAe?$AAc@ 00000001800069c8     libucrt:lcidtoname_downlevel.obj
 0001:000059d8       ??_C@_1O@GBAPEKMJ@?$AAq?$AAu?$AAz?$AA?9?$AAp?$AAe@ 00000001800069d8     libucrt:lcidtoname_downlevel.obj
 0001:000059e8       ??_C@_1M@CLGLEFBO@?$AAr?$AAo?$AA?9?$AAr?$AAo@ 00000001800069e8     libucrt:lcidtoname_downlevel.obj
 0001:000059f8       ??_C@_1M@CEEDODME@?$AAr?$AAu?$AA?9?$AAr?$AAu@ 00000001800069f8     libucrt:lcidtoname_downlevel.obj
 0001:00005a08       ??_C@_1M@HPKKKMPP@?$AAs?$AAa?$AA?9?$AAi?$AAn@ 0000000180006a08     libucrt:lcidtoname_downlevel.obj
 0001:00005a18       ??_C@_1M@BKMAIGOJ@?$AAs?$AAe?$AA?9?$AAf?$AAi@ 0000000180006a18     libucrt:lcidtoname_downlevel.obj
 0001:00005a28       ??_C@_1M@NDPIFLFI@?$AAs?$AAe?$AA?9?$AAn?$AAo@ 0000000180006a28     libucrt:lcidtoname_downlevel.obj
 0001:00005a38       ??_C@_1M@DANKKHJ@?$AAs?$AAe?$AA?9?$AAs?$AAe@ 0000000180006a38     libucrt:lcidtoname_downlevel.obj
 0001:00005a48       ??_C@_1M@PNBLONPJ@?$AAs?$AAk?$AA?9?$AAs?$AAk@ 0000000180006a48     libucrt:lcidtoname_downlevel.obj
 0001:00005a58       ??_C@_1M@LFMODOAL@?$AAs?$AAl?$AA?9?$AAs?$AAi@ 0000000180006a58     libucrt:lcidtoname_downlevel.obj
 0001:00005a68       ??_C@_1O@DFKOMPG@?$AAs?$AAm?$AAa?$AA?9?$AAn?$AAo@ 0000000180006a68     libucrt:lcidtoname_downlevel.obj
 0001:00005a78       ??_C@_1O@NDKPBNNH@?$AAs?$AAm?$AAa?$AA?9?$AAs?$AAe@ 0000000180006a78     libucrt:lcidtoname_downlevel.obj
 0001:00005a88       ??_C@_1O@PLLKBHAB@?$AAs?$AAm?$AAj?$AA?9?$AAn?$AAo@ 0000000180006a88     libucrt:lcidtoname_downlevel.obj
 0001:00005a98       ??_C@_1O@CLEPOGCA@?$AAs?$AAm?$AAj?$AA?9?$AAs?$AAe@ 0000000180006a98     libucrt:lcidtoname_downlevel.obj
 0001:00005aa8       ??_C@_1O@DLGJGKMK@?$AAs?$AAm?$AAn?$AA?9?$AAf?$AAi@ 0000000180006aa8     libucrt:lcidtoname_downlevel.obj
 0001:00005ab8       ??_C@_1O@OJDJGAJC@?$AAs?$AAm?$AAs?$AA?9?$AAf?$AAi@ 0000000180006ab8     libucrt:lcidtoname_downlevel.obj
 0001:00005ac8       ??_C@_1M@BOFOGHPB@?$AAs?$AAq?$AA?9?$AAa?$AAl@ 0000000180006ac8     libucrt:lcidtoname_downlevel.obj
 0001:00005ad8       ??_C@_1BG@LJBBIPGB@?$AAs?$AAr?$AA?9?$AAb?$AAa?$AA?9?$AAc?$AAy?$AAr?$AAl@ 0000000180006ad8     libucrt:lcidtoname_downlevel.obj
 0001:00005af0       ??_C@_1BG@JLBENFOE@?$AAs?$AAr?$AA?9?$AAb?$AAa?$AA?9?$AAl?$AAa?$AAt?$AAn@ 0000000180006af0     libucrt:lcidtoname_downlevel.obj
 0001:00005b08       ??_C@_1BG@KODPNHE@?$AAs?$AAr?$AA?9?$AAs?$AAp?$AA?9?$AAc?$AAy?$AAr?$AAl@ 0000000180006b08     libucrt:lcidtoname_downlevel.obj
 0001:00005b20       ??_C@_1BG@CIOGKHPB@?$AAs?$AAr?$AA?9?$AAs?$AAp?$AA?9?$AAl?$AAa?$AAt?$AAn@ 0000000180006b20     libucrt:lcidtoname_downlevel.obj
 0001:00005b38       ??_C@_1M@NGFJLMAC@?$AAs?$AAv?$AA?9?$AAf?$AAi@ 0000000180006b38     libucrt:lcidtoname_downlevel.obj
 0001:00005b48       ??_C@_1M@MPJEJAJC@?$AAs?$AAv?$AA?9?$AAs?$AAe@ 0000000180006b48     libucrt:lcidtoname_downlevel.obj
 0001:00005b58       ??_C@_1M@MPNDHLFK@?$AAs?$AAw?$AA?9?$AAk?$AAe@ 0000000180006b58     libucrt:lcidtoname_downlevel.obj
 0001:00005b68       ??_C@_1O@KOHBJJI@?$AAs?$AAy?$AAr?$AA?9?$AAs?$AAy@ 0000000180006b68     libucrt:lcidtoname_downlevel.obj
 0001:00005b78       ??_C@_1M@LDCEFHA@?$AAt?$AAa?$AA?9?$AAi?$AAn@ 0000000180006b78     libucrt:lcidtoname_downlevel.obj
 0001:00005b88       ??_C@_1M@CNJOFAK@?$AAt?$AAe?$AA?9?$AAi?$AAn@ 0000000180006b88     libucrt:lcidtoname_downlevel.obj
 0001:00005b98       ??_C@_1M@GNAECACD@?$AAt?$AAh?$AA?9?$AAt?$AAh@ 0000000180006b98     libucrt:lcidtoname_downlevel.obj
 0001:00005ba8       ??_C@_1M@CHBIHOJO@?$AAt?$AAn?$AA?9?$AAz?$AAa@ 0000000180006ba8     libucrt:lcidtoname_downlevel.obj
 0001:00005bb8       ??_C@_1M@GCCMIGPJ@?$AAt?$AAr?$AA?9?$AAt?$AAr@ 0000000180006bb8     libucrt:lcidtoname_downlevel.obj
 0001:00005bc8       ??_C@_1M@CELMCNBK@?$AAt?$AAt?$AA?9?$AAr?$AAu@ 0000000180006bc8     libucrt:lcidtoname_downlevel.obj
 0001:00005bd8       ??_C@_1M@KLMCELGA@?$AAu?$AAk?$AA?9?$AAu?$AAa@ 0000000180006bd8     libucrt:lcidtoname_downlevel.obj
 0001:00005be8       ??_C@_1M@EPAJJAJF@?$AAu?$AAr?$AA?9?$AAp?$AAk@ 0000000180006be8     libucrt:lcidtoname_downlevel.obj
 0001:00005bf8       ??_C@_1BG@GEGPMCDJ@?$AAu?$AAz?$AA?9?$AAu?$AAz?$AA?9?$AAc?$AAy?$AAr?$AAl@ 0000000180006bf8     libucrt:lcidtoname_downlevel.obj
 0001:00005c10       ??_C@_1BG@EGGKJILM@?$AAu?$AAz?$AA?9?$AAu?$AAz?$AA?9?$AAl?$AAa?$AAt?$AAn@ 0000000180006c10     libucrt:lcidtoname_downlevel.obj
 0001:00005c28       ??_C@_1M@GFOCLFF@?$AAv?$AAi?$AA?9?$AAv?$AAn@ 0000000180006c28     libucrt:lcidtoname_downlevel.obj
 0001:00005c38       ??_C@_1M@CPAMEDFI@?$AAx?$AAh?$AA?9?$AAz?$AAa@ 0000000180006c38     libucrt:lcidtoname_downlevel.obj
 0001:00005c48       ??_C@_1O@EBKIFIGN@?$AAz?$AAh?$AA?9?$AAc?$AAh?$AAs@ 0000000180006c48     libucrt:lcidtoname_downlevel.obj
 0001:00005c58       ??_C@_1O@NMHPGANE@?$AAz?$AAh?$AA?9?$AAc?$AAh?$AAt@ 0000000180006c58     libucrt:lcidtoname_downlevel.obj
 0001:00005c68       ??_C@_1M@LPINJOMC@?$AAz?$AAh?$AA?9?$AAc?$AAn@ 0000000180006c68     libucrt:lcidtoname_downlevel.obj
 0001:00005c78       ??_C@_1M@OCJEJODD@?$AAz?$AAh?$AA?9?$AAh?$AAk@ 0000000180006c78     libucrt:lcidtoname_downlevel.obj
 0001:00005c88       ??_C@_1M@DNDLJINH@?$AAz?$AAh?$AA?9?$AAm?$AAo@ 0000000180006c88     libucrt:lcidtoname_downlevel.obj
 0001:00005c98       ??_C@_1M@MBFDNDND@?$AAz?$AAh?$AA?9?$AAs?$AAg@ 0000000180006c98     libucrt:lcidtoname_downlevel.obj
 0001:00005ca8       ??_C@_1M@IMEPLEPE@?$AAz?$AAh?$AA?9?$AAt?$AAw@ 0000000180006ca8     libucrt:lcidtoname_downlevel.obj
 0001:00005cb8       ??_C@_1M@BBGHNHJP@?$AAz?$AAu?$AA?9?$AAz?$AAa@ 0000000180006cb8     libucrt:lcidtoname_downlevel.obj
 0001:00005f20       ??_C@_1BA@BALFACEM@?$AAC?$AAO?$AAN?$AAO?$AAU?$AAT?$AA$@ 0000000180006f20     libucrt:initcon.obj
 0001:00005f30       __log10_256_lead           0000000180006f30     libucrt:log10_256_lead_tail_table.obj
 0001:00006740       __log10_256_tail           0000000180007740     libucrt:log10_256_lead_tail_table.obj
 0001:00006f50       __log_F_inv_qword          0000000180007f50     libucrt:log_f_inv_qword_table.obj
 0001:00007760       ??_C@_05HGHHAHAP@log10@    0000000180008760     libucrt:log_special.obj
 0001:000077b0       _load_config_used          00000001800087b0     LIBCMT:loadcfg.obj
 0001:000078b8       ??_R4exception@std@@6B@    00000001800088b8     LIBCMT:throw_bad_alloc.obj
 0001:000078e0       ??_R3exception@std@@8      00000001800088e0     LIBCMT:throw_bad_alloc.obj
 0001:000078f8       ??_R2exception@std@@8      00000001800088f8     LIBCMT:throw_bad_alloc.obj
 0001:00007908       ??_R1A@?0A@EA@exception@std@@8 0000000180008908     LIBCMT:throw_bad_alloc.obj
 0001:00007930       ??_R4bad_alloc@std@@6B@    0000000180008930     LIBCMT:throw_bad_alloc.obj
 0001:00007958       ??_R3bad_alloc@std@@8      0000000180008958     LIBCMT:throw_bad_alloc.obj
 0001:00007970       ??_R2bad_alloc@std@@8      0000000180008970     LIBCMT:throw_bad_alloc.obj
 0001:00007988       ??_R1A@?0A@EA@bad_alloc@std@@8 0000000180008988     LIBCMT:throw_bad_alloc.obj
 0001:000079b0       ??_R4bad_array_new_length@std@@6B@ 00000001800089b0     LIBCMT:throw_bad_alloc.obj
 0001:000079d8       ??_R3bad_array_new_length@std@@8 00000001800089d8     LIBCMT:throw_bad_alloc.obj
 0001:000079f0       ??_R2bad_array_new_length@std@@8 00000001800089f0     LIBCMT:throw_bad_alloc.obj
 0001:00007a10       ??_R1A@?0A@EA@bad_array_new_length@std@@8 0000000180008a10     LIBCMT:throw_bad_alloc.obj
 0001:00007a38       ??_R4type_info@@6B@        0000000180008a38     LIBCMT:std_type_info_static.obj
 0001:00007a60       ??_R3type_info@@8          0000000180008a60     LIBCMT:std_type_info_static.obj
 0001:00007a78       ??_R2type_info@@8          0000000180008a78     LIBCMT:std_type_info_static.obj
 0001:00007a88       ??_R1A@?0A@EA@type_info@@8 0000000180008a88     LIBCMT:std_type_info_static.obj
 0001:00007d70       __rtc_iaa                  0000000180008d70     LIBCMT:initsect.obj
 0001:00007d78       __rtc_izz                  0000000180008d78     LIBCMT:initsect.obj
 0001:00007d80       __rtc_taa                  0000000180008d80     LIBCMT:initsect.obj
 0001:00007d88       __rtc_tzz                  0000000180008d88     LIBCMT:initsect.obj
 0001:00007da0       _alloca_probe              0000000180008da0 f   chkstk.obj
 0001:00007da0       __chkstk                   0000000180008da0 f   chkstk.obj
 0001:00007e00       ??1?$DialogBuilderBase@UFarDialogItem@@@@MEAA@XZ 0000000180008e00 f i Brackets.obj
 0001:00007e80       ??_E?$DialogBuilderBase@UFarDialogItem@@@@MEAAPEAXI@Z 0000000180008e80 f i Brackets.obj
 0001:00007e80       ??_G?$DialogBuilderBase@UFarDialogItem@@@@MEAAPEAXI@Z 0000000180008e80 f i Brackets.obj
 0001:00007ec0       ??_G?$DialogItemBinding@UFarDialogItem@@@@UEAAPEAXI@Z 0000000180008ec0 f i Brackets.obj
 0001:00007ec0       ??_E?$DialogItemBinding@UFarDialogItem@@@@UEAAPEAXI@Z 0000000180008ec0 f i Brackets.obj
 0001:00007ef0       ??_GPluginCheckBoxBinding@@UEAAPEAXI@Z 0000000180008ef0 f i Brackets.obj
 0001:00007ef0       ??_EPluginCheckBoxBinding@@UEAAPEAXI@Z 0000000180008ef0 f i Brackets.obj
 0001:00007ef0       ??_GPluginEditFieldBinding@@UEAAPEAXI@Z 0000000180008ef0 f i Brackets.obj
 0001:00007ef0       ??_EPluginEditFieldBinding@@UEAAPEAXI@Z 0000000180008ef0 f i Brackets.obj
 0001:00007f20       ??_EPluginDialogBuilder@@UEAAPEAXI@Z 0000000180008f20 f i Brackets.obj
 0001:00007f20       ??_GPluginDialogBuilder@@UEAAPEAXI@Z 0000000180008f20 f i Brackets.obj
 0001:00007f70       ??_GPluginUIntEditFieldBinding@@UEAAPEAXI@Z 0000000180008f70 f i Brackets.obj
 0001:00007f70       ??_EPluginIntEditFieldBinding@@UEAAPEAXI@Z 0000000180008f70 f i Brackets.obj
 0001:00007f70       ??_EPluginUIntEditFieldBinding@@UEAAPEAXI@Z 0000000180008f70 f i Brackets.obj
 0001:00007f70       ??_GPluginIntEditFieldBinding@@UEAAPEAXI@Z 0000000180008f70 f i Brackets.obj
 0001:00007fa0       ??_EPluginRadioButtonBinding@@UEAAPEAXI@Z 0000000180008fa0 f i Brackets.obj
 0001:00007fa0       ??_GPluginRadioButtonBinding@@UEAAPEAXI@Z 0000000180008fa0 f i Brackets.obj
 0001:00007fd0       ?AddButtons@?$DialogBuilderBase@UFarDialogItem@@@@QEAAXHPEBHHH@Z 0000000180008fd0 f i Brackets.obj
 0001:000082e0       ?AddDialogItem@?$DialogBuilderBase@UFarDialogItem@@@@IEAAPEAUFarDialogItem@@W4FARDIALOGITEMTYPES@@PEB_W@Z 00000001800092e0 f i Brackets.obj
 0001:00008490       ?AddUIntEditField@?$DialogBuilderBase@UFarDialogItem@@@@UEAAPEAUFarDialogItem@@PEAIH@Z 0000000180009490 f i Brackets.obj
 0001:00008490       ?CreateCheckBoxBinding@?$DialogBuilderBase@UFarDialogItem@@@@MEAAPEAU?$DialogItemBinding@UFarDialogItem@@@@PEAHH@Z 0000000180009490 f i Brackets.obj
 0001:00008490       ?AddIntEditField@?$DialogBuilderBase@UFarDialogItem@@@@UEAAPEAUFarDialogItem@@PEAHH@Z 0000000180009490 f i Brackets.obj
 0001:00008490       ?CreateRadioButtonBinding@?$DialogBuilderBase@UFarDialogItem@@@@MEAAPEAU?$DialogItemBinding@UFarDialogItem@@@@PEAH@Z 0000000180009490 f i Brackets.obj
 0001:00008490       ?GetLangString@?$DialogBuilderBase@UFarDialogItem@@@@MEAAPEB_WH@Z 0000000180009490 f i Brackets.obj
 0001:000084a0       ?AddIntEditField@PluginDialogBuilder@@UEAAPEAUFarDialogItem@@PEAHH@Z 00000001800094a0 f i Brackets.obj
 0001:000085f0       ?AddUIntEditField@PluginDialogBuilder@@UEAAPEAUFarDialogItem@@PEAIH@Z 00000001800095f0 f i Brackets.obj
 0001:00008740       ?Config@@YAHXZ             0000000180009740 f   Brackets.obj
 0001:0000ae70       ?CreateCheckBoxBinding@PluginDialogBuilder@@MEAAPEAU?$DialogItemBinding@UFarDialogItem@@@@PEAHH@Z 000000018000be70 f i Brackets.obj
 0001:0000aef0       ?CreateRadioButtonBinding@PluginDialogBuilder@@MEAAPEAU?$DialogItemBinding@UFarDialogItem@@@@PEAH@Z 000000018000bef0 f i Brackets.obj
 0001:0000af60       ?DoShowDialog@?$DialogBuilderBase@UFarDialogItem@@@@MEAA_JXZ 000000018000bf60 f i Brackets.obj
 0001:0000af70       ?DoShowDialog@PluginDialogBuilder@@MEAA_JXZ 000000018000bf70 f i Brackets.obj
 0001:0000b020       ?GetLangString@PluginDialogBuilder@@MEAAPEB_WH@Z 000000018000c020 f i Brackets.obj
 0001:0000b030       _guard_check_icall_nop     000000018000c030 f i LIBCMT:guard_support.obj
 0001:0000b030       ?SaveValue@?$DialogItemBinding@UFarDialogItem@@@@UEAAXPEAUFarDialogItem@@H@Z 000000018000c030 f i Brackets.obj
 0001:0000b030       ?InitDialogItem@?$DialogBuilderBase@UFarDialogItem@@@@MEAAXPEAUFarDialogItem@@PEB_W@Z 000000018000c030 f i Brackets.obj
 0001:0000b040       ?InitDialogItem@PluginDialogBuilder@@MEAAXPEAUFarDialogItem@@PEB_W@Z 000000018000c040 f i Brackets.obj
 0001:0000b070       ?SaveValue@PluginCheckBoxBinding@@UEAAXPEAUFarDialogItem@@H@Z 000000018000c070 f i Brackets.obj
 0001:0000b0c0       ?SaveValue@PluginEditFieldBinding@@UEAAXPEAUFarDialogItem@@H@Z 000000018000c0c0 f i Brackets.obj
 0001:0000b100       ?SaveValue@PluginIntEditFieldBinding@@UEAAXPEAUFarDialogItem@@H@Z 000000018000c100 f i Brackets.obj
 0001:0000b150       ?SaveValue@PluginRadioButtonBinding@@UEAAXPEAUFarDialogItem@@H@Z 000000018000c150 f i Brackets.obj
 0001:0000b1a0       ?SaveValue@PluginUIntEditFieldBinding@@UEAAXPEAUFarDialogItem@@H@Z 000000018000c1a0 f i Brackets.obj
 0001:0000b1f0       ?ShowMenu@@YAHH@Z          000000018000c1f0 f   Brackets.obj
 0001:0000b380       ?TextWidth@?$DialogBuilderBase@UFarDialogItem@@@@MEAAHAEBUFarDialogItem@@@Z 000000018000c380 f i Brackets.obj
 0001:0000b390       ?TextWidth@PluginDialogBuilder@@MEAAHAEBUFarDialogItem@@@Z 000000018000c390 f i Brackets.obj
 0001:0000b3a0       ?UpdateBorderSize@?$DialogBuilderBase@UFarDialogItem@@@@IEAAXXZ 000000018000c3a0 f i Brackets.obj
 0001:0000b580       ConfigureW                 000000018000c580 f   Brackets.obj
 0001:0000b590       GetGlobalInfoW             000000018000c590 f   Brackets.obj
 0001:0000b610       GetPluginInfoW             000000018000c610 f   Brackets.obj
 0001:0000b680       OpenW                      000000018000c680 f   Brackets.obj
 0001:0000c390       SetStartupInfoW            000000018000d390 f   Brackets.obj
 0001:0000c6cc       ??2@YAPEAX_K@Z             000000018000d6cc f   LIBCMT:new_scalar.obj
 0001:0000c708       ??3@YAXPEAX_K@Z            000000018000d708 f   LIBCMT:delete_scalar_size.obj
 0001:0000c708       ??_V@YAXPEAX@Z             000000018000d708 f   LIBCMT:delete_array.obj
 0001:0000c710       ??_U@YAPEAX_K@Z            000000018000d710 f   LIBCMT:new_array.obj
 0001:0000ca38       _DllMainCRTStartup         000000018000da38 f   LIBCMT:dll_dllmain.obj
 0001:0000ca78       ??0bad_alloc@std@@QEAA@AEBV01@@Z 000000018000da78 f i LIBCMT:throw_bad_alloc.obj
 0001:0000cab4       ??0bad_alloc@std@@QEAA@XZ  000000018000dab4 f i LIBCMT:throw_bad_alloc.obj
 0001:0000cad4       ??0bad_array_new_length@std@@QEAA@AEBV01@@Z 000000018000dad4 f i LIBCMT:throw_bad_alloc.obj
 0001:0000cb10       ??0bad_array_new_length@std@@QEAA@XZ 000000018000db10 f i LIBCMT:throw_bad_alloc.obj
 0001:0000cb30       ??0exception@std@@QEAA@AEBV01@@Z 000000018000db30 f i LIBCMT:throw_bad_alloc.obj
 0001:0000cb64       ??1bad_array_new_length@std@@UEAA@XZ 000000018000db64 f i LIBCMT:throw_bad_alloc.obj
 0001:0000cb64       ??1bad_alloc@std@@UEAA@XZ  000000018000db64 f i LIBCMT:throw_bad_alloc.obj
 0001:0000cb78       ??_Ebad_alloc@std@@UEAAPEAXI@Z 000000018000db78 f i LIBCMT:throw_bad_alloc.obj
 0001:0000cb78       ??_Gbad_alloc@std@@UEAAPEAXI@Z 000000018000db78 f i LIBCMT:throw_bad_alloc.obj
 0001:0000cb78       ??_Eexception@std@@UEAAPEAXI@Z 000000018000db78 f i LIBCMT:throw_bad_alloc.obj
 0001:0000cb78       ??_Gbad_array_new_length@std@@UEAAPEAXI@Z 000000018000db78 f i LIBCMT:throw_bad_alloc.obj
 0001:0000cb78       ??_Gexception@std@@UEAAPEAXI@Z 000000018000db78 f i LIBCMT:throw_bad_alloc.obj
 0001:0000cb78       ??_Ebad_array_new_length@std@@UEAAPEAXI@Z 000000018000db78 f i LIBCMT:throw_bad_alloc.obj
 0001:0000cbbc       ?__scrt_throw_std_bad_alloc@@YAXXZ 000000018000dbbc f   LIBCMT:throw_bad_alloc.obj
 0001:0000cbdc       ?__scrt_throw_std_bad_array_new_length@@YAXXZ 000000018000dbdc f   LIBCMT:throw_bad_alloc.obj
 0001:0000cbfc       ?what@exception@std@@UEBAPEBDXZ 000000018000dbfc f i LIBCMT:throw_bad_alloc.obj
 0001:0000cc10       ??3@YAXPEAX@Z              000000018000dc10 f   LIBCMT:delete_scalar.obj
 0001:0000cc18       __security_init_cookie     000000018000dc18 f   LIBCMT:gs_support.obj
 0001:0000ccc4       _get_startup_argv_mode     000000018000dcc4 f   LIBCMT:argv_mode.obj
 0001:0000ccc4       DllMain                    000000018000dcc4 f   LIBCMT:dll_dllmain_stub.obj
 0001:0000cccc       ?__scrt_initialize_type_info@@YAXXZ 000000018000dccc f   LIBCMT:tncleanup.obj
 0001:0000ccdc       ?__scrt_uninitialize_type_info@@YAXXZ 000000018000dcdc f   LIBCMT:tncleanup.obj
 0001:0000cce8       __local_stdio_printf_options 000000018000dce8 f i LIBCMT:default_local_stdio_options.obj
 0001:0000ccf0       __local_stdio_scanf_options 000000018000dcf0 f i LIBCMT:default_local_stdio_options.obj
 0001:0000ccf8       __scrt_initialize_default_local_stdio_options 000000018000dcf8 f   LIBCMT:default_local_stdio_options.obj
 0001:0000cd14       __scrt_acquire_startup_lock 000000018000dd14 f   LIBCMT:utility.obj
 0001:0000cd50       __scrt_dllmain_after_initialize_c 000000018000dd50 f   LIBCMT:utility.obj
 0001:0000cd84       __scrt_dllmain_before_initialize_c 000000018000dd84 f   LIBCMT:utility.obj
 0001:0000cd9c       __scrt_dllmain_crt_thread_attach 000000018000dd9c f   LIBCMT:utility.obj
 0001:0000cdc4       __scrt_dllmain_crt_thread_detach 000000018000ddc4 f   LIBCMT:utility.obj
 0001:0000cddc       __scrt_dllmain_exception_filter 000000018000dddc f   LIBCMT:utility.obj
 0001:0000ce3c       __scrt_dllmain_uninitialize_c 000000018000de3c f   LIBCMT:utility.obj
 0001:0000ce6c       __scrt_dllmain_uninitialize_critical 000000018000de6c f   LIBCMT:utility.obj
 0001:0000ce80       __scrt_initialize_crt      000000018000de80 f   LIBCMT:utility.obj
 0001:0000cecc       __scrt_initialize_onexit_tables 000000018000decc f   LIBCMT:utility.obj
 0001:0000cf58       __scrt_is_nonwritable_in_current_image 000000018000df58 f   LIBCMT:utility.obj
 0001:0000cff0       __scrt_release_startup_lock 000000018000dff0 f   LIBCMT:utility.obj
 0001:0000d014       __scrt_uninitialize_crt    000000018000e014 f   LIBCMT:utility.obj
 0001:0000d040       __scrt_get_dyn_tls_init_callback 000000018000e040 f   LIBCMT:dyn_tls_init.obj
 0001:0000d048       __crt_debugger_hook        000000018000e048 f   LIBCMT:utility_desktop.obj
 0001:0000d050       __scrt_fastfail            000000018000e050 f   LIBCMT:utility_desktop.obj
 0001:0000d19c       _RTC_Initialize            000000018000e19c f   LIBCMT:initsect.obj
 0001:0000d1d8       _RTC_Terminate             000000018000e1d8 f   LIBCMT:initsect.obj
 0001:0000d214       ??_Gtype_info@@UEAAPEAXI@Z 000000018000e214 f i LIBCMT:std_type_info_static.obj
 0001:0000d214       ??_Etype_info@@UEAAPEAXI@Z 000000018000e214 f i LIBCMT:std_type_info_static.obj
 0001:0000d240       __isa_available_init       000000018000e240 f   LIBCMT:cpu_disp.obj
 0001:0000d3e4       __scrt_is_ucrt_dll_in_use  000000018000e3e4 f   LIBCMT:ucrt_detection.obj
 0001:0000d400       memset_repmovs             000000018000e400 f   libvcruntime:memset.obj
 0001:0000d420       memset                     000000018000e420 f   libvcruntime:memset.obj
 0001:0000d5b0       __C_specific_handler       000000018000e5b0 f   libvcruntime:riscchandler.obj
 0001:0000d7bc       __std_exception_copy       000000018000e7bc f   libvcruntime:std_exception.obj
 0001:0000d84c       __std_exception_destroy    000000018000e84c f   libvcruntime:std_exception.obj
 0001:0000d874       _CxxThrowException         000000018000e874 f   libvcruntime:throw.obj
 0001:0000d914       __std_type_info_destroy_list 000000018000e914 f   libvcruntime:std_type_info.obj
 0001:0000d940       __vcrt_initialize          000000018000e940 f   libvcruntime:initialization.obj
 0001:0000d968       __vcrt_thread_attach       000000018000e968 f   libvcruntime:initialization.obj
 0001:0000d97c       __vcrt_thread_detach       000000018000e97c f   libvcruntime:initialization.obj
 0001:0000d990       __vcrt_uninitialize        000000018000e990 f   libvcruntime:initialization.obj
 0001:0000d9ac       __vcrt_uninitialize_critical 000000018000e9ac f   libvcruntime:initialization.obj
 0001:0000d9bc       __DestructExceptionObject  000000018000e9bc f   libvcruntime:ehhelpers.obj
 0001:0000da2c       ?_CallMemberFunction0@@YAXQEAX0@Z 000000018000ea2c f i libvcruntime:ehhelpers.obj
 0001:0000da40       _NLG_Notify                000000018000ea40 f   libvcruntime:notify.obj
 0001:0000da60       __NLG_Dispatch2            000000018000ea60 f   libvcruntime:notify.obj
 0001:0000da70       __NLG_Return2              000000018000ea70 f   libvcruntime:notify.obj
 0001:0000da74       __except_validate_context_record 000000018000ea74 f   libvcruntime:jbcxrval.obj
 0001:0000daac       __vcrt_freefls             000000018000eaac f   libvcruntime:per_thread_data.obj
 0001:0000dacc       __vcrt_freeptd             000000018000eacc f   libvcruntime:per_thread_data.obj
 0001:0000db1c       __vcrt_getptd              000000018000eb1c f   libvcruntime:per_thread_data.obj
 0001:0000db38       __vcrt_getptd_noexit       000000018000eb38 f   libvcruntime:per_thread_data.obj
 0001:0000dbf8       __vcrt_initialize_ptd      000000018000ebf8 f   libvcruntime:per_thread_data.obj
 0001:0000dc40       __vcrt_uninitialize_ptd    000000018000ec40 f   libvcruntime:per_thread_data.obj
 0001:0000dc64       __vcrt_initialize_locks    000000018000ec64 f   libvcruntime:locks.obj
 0001:0000dc98       __vcrt_uninitialize_locks  000000018000ec98 f   libvcruntime:locks.obj
 0001:0000dce0       memcpy_repmovs             000000018000ece0 f   libvcruntime:memcpy.obj
 0001:0000dd00       memmove                    000000018000ed00 f   libvcruntime:memcpy.obj
 0001:0000dd00       memcpy                     000000018000ed00 f   libvcruntime:memcpy.obj
 0001:0000e234       __vcrt_FlsAlloc            000000018000f234 f   libvcruntime:winapi_downlevel.obj
 0001:0000e27c       __vcrt_FlsFree             000000018000f27c f   libvcruntime:winapi_downlevel.obj
 0001:0000e2c4       __vcrt_FlsGetValue         000000018000f2c4 f   libvcruntime:winapi_downlevel.obj
 0001:0000e30c       __vcrt_FlsSetValue         000000018000f30c f   libvcruntime:winapi_downlevel.obj
 0001:0000e360       __vcrt_InitializeCriticalSectionEx 000000018000f360 f   libvcruntime:winapi_downlevel.obj
 0001:0000e3e0       _CallSettingFrame          000000018000f3e0 f   libvcruntime:handlers.obj
 0001:0000e430       _CallSettingFrame_LookupContinuationIndex 000000018000f430 f   libvcruntime:handlers.obj
 0001:0000e460       _CallSettingFrame_NotifyContinuationAddr 000000018000f460 f   libvcruntime:handlers.obj
 0001:0000e490       _CallSettingFrameEncoded   000000018000f490 f   libvcruntime:handlers.obj
 0001:0000e4d8       __acrt_initialize_new_handler 000000018000f4d8 f   libucrt:new_handler.obj
 0001:0000e4e0       _callnewh                  000000018000f4e0 f   libucrt:new_handler.obj
 0001:0000e510       _query_new_handler         000000018000f510 f   libucrt:new_handler.obj
 0001:0000e544       malloc                     000000018000f544 f   libucrt:malloc.obj
 0001:0000e54c       _initterm                  000000018000f54c f   libucrt:initterm.obj
 0001:0000e5b0       _initterm_e                000000018000f5b0 f   libucrt:initterm.obj
 0001:0000e5f0       free                       000000018000f5f0 f   libucrt:free.obj
 0001:0000e604       _seh_filter_dll            000000018000f604 f   libucrt:exception_filter.obj
 0001:0000e618       _seh_filter_exe            000000018000f618 f   libucrt:exception_filter.obj
 0001:0000ea08       __acrt_initialize_thread_local_exit_callback 000000018000fa08 f   libucrt:exit.obj
 0001:0000ea10       _cexit                     000000018000fa10 f   libucrt:exit.obj
 0001:0000ea20       _exit                      000000018000fa20 f   libucrt:exit.obj
 0001:0000ea2c       _is_c_termination_complete 000000018000fa2c f   libucrt:exit.obj
 0001:0000ebf8       __acrt_allocate_buffer_for_argv 000000018000fbf8 f   libucrt:argv_parsing.obj
 0001:0000ec58       _configure_narrow_argv     000000018000fc58 f   libucrt:argv_parsing.obj
 0001:0000efd0       __dcrt_uninitialize_environments_nolock 000000018000ffd0 f   libucrt:environment_initialization.obj
 0001:0000f008       _initialize_narrow_environment 0000000180010008 f   libucrt:environment_initialization.obj
 0001:0000f164       _execute_onexit_table      0000000180010164 f   libucrt:onexit.obj
 0001:0000f1a0       _initialize_onexit_table   00000001800101a0 f   libucrt:onexit.obj
 0001:0000f200       __acrt_uninitialize_command_line 0000000180010200 f   libucrt:argv_data.obj
 0001:0000f2f8       __acrt_initialize          00000001800102f8 f   libucrt:initialization.obj
 0001:0000f30c       __acrt_thread_attach       000000018001030c f   libucrt:initialization.obj
 0001:0000f320       __acrt_thread_detach       0000000180010320 f   libucrt:initialization.obj
 0001:0000f330       __acrt_uninitialize        0000000180010330 f   libucrt:initialization.obj
 0001:0000f368       __acrt_uninitialize_critical 0000000180010368 f   libucrt:initialization.obj
 0001:0000f378       terminate                  0000000180010378 f   libucrt:terminate.obj
 0001:0000f398       strcpy_s                   0000000180010398 f   libucrt:strcpy_s.obj
 0001:0000f3f8       abort                      00000001800103f8 f   libucrt:abort.obj
 0001:0000f450       ??0_LocaleUpdate@@QEAA@QEAU__crt_locale_pointers@@@Z 0000000180010450 f i libucrt:output.obj
 0001:0000f500       strncmp                    0000000180010500 f   libucrt:strncmp.obj
 0001:0000f580       calloc                     0000000180010580 f   libucrt:calloc.obj
 0001:0000f588       wcsncmp                    0000000180010588 f   libucrt:wcsncmp.obj
 0001:0000f5b4       __acrt_initialize_locks    00000001800105b4 f   libucrt:locks.obj
 0001:0000f5fc       __acrt_lock                00000001800105fc f   libucrt:locks.obj
 0001:0000f618       __acrt_uninitialize_locks  0000000180010618 f   libucrt:locks.obj
 0001:0000f650       __acrt_unlock              0000000180010650 f   libucrt:locks.obj
 0001:0000f66c       _malloc_base               000000018001066c f   libucrt:malloc_base.obj
 0001:0000f6cc       _free_base                 00000001800106cc f   libucrt:free_base.obj
 0001:0000fa84       __acrt_freeptd             0000000180010a84 f   libucrt:per_thread_data.obj
 0001:0000fac8       __acrt_getptd              0000000180010ac8 f   libucrt:per_thread_data.obj
 0001:0000fb9c       __acrt_getptd_head         0000000180010b9c f   libucrt:per_thread_data.obj
 0001:0000fc44       __acrt_getptd_noexit       0000000180010c44 f   libucrt:per_thread_data.obj
 0001:0000fd10       __acrt_initialize_ptd      0000000180010d10 f   libucrt:per_thread_data.obj
 0001:0000fd4c       __acrt_uninitialize_ptd    0000000180010d4c f   libucrt:per_thread_data.obj
 0001:0000fd70       __acrt_get_process_end_policy 0000000180010d70 f   libucrt:win_policies.obj
 0001:0000fdac       __acrt_call_reportfault    0000000180010dac f   libucrt:invalid_parameter.obj
 0001:0000ff08       __acrt_initialize_invalid_parameter_handler 0000000180010f08 f   libucrt:invalid_parameter.obj
 0001:0000ff10       _invalid_parameter         0000000180010f10 f   libucrt:invalid_parameter.obj
 0001:0000ffc0       _invalid_parameter_noinfo  0000000180010fc0 f   libucrt:invalid_parameter.obj
 0001:0000ffe0       _invoke_watson             0000000180010fe0 f   libucrt:invalid_parameter.obj
 0001:00010028       __acrt_errno_from_os_error 0000000180011028 f   libucrt:errno.obj
 0001:00010070       __acrt_errno_map_os_error  0000000180011070 f   libucrt:errno.obj
 0001:000100c0       __doserrno                 00000001800110c0 f   libucrt:errno.obj
 0001:000100e0       _errno                     00000001800110e0 f   libucrt:errno.obj
 0001:00010100       _calloc_base               0000000180011100 f   libucrt:calloc_base.obj
 0001:0001018c       ??$__acrt_mbs_to_wcs_cp@U__crt_win32_buffer_internal_dynamic_resizing@@@@YAHQEBDAEAV?$__crt_win32_buffer@_WU__crt_win32_buffer_internal_dynamic_resizing@@@@I@Z 000000018001118c f i libucrt:argv_wildcards.obj
 0001:00010304       ??$__acrt_wcs_to_mbs_cp@U__crt_win32_buffer_internal_dynamic_resizing@@@@YAHQEB_WAEAV?$__crt_win32_buffer@DU__crt_win32_buffer_internal_dynamic_resizing@@@@I@Z 0000000180011304 f i libucrt:argv_wildcards.obj
 0001:00010b34       __acrt_expand_narrow_argv_wildcards 0000000180011b34 f   libucrt:argv_wildcards.obj
 0001:00010b3c       ??$__acrt_wcs_to_mbs_cp@U__crt_win32_buffer_no_resizing@@@@YAHQEB_WAEAV?$__crt_win32_buffer@DU__crt_win32_buffer_no_resizing@@@@I@Z 0000000180011b3c f i libucrt:getmodulefilenamea.obj
 0001:00010c50       __acrt_GetModuleFileNameA  0000000180011c50 f   libucrt:getmodulefilenamea.obj
 0001:0001149c       __acrt_initialize_multibyte 000000018001249c f   libucrt:mbctype.obj
 0001:000114fc       __acrt_update_thread_multibyte_data 00000001800124fc f   libucrt:mbctype.obj
 0001:00011518       _setmbcp_nolock            0000000180012518 f   libucrt:mbctype.obj
 0001:0001184c       _ismbblead                 000000018001284c f   libucrt:ismbbyte.obj
 0001:00011860       __acrt_initialize_command_line 0000000180012860 f   libucrt:argv_data.obj
 0001:00011888       __acrt_MultiByteToWideChar 0000000180012888 f   libucrt:multibytetowidechar.obj
 0001:000118e4       __acrt_WideCharToMultiByte 00000001800128e4 f   libucrt:widechartomultibyte.obj
 0001:0001197c       __dcrt_get_narrow_environment_from_os 000000018001297c f   libucrt:get_environment_from_os.obj
 0001:00011a80       _recalloc_base             0000000180012a80 f   libucrt:recalloc.obj
 0001:00011cf0       __acrt_AppPolicyGetProcessTerminationMethodInternal 0000000180012cf0 f   libucrt:winapi_thunks.obj
 0001:00011d40       __acrt_AreFileApisANSI     0000000180012d40 f   libucrt:winapi_thunks.obj
 0001:00011d7c       __acrt_FlsAlloc            0000000180012d7c f   libucrt:winapi_thunks.obj
 0001:00011dc4       __acrt_FlsFree             0000000180012dc4 f   libucrt:winapi_thunks.obj
 0001:00011e0c       __acrt_FlsGetValue         0000000180012e0c f   libucrt:winapi_thunks.obj
 0001:00011e54       __acrt_FlsSetValue         0000000180012e54 f   libucrt:winapi_thunks.obj
 0001:00011ea8       __acrt_InitializeCriticalSectionEx 0000000180012ea8 f   libucrt:winapi_thunks.obj
 0001:00011f0c       __acrt_LCMapStringEx       0000000180012f0c f   libucrt:winapi_thunks.obj
 0001:00011fe8       __acrt_LocaleNameToLCID    0000000180012fe8 f   libucrt:winapi_thunks.obj
 0001:00012038       __acrt_initialize_winapi_thunks 0000000180013038 f   libucrt:winapi_thunks.obj
 0001:0001206c       __acrt_uninitialize_winapi_thunks 000000018001306c f   libucrt:winapi_thunks.obj
 0001:000120b0       __acrt_initialize_heap     00000001800130b0 f   libucrt:heap_handle.obj
 0001:000120cc       __acrt_uninitialize_heap   00000001800130cc f   libucrt:heap_handle.obj
 0001:000122d4       __acrt_initialize_lowio    00000001800132d4 f   libucrt:ioinit.obj
 0001:00012310       __acrt_uninitialize_lowio  0000000180013310 f   libucrt:ioinit.obj
 0001:00012350       __acrt_execute_initializers 0000000180013350 f   libucrt:shared_initialization.obj
 0001:000123d0       __acrt_execute_uninitializers 00000001800133d0 f   libucrt:shared_initialization.obj
 0001:00012454       __acrt_get_sigabrt_handler 0000000180013454 f   libucrt:signal.obj
 0001:00012484       __acrt_initialize_signal_handlers 0000000180013484 f   libucrt:signal.obj
 0001:000124a4       raise                      00000001800134a4 f   libucrt:signal.obj
 0001:00012710       __acrt_has_user_matherr    0000000180013710 f   libucrt:matherr.obj
 0001:00012730       __acrt_initialize_user_matherr 0000000180013730 f   libucrt:matherr.obj
 0001:00012738       __acrt_invoke_user_matherr 0000000180013738 f   libucrt:matherr.obj
 0001:00012944       __acrt_stdio_flush_nolock  0000000180013944 f   libucrt:fflush.obj
 0001:000129c0       _fflush_nolock             00000001800139c0 f   libucrt:fflush.obj
 0001:00012a0c       _flushall                  0000000180013a0c f   libucrt:fflush.obj
 0001:00012a14       __acrt_initialize_stdio    0000000180013a14 f   libucrt:_file.obj
 0001:00012b34       __acrt_uninitialize_stdio  0000000180013b34 f   libucrt:_file.obj
 0001:00012b90       _lock_file                 0000000180013b90 f   libucrt:_file.obj
 0001:00012b9c       _unlock_file               0000000180013b9c f   libucrt:_file.obj
 0001:00012ba8       _mbtowc_l                  0000000180013ba8 f   libucrt:mbtowc.obj
 0001:00012d28       mbtowc                     0000000180013d28 f   libucrt:mbtowc.obj
 0001:00012d30       __acrt_update_locale_info  0000000180013d30 f   libucrt:locale_update.obj
 0001:00012d64       __acrt_update_multibyte_info 0000000180013d64 f   libucrt:locale_update.obj
 0001:00012d98       _fileno                    0000000180013d98 f   libucrt:fileno.obj
 0001:00012e30       __acrt_set_locale_changed  0000000180013e30 f   libucrt:wsetlocale.obj
 0001:00012e3c       __acrt_uninitialize_locale 0000000180013e3c f   libucrt:wsetlocale.obj
 0001:00012e6c       __pctype_func              0000000180013e6c f   libucrt:ctype.obj
 0001:00012e9c       _query_new_mode            0000000180013e9c f   libucrt:new_mode.obj
 0001:00012ea4       __acrt_add_locale_ref      0000000180013ea4 f   libucrt:locale_refcounting.obj
 0001:00012f30       __acrt_free_locale         0000000180013f30 f   libucrt:locale_refcounting.obj
 0001:000130a8       __acrt_locale_add_lc_time_reference 00000001800140a8 f   libucrt:locale_refcounting.obj
 0001:000130d0       __acrt_locale_free_lc_time_if_unreferenced 00000001800140d0 f   libucrt:locale_refcounting.obj
 0001:00013108       __acrt_locale_release_lc_time_reference 0000000180014108 f   libucrt:locale_refcounting.obj
 0001:00013130       __acrt_release_locale_ref  0000000180014130 f   libucrt:locale_refcounting.obj
 0001:000131d8       __acrt_update_thread_locale_data 00000001800141d8 f   libucrt:locale_refcounting.obj
 0001:00013244       _updatetlocinfoEx_nolock   0000000180014244 f   libucrt:locale_refcounting.obj
 0001:000132b0       qsort                      00000001800142b0 f   libucrt:qsort.obj
 0001:00013660       strncpy_s                  0000000180014660 f   libucrt:strncpy_s.obj
 0001:000137e0       strpbrk                    00000001800147e0 f   libucrt:strpbrk.obj
 0001:00013bc0       _mbsdec                    0000000180014bc0 f   libucrt:mbsdec.obj
 0001:00013bc8       _mbsdec_l                  0000000180014bc8 f   libucrt:mbsdec.obj
 0001:00013c5c       __acrt_GetStringTypeA      0000000180014c5c f   libucrt:getstringtypea.obj
 0001:00014104       __acrt_LCMapStringA        0000000180015104 f   libucrt:lcmapstringa.obj
 0001:000141b4       _msize_base                00000001800151b4 f   libucrt:msize.obj
 0001:000141f0       _realloc_base              00000001800151f0 f   libucrt:realloc_base.obj
 0001:0001426c       __acrt_DownlevelLocaleNameToLCID 000000018001526c f   libucrt:lcidtoname_downlevel.obj
 0001:0001431c       __acrt_lowio_create_handle_array 000000018001531c f   libucrt:osfinfo.obj
 0001:000143c4       __acrt_lowio_destroy_handle_array 00000001800153c4 f   libucrt:osfinfo.obj
 0001:00014414       __acrt_lowio_ensure_fh_exists 0000000180015414 f   libucrt:osfinfo.obj
 0001:000144bc       __acrt_lowio_lock_fh       00000001800154bc f   libucrt:osfinfo.obj
 0001:000144e4       __acrt_lowio_unlock_fh     00000001800154e4 f   libucrt:osfinfo.obj
 0001:0001450c       _free_osfhnd               000000018001550c f   libucrt:osfinfo.obj
 0001:000145c8       _get_osfhandle             00000001800155c8 f   libucrt:osfinfo.obj
 0001:000146cc       _commit                    00000001800156cc f   libucrt:commit.obj
 0001:00014fc0       _write                     0000000180015fc0 f   libucrt:write.obj
 0001:000150ac       _write_nolock              00000001800160ac f   libucrt:write.obj
 0001:00015388       _fcloseall                 0000000180016388 f   libucrt:closeall.obj
 0001:0001543c       __acrt_stdio_free_buffer_nolock 000000018001643c f   libucrt:_freebuf.obj
 0001:0001547c       _isatty                    000000018001647c f   libucrt:isatty.obj
 0001:000154dc       _isleadbyte_l              00000001800164dc f i libucrt:_wctype.obj
 0001:00015528       ?__mbrtowc_utf8@__crt_mbstring@@YA_KPEA_WPEBD_KPEAU_Mbstatet@@@Z 0000000180016528 f   libucrt:mbrtowc.obj
 0001:00015564       ?__mbsrtowcs_utf8@__crt_mbstring@@YA_KPEA_WPEAPEBD_KPEAU_Mbstatet@@@Z 0000000180016564 f   libucrt:mbrtowc.obj
 0001:000156dc       __acrt_locale_free_monetary 00000001800166dc f   libucrt:initmon.obj
 0001:000157e8       __acrt_locale_free_numeric 00000001800167e8 f   libucrt:initnum.obj
 0001:000158ac       __acrt_locale_free_time    00000001800168ac f   libucrt:inittime.obj
 0001:000159b4       __strncnt                  00000001800169b4 f   libucrt:strncnt.obj
 0001:000159cc       __ascii_wcsnicmp           00000001800169cc f   libucrt:wcsnicmp.obj
 0001:00015a18       _query_app_type            0000000180016a18 f   libucrt:report_runtime_error.obj
 0001:00015abc       _lseeki64_nolock           0000000180016abc f   libucrt:lseek.obj
 0001:00015ac4       _putwch_nolock             0000000180016ac4 f   libucrt:putwch.obj
 0001:00015b00       _fclose_nolock             0000000180016b00 f   libucrt:fclose.obj
 0001:00015b84       fclose                     0000000180016b84 f   libucrt:fclose.obj
 0001:00015be8       ?__mbrtoc32_utf8@__crt_mbstring@@YA_KPEA_UPEBD_KPEAU_Mbstatet@@@Z 0000000180016be8 f   libucrt:mbrtoc32.obj
 0001:00015dd0       log10                      0000000180016dd0 f   libucrt:log10.obj
 0001:0001637c       __dcrt_lowio_ensure_console_output_initialized 000000018001737c f   libucrt:initcon.obj
 0001:000163d0       __dcrt_terminate_console_output 00000001800173d0 f   libucrt:initcon.obj
 0001:000163ec       __dcrt_write_console       00000001800173ec f   libucrt:initcon.obj
 0001:00016520       _close                     0000000180017520 f   libucrt:close.obj
 0001:000165c4       _close_nolock              00000001800175c4 f   libucrt:close.obj
 0001:00016684       ?__acrt_stdio_free_stream@@YAXV__crt_stdio_stream@@@Z 0000000180017684 f   libucrt:stream.obj
 0001:000167c4       _handle_error              00000001800177c4 f   libucrt:libm_error.obj
 0001:000168f0       __acrt_initialize_fma3     00000001800178f0 f   libucrt:fma3_available.obj
 0001:00016960       _log10_special             0000000180017960 f   libucrt:log_special.obj
 0001:00016a30       _get_fpsr                  0000000180017a30 f   libucrt:fpsr.obj
 0001:00016a40       _set_fpsr                  0000000180017a40 f   libucrt:fpsr.obj
 0001:00016a4a       _fclrf                     0000000180017a4a f   libucrt:fpsr.obj
 0001:00016a5e       _frnd                      0000000180017a5e f   libucrt:fpsr.obj
 0001:00016a80       _raise_exc                 0000000180017a80 f   libucrt:fpexcept.obj
 0001:00016aa8       _raise_exc_ex              0000000180017aa8 f   libucrt:fpexcept.obj
 0001:00016db8       _set_errno_from_matherr    0000000180017db8 f   libucrt:fpexcept.obj
 0001:00016de8       _clrfp                     0000000180017de8 f   libucrt:fpctrl.obj
 0001:00016e08       _ctrlfp                    0000000180017e08 f   libucrt:fpctrl.obj
 0001:00016e84       _set_statfp                0000000180017e84 f   libucrt:fpctrl.obj
 0001:00016ea4       _statfp                    0000000180017ea4 f   libucrt:fpctrl.obj
 0001:00016eb5       IsProcessorFeaturePresent  0000000180017eb5 f   kernel32:KERNEL32.dll
 0001:00016ec0       _FindPESection             0000000180017ec0 f   LIBCMT:pesect.obj
 0001:00016f10       _IsNonwritableInCurrentImage 0000000180017f10 f   LIBCMT:pesect.obj
 0001:00016f60       _ValidateImageBase         0000000180017f60 f   LIBCMT:pesect.obj
 0001:00016f90       __GSHandlerCheck           0000000180017f90 f   LIBCMT:gshandler.obj
 0001:00016fb0       __GSHandlerCheckCommon     0000000180017fb0 f   LIBCMT:gshandler.obj
 0001:00017020       __security_check_cookie    0000000180018020 f   LIBCMT:amdsecgs.obj
 0001:00017044       __raise_securityfailure    0000000180018044 f   LIBCMT:gs_report.obj
 0001:00017078       __report_gsfailure         0000000180018078 f   LIBCMT:gs_report.obj
 0001:0001714c       __report_rangecheckfailure 000000018001814c f   LIBCMT:gs_report.obj
 0001:00017160       __report_securityfailure   0000000180018160 f   LIBCMT:gs_report.obj
 0001:000172f0       memcmp                     00000001800182f0 f   libvcruntime:memcmp.obj
 0001:000173d0       _guard_dispatch_icall_nop  00000001800183d0 f   LIBCMT:guard_dispatch.obj
 0001:00018308       _TI2?AVbad_alloc@std@@     0000000180019308     LIBCMT:throw_bad_alloc.obj
 0001:00018328       _CTA2?AVbad_alloc@std@@    0000000180019328     LIBCMT:throw_bad_alloc.obj
 0001:00018340       _CT??_R0?AVbad_alloc@std@@@8??0bad_alloc@std@@QEAA@AEBV01@@Z24 0000000180019340     LIBCMT:throw_bad_alloc.obj
 0001:00018368       _CT??_R0?AVexception@std@@@8??0exception@std@@QEAA@AEBV01@@Z24 0000000180019368     LIBCMT:throw_bad_alloc.obj
 0001:00018390       _TI3?AVbad_array_new_length@std@@ 0000000180019390     LIBCMT:throw_bad_alloc.obj
 0001:000183b0       _CTA3?AVbad_array_new_length@std@@ 00000001800193b0     LIBCMT:throw_bad_alloc.obj
 0001:000183d0       _CT??_R0?AVbad_array_new_length@std@@@8??0bad_array_new_length@std@@QEAA@AEBV01@@Z24 00000001800193d0     LIBCMT:throw_bad_alloc.obj
 0002:00000070       __scrt_native_dllmain_reason 000000018001a070     LIBCMT:utility.obj
 0002:00000078       __security_cookie_complement 000000018001a078     LIBCMT:gs_cookie.obj
 0002:00000080       __security_cookie          000000018001a080     LIBCMT:gs_cookie.obj
 0002:00000088       __isa_available            000000018001a088     LIBCMT:cpu_disp.obj
 0002:0000008c       __isa_enabled              000000018001a08c     LIBCMT:cpu_disp.obj
 0002:00000090       __memcpy_nt_iters          000000018001a090     LIBCMT:cpu_disp.obj
 0002:00000098       __memset_nt_iters          000000018001a098     LIBCMT:cpu_disp.obj
 0002:000000b0       __abort_behavior           000000018001a0b0     libucrt:abort.obj
 0002:000000d0       __acrt_initial_multibyte_data 000000018001a0d0     libucrt:mbctype.obj
 0002:00000610       __acrt_initial_locale_data 000000018001a610     libucrt:nlsdata.obj
 0002:00000768       __acrt_initial_locale_pointers 000000018001a768     libucrt:nlsdata.obj
 0002:00000778       __acrt_wide_c_locale_string 000000018001a778     libucrt:nlsdata.obj
 0002:00000780       _iob                       000000018001a780     libucrt:_file.obj
 0002:00000888       __globallocalestatus       000000018001a888     libucrt:glstatus.obj
 0002:00000890       __acrt_lconv_c             000000018001a890     libucrt:localeconv.obj
 0002:00000928       __acrt_lconv_static_decimal 000000018001a928     libucrt:localeconv.obj
 0002:0000092c       __acrt_lconv_static_W_decimal 000000018001a92c     libucrt:localeconv.obj
 0002:00000930       _lookuptrailbytes          000000018001a930     libucrt:read.obj
 0002:00000a50       _fltused                   000000018001aa50     LIBCMT:fltused.obj
 0002:00000a60       ??_R0?AVbad_alloc@std@@@8  000000018001aa60     LIBCMT:throw_bad_alloc.obj
 0002:00000a88       ??_R0?AVexception@std@@@8  000000018001aa88     LIBCMT:throw_bad_alloc.obj
 0002:00000ab0       ??_R0?AVbad_array_new_length@std@@@8 000000018001aab0     LIBCMT:throw_bad_alloc.obj
 0002:00000ae0       ??_R0?AVtype_info@@@8      000000018001aae0     LIBCMT:std_type_info_static.obj
 0002:00000cf0       ?__type_info_root_node@@3U__type_info_node@@A 000000018001acf0     LIBCMT:tncleanup.obj
 0002:00000d00       ?_OptionsStorage@?1??__local_stdio_printf_options@@9@4_KA 000000018001ad00     LIBCMT:default_local_stdio_options.obj
 0002:00000d08       ?_OptionsStorage@?1??__local_stdio_scanf_options@@9@4_KA 000000018001ad08     LIBCMT:default_local_stdio_options.obj
 0002:00000d10       __scrt_current_native_startup_state 000000018001ad10     LIBCMT:utility.obj
 0002:00000d18       __scrt_native_startup_lock 000000018001ad18     LIBCMT:utility.obj
 0002:00000d58       __scrt_debugger_hook_flag  000000018001ad58     LIBCMT:utility_desktop.obj
 0002:00000d5c       __favor                    000000018001ad5c     LIBCMT:cpu_disp.obj
 0002:00000d60       ?__WinRTOutOfMemoryExceptionCallback@@3P6APEAXXZEA 000000018001ad60     libvcruntime:ehhelpers.obj
 0002:00000d68       ?pArgList@UnDecorator@@0PEAVReplicator@@EA 000000018001ad68     libvcruntime:undname.obj
 0002:00000d70       ?pZNameList@UnDecorator@@0PEAVReplicator@@EA 000000018001ad70     libvcruntime:undname.obj
 0002:00000d78       ?pTemplateArgList@UnDecorator@@0PEAVReplicator@@EA 000000018001ad78     libvcruntime:undname.obj
 0002:00000d80       ?gName@UnDecorator@@0PEBDEB 000000018001ad80     libvcruntime:undname.obj
 0002:00000d88       ?name@UnDecorator@@0PEBDEB 000000018001ad88     libvcruntime:undname.obj
 0002:00000d90       ?disableFlags@UnDecorator@@0KA 000000018001ad90     libvcruntime:undname.obj
 0002:00000d94       ?fExplicitTemplateParams@UnDecorator@@0_NA 000000018001ad94     libvcruntime:undname.obj
 0002:00000d95       ?fGetTemplateArgumentList@UnDecorator@@0_NA 000000018001ad95     libvcruntime:undname.obj
 0002:00000d98       ?m_pGetParameter@UnDecorator@@0P6APEADJ@ZEA 000000018001ad98     libvcruntime:undname.obj
 0002:00000da0       ?m_CHPENameOffset@UnDecorator@@0KA 000000018001ada0     libvcruntime:undname.obj
 0002:00000da4       ?m_recursionLevel@UnDecorator@@0KA 000000018001ada4     libvcruntime:undname.obj
 0002:00000ec0       __pPurecall                000000018001aec0     libvcruntime:purevirt_data.obj
 0002:00000ee0       ?c_exit_complete@?1???R<lambda_6e4b09c48022b2350581041d5f6b0c4c>@@QEBA@XZ@4_NA 000000018001aee0     libucrt:exit.obj
 0002:00000ff8       _environ_table             000000018001aff8     libucrt:environment_initialization.obj
 0002:00001000       _wenviron_table            000000018001b000     libucrt:environment_initialization.obj
 0002:00001008       __dcrt_initial_wide_environment 000000018001b008     libucrt:environment_initialization.obj
 0002:00001010       __dcrt_initial_narrow_environment 000000018001b010     libucrt:environment_initialization.obj
 0002:00001018       __acrt_atexit_table        000000018001b018     libucrt:onexit.obj
 0002:00001030       __acrt_at_quick_exit_table 000000018001b030     libucrt:onexit.obj
 0002:00001290       _mbctype                   000000018001b290     libucrt:mbctype.obj
 0002:00001298       _mbcasemap                 000000018001b298     libucrt:mbctype.obj
 0002:000012a0       __acrt_current_multibyte_data 000000018001b2a0     libucrt:mbctype.obj
 0002:000012b0       _pgmptr                    000000018001b2b0     libucrt:argv_data.obj
 0002:000012b8       __argc                     000000018001b2b8     libucrt:argv_data.obj
 0002:000012c0       __argv                     000000018001b2c0     libucrt:argv_data.obj
 0002:000012c8       __wargv                    000000018001b2c8     libucrt:argv_data.obj
 0002:000012d0       _acmdln                    000000018001b2d0     libucrt:argv_data.obj
 0002:000012d8       _wcmdln                    000000018001b2d8     libucrt:argv_data.obj
 0002:00001490       __acrt_heap                000000018001b490     libucrt:heap_handle.obj
 0002:000014a0       __pioinfo                  000000018001b4a0     libucrt:ioinit.obj
 0002:000018a0       _nhandle                   000000018001b8a0     libucrt:ioinit.obj
 0002:000018d0       __acrt_current_locale_data 000000018001b8d0     libucrt:nlsdata.obj
 0002:000018d8       _nstream                   000000018001b8d8     libucrt:_file.obj
 0002:000018e0       __piob                     000000018001b8e0     libucrt:_file.obj
 0002:000018e8       __acrt_stdout_buffer       000000018001b8e8     libucrt:_sftbuf.obj
 0002:000018f0       __acrt_stderr_buffer       000000018001b8f0     libucrt:_sftbuf.obj
 0002:00001900       __acrt_locale_changed_data 000000018001b900     libucrt:wsetlocale.obj
 0002:00001908       __acrt_lconv_static_null   000000018001b908     libucrt:localeconv.obj
 0002:0000190c       __acrt_lconv_static_W_null 000000018001b90c     libucrt:localeconv.obj
 0002:00001920       __fma3_is_available        000000018001b920     libucrt:fma3_available.obj
 0002:00001924       __use_fma3_lib             000000018001b924     libucrt:fma3_available.obj
 0002:00001ea0       __scrt_ucrt_dll_is_in_use  000000018001bea0     <common>
 0002:00001ea8       __dyn_tls_init_callback    000000018001bea8     <common>
 0004:00000000       __imp_lstrcmpiW            000000018001d000     kernel32:KERNEL32.dll
 0004:00000008       __imp_lstrcpynW            000000018001d008     kernel32:KERNEL32.dll
 0004:00000010       __imp_lstrlenW             000000018001d010     kernel32:KERNEL32.dll
 0004:00000018       __imp_WriteConsoleW        000000018001d018     kernel32:KERNEL32.dll
 0004:00000020       __imp_CloseHandle          000000018001d020     kernel32:KERNEL32.dll
 0004:00000028       __imp_CreateFileW          000000018001d028     kernel32:KERNEL32.dll
 0004:00000030       __imp_QueryPerformanceCounter 000000018001d030     kernel32:KERNEL32.dll
 0004:00000038       __imp_GetCurrentProcessId  000000018001d038     kernel32:KERNEL32.dll
 0004:00000040       __imp_GetCurrentThreadId   000000018001d040     kernel32:KERNEL32.dll
 0004:00000048       __imp_GetSystemTimeAsFileTime 000000018001d048     kernel32:KERNEL32.dll
 0004:00000050       __imp_InitializeSListHead  000000018001d050     kernel32:KERNEL32.dll
 0004:00000058       __imp_RtlCaptureContext    000000018001d058     kernel32:KERNEL32.dll
 0004:00000060       __imp_RtlLookupFunctionEntry 000000018001d060     kernel32:KERNEL32.dll
 0004:00000068       __imp_RtlVirtualUnwind     000000018001d068     kernel32:KERNEL32.dll
 0004:00000070       __imp_IsDebuggerPresent    000000018001d070     kernel32:KERNEL32.dll
 0004:00000078       __imp_UnhandledExceptionFilter 000000018001d078     kernel32:KERNEL32.dll
 0004:00000080       __imp_SetUnhandledExceptionFilter 000000018001d080     kernel32:KERNEL32.dll
 0004:00000088       __imp_GetStartupInfoW      000000018001d088     kernel32:KERNEL32.dll
 0004:00000090       __imp_IsProcessorFeaturePresent 000000018001d090     kernel32:KERNEL32.dll
 0004:00000098       __imp_GetModuleHandleW     000000018001d098     kernel32:KERNEL32.dll
 0004:000000a0       __imp_RtlUnwindEx          000000018001d0a0     kernel32:KERNEL32.dll
 0004:000000a8       __imp_RtlPcToFileHeader    000000018001d0a8     kernel32:KERNEL32.dll
 0004:000000b0       __imp_RaiseException       000000018001d0b0     kernel32:KERNEL32.dll
 0004:000000b8       __imp_InterlockedFlushSList 000000018001d0b8     kernel32:KERNEL32.dll
 0004:000000c0       __imp_GetLastError         000000018001d0c0     kernel32:KERNEL32.dll
 0004:000000c8       __imp_SetLastError         000000018001d0c8     kernel32:KERNEL32.dll
 0004:000000d0       __imp_EnterCriticalSection 000000018001d0d0     kernel32:KERNEL32.dll
 0004:000000d8       __imp_LeaveCriticalSection 000000018001d0d8     kernel32:KERNEL32.dll
 0004:000000e0       __imp_DeleteCriticalSection 000000018001d0e0     kernel32:KERNEL32.dll
 0004:000000e8       __imp_InitializeCriticalSectionAndSpinCount 000000018001d0e8     kernel32:KERNEL32.dll
 0004:000000f0       __imp_TlsAlloc             000000018001d0f0     kernel32:KERNEL32.dll
 0004:000000f8       __imp_TlsGetValue          000000018001d0f8     kernel32:KERNEL32.dll
 0004:00000100       __imp_TlsSetValue          000000018001d100     kernel32:KERNEL32.dll
 0004:00000108       __imp_TlsFree              000000018001d108     kernel32:KERNEL32.dll
 0004:00000110       __imp_FreeLibrary          000000018001d110     kernel32:KERNEL32.dll
 0004:00000118       __imp_GetProcAddress       000000018001d118     kernel32:KERNEL32.dll
 0004:00000120       __imp_LoadLibraryExW       000000018001d120     kernel32:KERNEL32.dll
 0004:00000128       __imp_GetCurrentProcess    000000018001d128     kernel32:KERNEL32.dll
 0004:00000130       __imp_ExitProcess          000000018001d130     kernel32:KERNEL32.dll
 0004:00000138       __imp_TerminateProcess     000000018001d138     kernel32:KERNEL32.dll
 0004:00000140       __imp_GetModuleHandleExW   000000018001d140     kernel32:KERNEL32.dll
 0004:00000148       __imp_GetModuleFileNameW   000000018001d148     kernel32:KERNEL32.dll
 0004:00000150       __imp_HeapAlloc            000000018001d150     kernel32:KERNEL32.dll
 0004:00000158       __imp_HeapFree             000000018001d158     kernel32:KERNEL32.dll
 0004:00000160       __imp_FindClose            000000018001d160     kernel32:KERNEL32.dll
 0004:00000168       __imp_FindFirstFileExW     000000018001d168     kernel32:KERNEL32.dll
 0004:00000170       __imp_FindNextFileW        000000018001d170     kernel32:KERNEL32.dll
 0004:00000178       __imp_IsValidCodePage      000000018001d178     kernel32:KERNEL32.dll
 0004:00000180       __imp_GetACP               000000018001d180     kernel32:KERNEL32.dll
 0004:00000188       __imp_GetOEMCP             000000018001d188     kernel32:KERNEL32.dll
 0004:00000190       __imp_GetCPInfo            000000018001d190     kernel32:KERNEL32.dll
 0004:00000198       __imp_GetCommandLineA      000000018001d198     kernel32:KERNEL32.dll
 0004:000001a0       __imp_GetCommandLineW      000000018001d1a0     kernel32:KERNEL32.dll
 0004:000001a8       __imp_MultiByteToWideChar  000000018001d1a8     kernel32:KERNEL32.dll
 0004:000001b0       __imp_WideCharToMultiByte  000000018001d1b0     kernel32:KERNEL32.dll
 0004:000001b8       __imp_GetEnvironmentStringsW 000000018001d1b8     kernel32:KERNEL32.dll
 0004:000001c0       __imp_FreeEnvironmentStringsW 000000018001d1c0     kernel32:KERNEL32.dll
 0004:000001c8       __imp_LCMapStringW         000000018001d1c8     kernel32:KERNEL32.dll
 0004:000001d0       __imp_GetProcessHeap       000000018001d1d0     kernel32:KERNEL32.dll
 0004:000001d8       __imp_GetStdHandle         000000018001d1d8     kernel32:KERNEL32.dll
 0004:000001e0       __imp_GetFileType          000000018001d1e0     kernel32:KERNEL32.dll
 0004:000001e8       __imp_GetStringTypeW       000000018001d1e8     kernel32:KERNEL32.dll
 0004:000001f0       __imp_HeapSize             000000018001d1f0     kernel32:KERNEL32.dll
 0004:000001f8       __imp_HeapReAlloc          000000018001d1f8     kernel32:KERNEL32.dll
 0004:00000200       __imp_SetStdHandle         000000018001d200     kernel32:KERNEL32.dll
 0004:00000208       __imp_FlushFileBuffers     000000018001d208     kernel32:KERNEL32.dll
 0004:00000210       __imp_WriteFile            000000018001d210     kernel32:KERNEL32.dll
 0004:00000218       __imp_GetConsoleCP         000000018001d218     kernel32:KERNEL32.dll
 0004:00000220       __imp_GetConsoleMode       000000018001d220     kernel32:KERNEL32.dll
 0004:00000228       __imp_SetFilePointerEx     000000018001d228     kernel32:KERNEL32.dll
 0004:00000230       \177KERNEL32_NULL_THUNK_DATA 000000018001d230     kernel32:KERNEL32.dll
 0004:00000238       __imp_MessageBeep          000000018001d238     user32:USER32.dll
 0004:00000240       \177USER32_NULL_THUNK_DATA 000000018001d240     user32:USER32.dll
 0004:00000248       __guard_check_icall_fptr   000000018001d248     LIBCMT:guard_support.obj
 0004:00000250       __guard_dispatch_icall_fptr 000000018001d250     LIBCMT:guard_support.obj
 0004:00000258       __IMPORT_DESCRIPTOR_KERNEL32 000000018001d258     kernel32:KERNEL32.dll
 0004:0000026c       __IMPORT_DESCRIPTOR_USER32 000000018001d26c     user32:USER32.dll
 0004:00000280       __NULL_IMPORT_DESCRIPTOR   000000018001d280     kernel32:KERNEL32.dll

 entry point at        0001:0000ca38

 Static symbols

 0001:000004d0       ?tokenTable@@3QBUStringLiteral@@B 00000001800014d0     libvcruntime:undname.obj
 0001:000005d0       ?nameTable@@3QBUStringLiteral@@B 00000001800015d0     libvcruntime:undname.obj
 0001:00000b00       ?rttiTable@@3QBUStringLiteral@@B 0000000180001b00     libvcruntime:undname.obj
 0001:00000b50       ?IndirectionName@@3QBUStringLiteral@@B 0000000180001b50     libvcruntime:undname.obj
 0001:00000bb0       ?PrefixName@@3QBUStringLiteral@@B 0000000180001bb0     libvcruntime:undname.obj
 0001:00001288       ?module_names@?A0x81a78551@@3QBQEB_WB 0000000180002288     libvcruntime:winapi_downlevel.obj
 0001:00001348       ?candidate_modules@?1??try_get_FlsAlloc@@YAP6AKP6AXPEAX@Z@ZXZ@4QBW4module_id@?A0x81a78551@@B 0000000180002348     libvcruntime:winapi_downlevel.obj
 0001:00001360       ?candidate_modules@?1??try_get_FlsFree@@YAP6AHK@ZXZ@4QBW4module_id@?A0x81a78551@@B 0000000180002360     libvcruntime:winapi_downlevel.obj
 0001:00001370       ?candidate_modules@?1??try_get_FlsGetValue@@YAP6APEAXK@ZXZ@4QBW4module_id@?A0x81a78551@@B 0000000180002370     libvcruntime:winapi_downlevel.obj
 0001:00001388       ?candidate_modules@?1??try_get_FlsSetValue@@YAP6AHKPEAX@ZXZ@4QBW4module_id@?A0x81a78551@@B 0000000180002388     libvcruntime:winapi_downlevel.obj
 0001:000013a0       ?candidate_modules@?1??try_get_InitializeCriticalSectionEx@@YAP6AHPEAU_RTL_CRITICAL_SECTION@@KK@ZXZ@4QBW4module_id@?A0x81a78551@@B 00000001800023a0     libvcruntime:winapi_downlevel.obj
 0001:000014d0       __acrt_initializers        00000001800024d0     libucrt:initialization.obj
 0001:000015d0       ?errtable@@3QBUerrentry@?A0x31fdb9ec@@B 00000001800025d0     libucrt:errno.obj
 0001:00001738       ?_mb_locale_names@@3QBQEB_WB 0000000180002738     libucrt:mbctype.obj
 0001:000017a0       ?module_names@?A0x391cf84c@@3QBQEB_WB 00000001800027a0     libucrt:winapi_thunks.obj
 0001:00001ca8       ?candidate_modules@?1??try_get_AreFileApisANSI@@YAP6AHXZXZ@4QBW4module_id@?A0x391cf84c@@B 0000000180002ca8     libucrt:winapi_thunks.obj
 0001:00001cc0       ?candidate_modules@?1??try_get_FlsAlloc@@YAP6AKP6AXPEAX@Z@ZXZ@4QBW4module_id@?A0x391cf84c@@B 0000000180002cc0     libucrt:winapi_thunks.obj
 0001:00001cc8       ?candidate_modules@?1??try_get_FlsFree@@YAP6AHK@ZXZ@4QBW4module_id@?A0x391cf84c@@B 0000000180002cc8     libucrt:winapi_thunks.obj
 0001:00001cd0       ?candidate_modules@?1??try_get_FlsGetValue@@YAP6APEAXK@ZXZ@4QBW4module_id@?A0x391cf84c@@B 0000000180002cd0     libucrt:winapi_thunks.obj
 0001:00001cd8       ?candidate_modules@?1??try_get_FlsSetValue@@YAP6AHKPEAX@ZXZ@4QBW4module_id@?A0x391cf84c@@B 0000000180002cd8     libucrt:winapi_thunks.obj
 0001:00001ce0       ?candidate_modules@?1??try_get_InitializeCriticalSectionEx@@YAP6AHPEAU_RTL_CRITICAL_SECTION@@KK@ZXZ@4QBW4module_id@?A0x391cf84c@@B 0000000180002ce0     libucrt:winapi_thunks.obj
 0001:00001ce8       ?candidate_modules@?1??try_get_LCMapStringEx@@YAP6AHPEB_WK0HPEA_WHPEAU_nlsversioninfo@@PEAX_J@ZXZ@4QBW4module_id@?A0x391cf84c@@B 0000000180002ce8     libucrt:winapi_thunks.obj
 0001:00001d00       ?candidate_modules@?1??try_get_LocaleNameToLCID@@YAP6AKPEB_WK@ZXZ@4QBW4module_id@?A0x391cf84c@@B 0000000180002d00     libucrt:winapi_thunks.obj
 0001:00001d1c       ?candidate_modules@?1??try_get_AppPolicyGetProcessTerminationMethod@@YAP6AJPEAXPEAW4AppPolicyProcessTerminationMethod@@@ZXZ@4QBW4module_id@?A0x391cf84c@@B 0000000180002d1c     libucrt:winapi_thunks.obj
 0001:000029d0       ?LcidToLocaleNameTable@?A0x881e4c05@@3QBULcidToLocaleName@1@B 00000001800039d0     libucrt:lcidtoname_downlevel.obj
 0001:00004430       ?LocaleNameToIndexTable@?A0x881e4c05@@3QBULocaleNameIndex@1@B 0000000180005430     libucrt:lcidtoname_downlevel.obj
 0001:00005cd0       __real_ninf                0000000180006cd0     libucrt:log10.obj
 0001:00005ce0       __real_inf                 0000000180006ce0     libucrt:log10.obj
 0001:00005cf0       __real_neg_qnan            0000000180006cf0     libucrt:log10.obj
 0001:00005d00       __real_qnanbit             0000000180006d00     libucrt:log10.obj
 0001:00005d10       __int_1023                 0000000180006d10     libucrt:log10.obj
 0001:00005d20       __mask_001                 0000000180006d20     libucrt:log10.obj
 0001:00005d30       __mask_mant                0000000180006d30     libucrt:log10.obj
 0001:00005d40       __mask_mant_top8           0000000180006d40     libucrt:log10.obj
 0001:00005d50       __mask_mant9               0000000180006d50     libucrt:log10.obj
 0001:00005d60       __real_log10_e             0000000180006d60     libucrt:log10.obj
 0001:00005d70       __real_log10_e_lead        0000000180006d70     libucrt:log10.obj
 0001:00005d80       __real_log10_e_tail        0000000180006d80     libucrt:log10.obj
 0001:00005d90       __real_log10_2_lead        0000000180006d90     libucrt:log10.obj
 0001:00005da0       __real_log10_2_tail        0000000180006da0     libucrt:log10.obj
 0001:00005db0       __real_two                 0000000180006db0     libucrt:log10.obj
 0001:00005dc0       __real_one                 0000000180006dc0     libucrt:log10.obj
 0001:00005dd0       __real_half                0000000180006dd0     libucrt:log10.obj
 0001:00005de0       __mask_100                 0000000180006de0     libucrt:log10.obj
 0001:00005df0       __real_1_over_512          0000000180006df0     libucrt:log10.obj
 0001:00005e00       __real_1_over_2            0000000180006e00     libucrt:log10.obj
 0001:00005e10       __real_1_over_3            0000000180006e10     libucrt:log10.obj
 0001:00005e20       __real_1_over_4            0000000180006e20     libucrt:log10.obj
 0001:00005e30       __real_1_over_5            0000000180006e30     libucrt:log10.obj
 0001:00005e40       __real_1_over_6            0000000180006e40     libucrt:log10.obj
 0001:00005e50       __real_neg_1023            0000000180006e50     libucrt:log10.obj
 0001:00005e60       __mask_2045                0000000180006e60     libucrt:log10.obj
 0001:00005e70       __real_threshold           0000000180006e70     libucrt:log10.obj
 0001:00005e80       __real_near_one_lt         0000000180006e80     libucrt:log10.obj
 0001:00005e90       __real_near_one_gt         0000000180006e90     libucrt:log10.obj
 0001:00005ea0       __real_min_norm            0000000180006ea0     libucrt:log10.obj
 0001:00005eb0       __real_notsign             0000000180006eb0     libucrt:log10.obj
 0001:00005ec0       __real_ca1                 0000000180006ec0     libucrt:log10.obj
 0001:00005ed0       __real_ca2                 0000000180006ed0     libucrt:log10.obj
 0001:00005ee0       __real_ca3                 0000000180006ee0     libucrt:log10.obj
 0001:00005ef0       __real_ca4                 0000000180006ef0     libucrt:log10.obj
 0001:00005f00       __mask_lower               0000000180006f00     libucrt:log10.obj
 0001:00005f10       __flag_x_zero              0000000180006f10     libucrt:log10.obj
 0001:00005f14       __flag_x_neg               0000000180006f14     libucrt:log10.obj
 0001:00005f18       __flag_x_nan               0000000180006f18     libucrt:log10.obj
 0001:00007770       __real@433fffffffffffff    0000000180008770     libucrt:fpsr.obj
 0001:00007778       __real@c33fffffffffffff    0000000180008778     libucrt:fpsr.obj
 0001:00007780       GS_ExceptionPointers       0000000180008780     LIBCMT:gs_report.obj
 0001:00007d90       $$000000                   0000000180008d90     chkstk.obj
 0001:000082ac       $LN39                      00000001800092ac     Brackets.obj
 0001:0000ad80       $LN649                     000000018000bd80     Brackets.obj
 0001:0000adb0       $LN648                     000000018000bdb0     Brackets.obj
 0001:0000ade0       $LN647                     000000018000bde0     Brackets.obj
 0001:0000ae10       $LN646                     000000018000be10     Brackets.obj
 0001:0000ae40       $LN645                     000000018000be40     Brackets.obj
 0001:0000b544       $LN36                      000000018000c544     Brackets.obj
 0001:0000c718       ?dllmain_crt_dispatch@@YAHQEAUHINSTANCE__@@KQEAX@Z 000000018000d718 f   LIBCMT:dll_dllmain.obj
 0001:0000c768       ?dllmain_crt_process_attach@@YAHQEAUHINSTANCE__@@QEAX@Z 000000018000d768 f   LIBCMT:dll_dllmain.obj
 0001:0000c880       ?dllmain_crt_process_detach@@YAH_N@Z 000000018000d880 f   LIBCMT:dll_dllmain.obj
 0001:0000c904       ?dllmain_dispatch@@YAHQEAUHINSTANCE__@@KQEAX@Z 000000018000d904 f   LIBCMT:dll_dllmain.obj
 0001:0000d3f0       $$000000                   000000018000e3f0     libvcruntime:memset.obj
 0001:0000da30       $$000000                   000000018000ea30     libvcruntime:notify.obj
 0001:0000dcd0       $$000000                   000000018000ecd0     libvcruntime:memcpy.obj
 0001:0000e0d8       ?try_get_function@@YAPEAXW4function_id@?A0x81a78551@@QEBDQEBW4module_id@2@2@Z 000000018000f0d8 f   libvcruntime:winapi_downlevel.obj
 0001:0000e3d0       $$000000                   000000018000f3d0     libvcruntime:handlers.obj
 0001:0000e79c       ??$?RV<lambda_d80eeec6fff315bfe5c115232f3240e3>@@AEAV<lambda_6e4b09c48022b2350581041d5f6b0c4c>@@V<lambda_2358e3775559c9db80273638284d5e45>@@@?$__crt_seh_guarded_call@X@@QEAAX$$QEAV<lambda_d80eeec6fff315bfe5c115232f3240e3>@@AEAV<lambda_6e4b09c48022b2350581041d5f6b0c4c>@@$$QEAV<lambda_2358e3775559c9db80273638284d5e45>@@@Z 000000018000f79c f   libucrt:exit.obj
 0001:0000e7d4       ??R<lambda_6e4b09c48022b2350581041d5f6b0c4c>@@QEBA@XZ 000000018000f7d4 f   libucrt:exit.obj
 0001:0000e898       ?atexit_exception_filter@@YAHK@Z 000000018000f898 f   libucrt:exit.obj
 0001:0000e8a4       ?common_exit@@YAXHW4_crt_exit_cleanup_mode@@W4_crt_exit_return_mode@@@Z 000000018000f8a4 f   libucrt:exit.obj
 0001:0000e960       ?exit_or_terminate_process@@YAXI@Z 000000018000f960 f   libucrt:exit.obj
 0001:0000e9ac       ?try_cor_exit_process@@YAXI@Z 000000018000f9ac f   libucrt:exit.obj
 0001:0000ea34       ??$parse_command_line@D@@YAXPEADPEAPEAD0PEA_K2@Z 000000018000fa34 f   libucrt:argv_parsing.obj
 0001:0000ede0       ??$common_initialize_environment_nolock@D@@YAHXZ 000000018000fde0 f   libucrt:environment_initialization.obj
 0001:0000ee4c       ??$create_environment@D@@YAQEAPEADQEAD@Z 000000018000fe4c f   libucrt:environment_initialization.obj
 0001:0000ef54       ??$free_environment@D@@YAXQEAPEAD@Z 000000018000ff54 f   libucrt:environment_initialization.obj
 0001:0000ef54       ??$free_environment@_W@@YAXQEAPEA_W@Z 000000018000ff54 f   libucrt:environment_initialization.obj
 0001:0000ef98       ??$uninitialize_environment_internal@D@@YAXAEAPEAPEAD@Z 000000018000ff98 f   libucrt:environment_initialization.obj
 0001:0000efb4       ??$uninitialize_environment_internal@_W@@YAXAEAPEAPEA_W@Z 000000018000ffb4 f   libucrt:environment_initialization.obj
 0001:0000f010       ??$?RV<lambda_7777bce6b2f8c936911f934f8298dc43>@@AEAV<lambda_f03950bc5685219e0bcd2087efbe011e>@@V<lambda_3883c3dff614d5e0c5f61bb1ac94921c>@@@?$__crt_seh_guarded_call@H@@QEAAH$$QEAV<lambda_7777bce6b2f8c936911f934f8298dc43>@@AEAV<lambda_f03950bc5685219e0bcd2087efbe011e>@@$$QEAV<lambda_3883c3dff614d5e0c5f61bb1ac94921c>@@@Z 0000000180010010 f   libucrt:onexit.obj
 0001:0000f04c       ??R<lambda_f03950bc5685219e0bcd2087efbe011e>@@QEBAHXZ 000000018001004c f   libucrt:onexit.obj
 0001:0000f1c8       initialize_global_variables 00000001800101c8 f   libucrt:initialization.obj
 0001:0000f1dc       initialize_c               00000001800101dc f   libucrt:initialization.obj
 0001:0000f200       initialize_environment     0000000180010200 f   libucrt:initialization.obj
 0001:0000f200       initialize_global_state_isolation 0000000180010200 f   libucrt:initialization.obj
 0001:0000f200       report_memory_leaks        0000000180010200 f   libucrt:initialization.obj
 0001:0000f200       uninitialize_c             0000000180010200 f   libucrt:initialization.obj
 0001:0000f200       uninitialize_global_state_isolation 0000000180010200 f   libucrt:initialization.obj
 0001:0000f204       uninitialize_environment   0000000180010204 f   libucrt:initialization.obj
 0001:0000f214       initialize_pointers        0000000180010214 f   libucrt:initialization.obj
 0001:0000f254       uninitialize_vcruntime     0000000180010254 f   libucrt:initialization.obj
 0001:0000f25c       uninitialize_allocated_memory 000000018001025c f   libucrt:initialization.obj
 0001:0000f29c       uninitialize_allocated_io_buffers 000000018001029c f   libucrt:initialization.obj
 0001:0000f4f0       $$000000                   00000001800104f0     libucrt:strncmp.obj
 0001:0000f70c       ??$?RV<lambda_0ae27a3a962d80f24befdcbee591983d>@@AEAV<lambda_8d0ee55de4b1038c4002e0adecdf1839>@@V<lambda_dc504788e8f1664fe9b84e20bfb512f2>@@@?$__crt_seh_guarded_call@X@@QEAAX$$QEAV<lambda_0ae27a3a962d80f24befdcbee591983d>@@AEAV<lambda_8d0ee55de4b1038c4002e0adecdf1839>@@$$QEAV<lambda_dc504788e8f1664fe9b84e20bfb512f2>@@@Z 000000018001070c f   libucrt:per_thread_data.obj
 0001:0000f74c       ??$?RV<lambda_2d41944a1d46af3157314b8a01080d33>@@AEAV<lambda_8f455de75cd7d7f24b4096f044d8b9e6>@@V<lambda_aa500f224e6afead328df44964fe2772>@@@?$__crt_seh_guarded_call@X@@QEAAX$$QEAV<lambda_2d41944a1d46af3157314b8a01080d33>@@AEAV<lambda_8f455de75cd7d7f24b4096f044d8b9e6>@@$$QEAV<lambda_aa500f224e6afead328df44964fe2772>@@@Z 000000018001074c f   libucrt:per_thread_data.obj
 0001:0000f78c       ??$?RV<lambda_aa87e3671a710a21b5dc78c0bdf72e11>@@AEAV<lambda_92619d2358a28f41a33ba319515a20b9>@@V<lambda_6992ecaafeb10aed2b74cb1fae11a551>@@@?$__crt_seh_guarded_call@X@@QEAAX$$QEAV<lambda_aa87e3671a710a21b5dc78c0bdf72e11>@@AEAV<lambda_92619d2358a28f41a33ba319515a20b9>@@$$QEAV<lambda_6992ecaafeb10aed2b74cb1fae11a551>@@@Z 000000018001078c f   libucrt:per_thread_data.obj
 0001:0000f7d4       ??$?RV<lambda_f2e299630e499de9f9a165e60fcd3db5>@@AEAV<lambda_2ae9d31cdba2644fcbeaf08da7c24588>@@V<lambda_40d01ff24d0e7b3814fdbdcee8eab3c7>@@@?$__crt_seh_guarded_call@X@@QEAAX$$QEAV<lambda_f2e299630e499de9f9a165e60fcd3db5>@@AEAV<lambda_2ae9d31cdba2644fcbeaf08da7c24588>@@$$QEAV<lambda_40d01ff24d0e7b3814fdbdcee8eab3c7>@@@Z 00000001800107d4 f   libucrt:per_thread_data.obj
 0001:0000f834       ?construct_ptd_array@@YAXQEAU__acrt_ptd@@@Z 0000000180010834 f   libucrt:per_thread_data.obj
 0001:0000f904       ?destroy_fls@@YAXPEAX@Z    0000000180010904 f   libucrt:per_thread_data.obj
 0001:0000f924       ?destroy_ptd_array@@YAXQEAU__acrt_ptd@@@Z 0000000180010924 f   libucrt:per_thread_data.obj
 0001:0000fa1c       ?replace_current_thread_locale_nolock@@YAXQEAU__acrt_ptd@@QEAU__crt_locale_data@@@Z 0000000180010a1c f   libucrt:per_thread_data.obj
 0001:00010178       ?<lambda_invoker_cdecl>@<lambda_a1ce4c8ae42411fd470c77163914f50e>@@CAHPEBX0@Z 0000000180011178 f   libucrt:argv_wildcards.obj
 0001:00010490       ??$common_expand_argv_wildcards@D@@YAHQEAPEADQEAPEAPEAD@Z 0000000180011490 f   libucrt:argv_wildcards.obj
 0001:0001069c       ??$copy_and_add_argument_to_buffer@D@@YAHQEBD0_KAEAV?$argument_list@D@?A0x5f5c8891@@@Z 000000018001169c f   libucrt:argv_wildcards.obj
 0001:00010824       ??$expand_argument_wildcards@D@@YAHQEAD0AEAV?$argument_list@D@?A0x5f5c8891@@@Z 0000000180011824 f   libucrt:argv_wildcards.obj
 0001:00010d70       ??$?RV<lambda_efdfa57d1f175319df784efa44bb7b81>@@AEAV<lambda_5f0a4c1567f8adc6734073e5d1e1b35c>@@V<lambda_2e8a7d3640ea6ccb4c2413664c2db6fd>@@@?$__crt_seh_guarded_call@X@@QEAAX$$QEAV<lambda_efdfa57d1f175319df784efa44bb7b81>@@AEAV<lambda_5f0a4c1567f8adc6734073e5d1e1b35c>@@$$QEAV<lambda_2e8a7d3640ea6ccb4c2413664c2db6fd>@@@Z 0000000180011d70 f   libucrt:mbctype.obj
 0001:00010f2c       ?getSystemCP@@YAHH@Z       0000000180011f2c f   libucrt:mbctype.obj
 0001:00010fac       ?setSBCS@@YAXPEAU__crt_multibyte_data@@@Z 0000000180011fac f   libucrt:mbctype.obj
 0001:0001103c       ?setSBUpLow@@YAXPEAU__crt_multibyte_data@@@Z 000000018001203c f   libucrt:mbctype.obj
 0001:00011220       ?setmbcp_internal@@YAHH_NQEAU__acrt_ptd@@QEAPEAU__crt_multibyte_data@@@Z 0000000180012220 f   libucrt:mbctype.obj
 0001:000113e4       ?update_thread_multibyte_data_internal@@YAPEAU__crt_multibyte_data@@QEAU__acrt_ptd@@QEAPEAU1@@Z 00000001800123e4 f   libucrt:mbctype.obj
 0001:000117d4       ?x_ismbbtype_l@@YAHPEAU__crt_locale_pointers@@IHH@Z 00000001800127d4 f   libucrt:ismbbyte.obj
 0001:00011b18       ?try_get_function@@YAPEAXW4function_id@?A0x391cf84c@@QEBDQEBW4module_id@2@2@Z 0000000180012b18 f   libucrt:winapi_thunks.obj
 0001:000120d8       ?initialize_inherited_file_handles_nolock@@YAXXZ 00000001800130d8 f   libucrt:ioinit.obj
 0001:000121c8       ?initialize_stdio_handles_nolock@@YAXXZ 00000001800131c8 f   libucrt:ioinit.obj
 0001:0001240c       ??$?RV<lambda_450d765d439847d4c735a33c368b5fc0>@@AEAV<lambda_44731a7d0e6d81c3e6aa82d741081786>@@V<lambda_601a2a7da3b7a96e9554ac7215c4b07c>@@@?$__crt_seh_guarded_call@P6AXH@Z@@QEAAP6AXH@Z$$QEAV<lambda_450d765d439847d4c735a33c368b5fc0>@@AEAV<lambda_44731a7d0e6d81c3e6aa82d741081786>@@$$QEAV<lambda_601a2a7da3b7a96e9554ac7215c4b07c>@@@Z 000000018001340c f   libucrt:signal.obj
 0001:00012768       ??$?RV<lambda_842d9ff0dc9ef11c61343bbaebe7f885>@@AEAV<lambda_c5860995281e5c4ce005b3de8f5874ee>@@V<lambda_d90129c13df834fdcbf8d2b88dafcf2d>@@@?$__crt_seh_guarded_call@X@@QEAAX$$QEAV<lambda_842d9ff0dc9ef11c61343bbaebe7f885>@@AEAV<lambda_c5860995281e5c4ce005b3de8f5874ee>@@$$QEAV<lambda_d90129c13df834fdcbf8d2b88dafcf2d>@@@Z 0000000180013768 f   libucrt:fflush.obj
 0001:00012804       ??$?RV<lambda_886d6c58226a84441f68b9f2b8217b83>@@AEAV<lambda_ab61a845afdef5b7c387490eaf3616ee>@@V<lambda_f7f22ab5edc0698d5f6905b0d3f44752>@@@?$__crt_seh_guarded_call@X@@QEAAX$$QEAV<lambda_886d6c58226a84441f68b9f2b8217b83>@@AEAV<lambda_ab61a845afdef5b7c387490eaf3616ee>@@$$QEAV<lambda_f7f22ab5edc0698d5f6905b0d3f44752>@@@Z 0000000180013804 f   libucrt:fflush.obj
 0001:000128e4       ?common_flush_all@@YAH_N@Z 00000001800138e4 f   libucrt:fflush.obj
 0001:00012dc0       ??$?RV<lambda_410d79af7f07d98d83a3f525b3859a53>@@AEAV<lambda_3e16ef9562a7dcce91392c22ab16ea36>@@V<lambda_38119f0e861e05405d8a144b9b982f0a>@@@?$__crt_seh_guarded_call@X@@QEAAX$$QEAV<lambda_410d79af7f07d98d83a3f525b3859a53>@@AEAV<lambda_3e16ef9562a7dcce91392c22ab16ea36>@@$$QEAV<lambda_38119f0e861e05405d8a144b9b982f0a>@@@Z 0000000180013dc0 f   libucrt:wsetlocale.obj
 0001:00013734       fallbackMethod             0000000180014734 f   libucrt:strpbrk.obj
 0001:00013b04       $LN78                      0000000180014b04     libucrt:strpbrk.obj
 0001:00013b40       $LN77                      0000000180014b40     libucrt:strpbrk.obj
 0001:00013b80       $LN76                      0000000180014b80     libucrt:strpbrk.obj
 0001:00013dec       ?__acrt_LCMapStringA_stat@@YAHPEAU__crt_locale_pointers@@PEB_WKPEBDHPEADHHH@Z 0000000180014dec f   libucrt:lcmapstringa.obj
 0001:0001419c       ?initialize_multibyte@@YAHXZ 000000018001519c f   libucrt:multibyte_initializer.obj
 0001:00014640       ??$?RV<lambda_a37b2b86f63e897a80ea819b0eb08c01>@@AEAV<lambda_38ce7e780aa69e748d6df282ebc68efe>@@V<lambda_99fb1378e971ab6e7edea83e3a7a83a2>@@@?$__crt_seh_guarded_call@H@@QEAAH$$QEAV<lambda_a37b2b86f63e897a80ea819b0eb08c01>@@AEAV<lambda_38ce7e780aa69e748d6df282ebc68efe>@@$$QEAV<lambda_99fb1378e971ab6e7edea83e3a7a83a2>@@@Z 0000000180015640 f   libucrt:commit.obj
 0001:00014760       ?write_double_translated_ansi_nolock@@YA?AUwrite_result@?A0x17268360@@HQEBDI@Z 0000000180015760 f   libucrt:write.obj
 0001:00014c30       ?write_text_ansi_nolock@@YA?AUwrite_result@?A0x17268360@@HQEBDI@Z 0000000180015c30 f   libucrt:write.obj
 0001:00014d34       ?write_text_utf16le_nolock@@YA?AUwrite_result@?A0x17268360@@HQEBDI@Z 0000000180015d34 f   libucrt:write.obj
 0001:00014e50       ?write_text_utf8_nolock@@YA?AUwrite_result@?A0x17268360@@HQEBDI@Z 0000000180015e50 f   libucrt:write.obj
 0001:00015854       ?free_crt_array_internal@@YAXQEAPEBX_K@Z 0000000180016854 f   libucrt:inittime.obj
 0001:00015a20       ??$common_lseek_nolock@_J@@YA_JH_JH@Z 0000000180016a20 f   libucrt:lseek.obj
 0001:00015dd0       $$000000                   0000000180016dd0     libucrt:log10.obj
 0001:000164ac       ??$?RV<lambda_751a882b2c74d4b022dec766aa51a29a>@@AEAV<lambda_628dfdc04ba53c8bfc02c9951375f3f5>@@V<lambda_f6c7be5f7998530c34de24c7437d6b54>@@@?$__crt_seh_guarded_call@H@@QEAAH$$QEAV<lambda_751a882b2c74d4b022dec766aa51a29a>@@AEAV<lambda_628dfdc04ba53c8bfc02c9951375f3f5>@@$$QEAV<lambda_f6c7be5f7998530c34de24c7437d6b54>@@@Z 00000001800174ac f   libucrt:close.obj
 0001:000166a0       _call_matherr              00000001800176a0 f   libucrt:libm_error.obj
 0001:00016708       _exception_enabled         0000000180017708 f   libucrt:libm_error.obj
 0001:00016980       _log_special_common        0000000180017980 f   libucrt:log_special.obj
 0001:00016a20       $$000000                   0000000180017a20     libucrt:fpsr.obj
 0001:00017010       $$000000                   0000000180018010     LIBCMT:amdsecgs.obj
 0001:000171fc       capture_current_context    00000001800181fc f   LIBCMT:gs_report.obj
 0001:0001726c       capture_previous_context   000000018001826c f   LIBCMT:gs_report.obj
 0001:000172e0       $$000000                   00000001800182e0     libvcruntime:memcmp.obj
 0001:000173c0       $$000000                   00000001800183c0     LIBCMT:guard_dispatch.obj
 0001:000173e0       ?fin$0@?0??dllmain_crt_process_attach@@YAHQEAUHINSTANCE__@@QEAX@Z@4HA 00000001800183e0 f   LIBCMT:dll_dllmain.obj
 0001:000173f7       ?fin$0@?0??dllmain_crt_process_detach@@YAH_N@Z@4HA 00000001800183f7 f   LIBCMT:dll_dllmain.obj
 0001:00017410       ?fin$1@?0??dllmain_crt_process_detach@@YAH_N@Z@4HA 0000000180018410 f   LIBCMT:dll_dllmain.obj
 0001:00017424       ?filt$0@?0??dllmain_dispatch@@YAHQEAUHINSTANCE__@@KQEAX@Z@4HA 0000000180018424 f   LIBCMT:dll_dllmain.obj
 0001:0001745a       __scrt_is_nonwritable_in_current_image$filt$0 000000018001845a f   LIBCMT:utility.obj
 0001:00017472       __DestructExceptionObject$filt$0 0000000180018472 f   libvcruntime:ehhelpers.obj
 0001:00017508       _query_new_handler$fin$0   0000000180018508 f   libucrt:new_handler.obj
 0001:0001751e       ?fin$0@?0???$?RV<lambda_0ae27a3a962d80f24befdcbee591983d>@@AEAV<lambda_8d0ee55de4b1038c4002e0adecdf1839>@@V<lambda_dc504788e8f1664fe9b84e20bfb512f2>@@@?$__crt_seh_guarded_call@X@@QEAAX$$QEAV<lambda_0ae27a3a962d80f24befdcbee591983d>@@AEAV<lambda_8d0ee55de4b1038c4002e0adecdf1839>@@$$QEAV<lambda_dc504788e8f1664fe9b84e20bfb512f2>@@@Z@4HA 000000018001851e f   libucrt:per_thread_data.obj
 0001:0001751e       ?fin$0@?0???$?RV<lambda_2d41944a1d46af3157314b8a01080d33>@@AEAV<lambda_8f455de75cd7d7f24b4096f044d8b9e6>@@V<lambda_aa500f224e6afead328df44964fe2772>@@@?$__crt_seh_guarded_call@X@@QEAAX$$QEAV<lambda_2d41944a1d46af3157314b8a01080d33>@@AEAV<lambda_8f455de75cd7d7f24b4096f044d8b9e6>@@$$QEAV<lambda_aa500f224e6afead328df44964fe2772>@@@Z@4HA 000000018001851e f   libucrt:per_thread_data.obj
 0001:0001751e       ?fin$0@?0???$?RV<lambda_aa87e3671a710a21b5dc78c0bdf72e11>@@AEAV<lambda_92619d2358a28f41a33ba319515a20b9>@@V<lambda_6992ecaafeb10aed2b74cb1fae11a551>@@@?$__crt_seh_guarded_call@X@@QEAAX$$QEAV<lambda_aa87e3671a710a21b5dc78c0bdf72e11>@@AEAV<lambda_92619d2358a28f41a33ba319515a20b9>@@$$QEAV<lambda_6992ecaafeb10aed2b74cb1fae11a551>@@@Z@4HA 000000018001851e f   libucrt:per_thread_data.obj
 0001:0001751e       ?fin$0@?0???$?RV<lambda_f2e299630e499de9f9a165e60fcd3db5>@@AEAV<lambda_2ae9d31cdba2644fcbeaf08da7c24588>@@V<lambda_40d01ff24d0e7b3814fdbdcee8eab3c7>@@@?$__crt_seh_guarded_call@X@@QEAAX$$QEAV<lambda_f2e299630e499de9f9a165e60fcd3db5>@@AEAV<lambda_2ae9d31cdba2644fcbeaf08da7c24588>@@$$QEAV<lambda_40d01ff24d0e7b3814fdbdcee8eab3c7>@@@Z@4HA 000000018001851e f   libucrt:per_thread_data.obj
 0001:0001751e       ?fin$0@?0???$?RV<lambda_efdfa57d1f175319df784efa44bb7b81>@@AEAV<lambda_5f0a4c1567f8adc6734073e5d1e1b35c>@@V<lambda_2e8a7d3640ea6ccb4c2413664c2db6fd>@@@?$__crt_seh_guarded_call@X@@QEAAX$$QEAV<lambda_efdfa57d1f175319df784efa44bb7b81>@@AEAV<lambda_5f0a4c1567f8adc6734073e5d1e1b35c>@@$$QEAV<lambda_2e8a7d3640ea6ccb4c2413664c2db6fd>@@@Z@4HA 000000018001851e f   libucrt:mbctype.obj
 0001:0001751e       ?fin$0@?0???$?RV<lambda_450d765d439847d4c735a33c368b5fc0>@@AEAV<lambda_44731a7d0e6d81c3e6aa82d741081786>@@V<lambda_601a2a7da3b7a96e9554ac7215c4b07c>@@@?$__crt_seh_guarded_call@P6AXH@Z@@QEAAP6AXH@Z$$QEAV<lambda_450d765d439847d4c735a33c368b5fc0>@@AEAV<lambda_44731a7d0e6d81c3e6aa82d741081786>@@$$QEAV<lambda_601a2a7da3b7a96e9554ac7215c4b07c>@@@Z@4HA 000000018001851e f   libucrt:signal.obj
 0001:0001751e       ?fin$0@?0???$?RV<lambda_d80eeec6fff315bfe5c115232f3240e3>@@AEAV<lambda_6e4b09c48022b2350581041d5f6b0c4c>@@V<lambda_2358e3775559c9db80273638284d5e45>@@@?$__crt_seh_guarded_call@X@@QEAAX$$QEAV<lambda_d80eeec6fff315bfe5c115232f3240e3>@@AEAV<lambda_6e4b09c48022b2350581041d5f6b0c4c>@@$$QEAV<lambda_2358e3775559c9db80273638284d5e45>@@@Z@4HA 000000018001851e f   libucrt:exit.obj
 0001:0001751e       ?fin$0@?0???$?RV<lambda_7777bce6b2f8c936911f934f8298dc43>@@AEAV<lambda_f03950bc5685219e0bcd2087efbe011e>@@V<lambda_3883c3dff614d5e0c5f61bb1ac94921c>@@@?$__crt_seh_guarded_call@H@@QEAAH$$QEAV<lambda_7777bce6b2f8c936911f934f8298dc43>@@AEAV<lambda_f03950bc5685219e0bcd2087efbe011e>@@$$QEAV<lambda_3883c3dff614d5e0c5f61bb1ac94921c>@@@Z@4HA 000000018001851e f   libucrt:onexit.obj
 0001:00017538       ?filt$0@?0???R<lambda_6e4b09c48022b2350581041d5f6b0c4c>@@QEBA@XZ@4HA 0000000180018538 f   libucrt:exit.obj
 0001:00017553       ?fin$0@?0??update_thread_multibyte_data_internal@@YAPEAU__crt_multibyte_data@@QEAU__acrt_ptd@@QEAPEAU1@@Z@4HA 0000000180018553 f   libucrt:mbctype.obj
 0001:0001756c       __acrt_initialize_lowio$fin$0 000000018001856c f   libucrt:ioinit.obj
 0001:0001756c       __acrt_lowio_ensure_fh_exists$fin$0 000000018001856c f   libucrt:osfinfo.obj
 0001:00017585       raise$fin$0                0000000180018585 f   libucrt:signal.obj
 0001:000175a6       ?fin$0@?0???$?RV<lambda_842d9ff0dc9ef11c61343bbaebe7f885>@@AEAV<lambda_c5860995281e5c4ce005b3de8f5874ee>@@V<lambda_d90129c13df834fdcbf8d2b88dafcf2d>@@@?$__crt_seh_guarded_call@X@@QEAAX$$QEAV<lambda_842d9ff0dc9ef11c61343bbaebe7f885>@@AEAV<lambda_c5860995281e5c4ce005b3de8f5874ee>@@$$QEAV<lambda_d90129c13df834fdcbf8d2b88dafcf2d>@@@Z@4HA 00000001800185a6 f   libucrt:fflush.obj
 0001:000175c1       ?fin$0@?0???$?RV<lambda_886d6c58226a84441f68b9f2b8217b83>@@AEAV<lambda_ab61a845afdef5b7c387490eaf3616ee>@@V<lambda_f7f22ab5edc0698d5f6905b0d3f44752>@@@?$__crt_seh_guarded_call@X@@QEAAX$$QEAV<lambda_886d6c58226a84441f68b9f2b8217b83>@@AEAV<lambda_ab61a845afdef5b7c387490eaf3616ee>@@$$QEAV<lambda_f7f22ab5edc0698d5f6905b0d3f44752>@@@Z@4HA 00000001800185c1 f   libucrt:fflush.obj
 0001:000175de       ?fin$0@?0???$?RV<lambda_410d79af7f07d98d83a3f525b3859a53>@@AEAV<lambda_3e16ef9562a7dcce91392c22ab16ea36>@@V<lambda_38119f0e861e05405d8a144b9b982f0a>@@@?$__crt_seh_guarded_call@X@@QEAAX$$QEAV<lambda_410d79af7f07d98d83a3f525b3859a53>@@AEAV<lambda_3e16ef9562a7dcce91392c22ab16ea36>@@$$QEAV<lambda_38119f0e861e05405d8a144b9b982f0a>@@@Z@4HA 00000001800185de f   libucrt:wsetlocale.obj
 0001:000175f8       __acrt_update_thread_locale_data$fin$0 00000001800185f8 f   libucrt:locale_refcounting.obj
 0001:00017611       ?fin$0@?0???$?RV<lambda_751a882b2c74d4b022dec766aa51a29a>@@AEAV<lambda_628dfdc04ba53c8bfc02c9951375f3f5>@@V<lambda_f6c7be5f7998530c34de24c7437d6b54>@@@?$__crt_seh_guarded_call@H@@QEAAH$$QEAV<lambda_751a882b2c74d4b022dec766aa51a29a>@@AEAV<lambda_628dfdc04ba53c8bfc02c9951375f3f5>@@$$QEAV<lambda_f6c7be5f7998530c34de24c7437d6b54>@@@Z@4HA 0000000180018611 f   libucrt:close.obj
 0001:00017611       ?fin$0@?0???$?RV<lambda_a37b2b86f63e897a80ea819b0eb08c01>@@AEAV<lambda_38ce7e780aa69e748d6df282ebc68efe>@@V<lambda_99fb1378e971ab6e7edea83e3a7a83a2>@@@?$__crt_seh_guarded_call@H@@QEAAH$$QEAV<lambda_a37b2b86f63e897a80ea819b0eb08c01>@@AEAV<lambda_38ce7e780aa69e748d6df282ebc68efe>@@$$QEAV<lambda_99fb1378e971ab6e7edea83e3a7a83a2>@@@Z@4HA 0000000180018611 f   libucrt:commit.obj
 0001:0001762b       _write$fin$0               000000018001862b f   libucrt:write.obj
 0001:00017642       _fcloseall$fin$0           0000000180018642 f   libucrt:closeall.obj
 0001:0001765b       fclose$fin$0               000000018001865b f   libucrt:fclose.obj
 0001:00017673       _ctrlfp$filt$0             0000000180018673 f   libucrt:fpctrl.obj
 0001:000176a0       _IsNonwritableInCurrentImage$filt$0 00000001800186a0 f   LIBCMT:pesect.obj
 0001:000176c0       $xdatasym                  00000001800186c0     chkstk.obj
 0001:000176c8       $unwind$ConfigureW         00000001800186c8     Brackets.obj
 0001:000176c8       $unwind$GetGlobalInfoW     00000001800186c8     Brackets.obj
 0001:000176c8       $unwind$__scrt_initialize_default_local_stdio_options 00000001800186c8     LIBCMT:default_local_stdio_options.obj
 0001:000176c8       $unwind$?dllmain_crt_dispatch@@YAHQEAUHINSTANCE__@@KQEAX@Z 00000001800186c8     LIBCMT:dll_dllmain.obj
 0001:000176c8       $unwind$__report_rangecheckfailure 00000001800186c8     LIBCMT:gs_report.obj
 0001:000176c8       $unwind$__GSHandlerCheck   00000001800186c8     LIBCMT:gshandler.obj
 0001:000176c8       $unwind$__scrt_acquire_startup_lock 00000001800186c8     LIBCMT:utility.obj
 0001:000176c8       $unwind$__scrt_dllmain_after_initialize_c 00000001800186c8     LIBCMT:utility.obj
 0001:000176c8       $unwind$__scrt_dllmain_before_initialize_c 00000001800186c8     LIBCMT:utility.obj
 0001:000176c8       $unwind$__scrt_dllmain_crt_thread_attach 00000001800186c8     LIBCMT:utility.obj
 0001:000176c8       $unwind$__scrt_dllmain_crt_thread_detach 00000001800186c8     LIBCMT:utility.obj
 0001:000176c8       $unwind$__scrt_dllmain_uninitialize_c 00000001800186c8     LIBCMT:utility.obj
 0001:000176c8       $unwind$__scrt_dllmain_uninitialize_critical 00000001800186c8     LIBCMT:utility.obj
 0001:000176c8       $unwind$__vcrt_initialize  00000001800186c8     libvcruntime:initialization.obj
 0001:000176c8       $unwind$__vcrt_thread_attach 00000001800186c8     libvcruntime:initialization.obj
 0001:000176c8       $unwind$__vcrt_thread_detach 00000001800186c8     libvcruntime:initialization.obj
 0001:000176c8       $unwind$__vcrt_uninitialize 00000001800186c8     libvcruntime:initialization.obj
 0001:000176c8       $unwind$__vcrt_uninitialize_critical 00000001800186c8     libvcruntime:initialization.obj
 0001:000176c8       $unwind$__vcrt_initialize_locks 00000001800186c8     libvcruntime:locks.obj
 0001:000176c8       $unwind$__vcrt_freefls     00000001800186c8     libvcruntime:per_thread_data.obj
 0001:000176c8       $unwind$__vcrt_getptd      00000001800186c8     libvcruntime:per_thread_data.obj
 0001:000176c8       $unwind$__vcrt_initialize_ptd 00000001800186c8     libvcruntime:per_thread_data.obj
 0001:000176c8       $unwind$__vcrt_uninitialize_ptd 00000001800186c8     libvcruntime:per_thread_data.obj
 0001:000176c8       $unwind$__dcrt_terminate_console_output 00000001800186c8     libucrt:initcon.obj
 0001:000176c8       $unwind$??$uninitialize_environment_internal@D@@YAXAEAPEAPEAD@Z 00000001800186c8     libucrt:environment_initialization.obj
 0001:000176c8       $unwind$??$uninitialize_environment_internal@_W@@YAXAEAPEAPEA_W@Z 00000001800186c8     libucrt:environment_initialization.obj
 0001:000176c8       $unwind$__dcrt_uninitialize_environments_nolock 00000001800186c8     libucrt:environment_initialization.obj
 0001:000176c8       $unwind$__acrt_initialize_heap 00000001800186c8     libucrt:heap_handle.obj
 0001:000176c8       $unwind$_msize_base        00000001800186c8     libucrt:msize.obj
 0001:000176c8       $unwind$?initialize_multibyte@@YAHXZ 00000001800186c8     libucrt:multibyte_initializer.obj
 0001:000176c8       $unwind$__acrt_thread_attach 00000001800186c8     libucrt:initialization.obj
 0001:000176c8       $unwind$__acrt_thread_detach 00000001800186c8     libucrt:initialization.obj
 0001:000176c8       $unwind$__acrt_uninitialize 00000001800186c8     libucrt:initialization.obj
 0001:000176c8       $unwind$__acrt_uninitialize_critical 00000001800186c8     libucrt:initialization.obj
 0001:000176c8       $unwind$initialize_c       00000001800186c8     libucrt:initialization.obj
 0001:000176c8       $unwind$uninitialize_allocated_io_buffers 00000001800186c8     libucrt:initialization.obj
 0001:000176c8       $unwind$uninitialize_environment 00000001800186c8     libucrt:initialization.obj
 0001:000176c8       $unwind$__acrt_initialize_ptd 00000001800186c8     libucrt:per_thread_data.obj
 0001:000176c8       $unwind$__acrt_uninitialize_ptd 00000001800186c8     libucrt:per_thread_data.obj
 0001:000176c8       $unwind$__acrt_AreFileApisANSI 00000001800186c8     libucrt:winapi_thunks.obj
 0001:000176c8       $unwind$__pctype_func      00000001800186c8     libucrt:ctype.obj
 0001:000176c8       $unwind$__acrt_release_locale_ref 00000001800186c8     libucrt:locale_refcounting.obj
 0001:000176c8       $unwind$_isatty            00000001800186c8     libucrt:isatty.obj
 0001:000176c8       $unwind$_get_osfhandle     00000001800186c8     libucrt:osfinfo.obj
 0001:000176c8       $unwind$__acrt_initialize_multibyte 00000001800186c8     libucrt:mbctype.obj
 0001:000176c8       $unwind$__acrt_update_thread_multibyte_data 00000001800186c8     libucrt:mbctype.obj
 0001:000176c8       $unwind$__doserrno         00000001800186c8     libucrt:errno.obj
 0001:000176c8       $unwind$_errno             00000001800186c8     libucrt:errno.obj
 0001:000176c8       $unwind$_invoke_watson     00000001800186c8     libucrt:invalid_parameter.obj
 0001:000176c8       $unwind$abort              00000001800186c8     libucrt:abort.obj
 0001:000176c8       $unwind$__acrt_initialize_command_line 00000001800186c8     libucrt:argv_data.obj
 0001:000176c8       $unwind$_fileno            00000001800186c8     libucrt:fileno.obj
 0001:000176c8       $unwind$_statfp            00000001800186c8     libucrt:fpctrl.obj
 0001:000176c8       $unwind$_set_errno_from_matherr 00000001800186c8     libucrt:fpexcept.obj
 0001:000176d0       $unwind$??_G?$DialogItemBinding@UFarDialogItem@@@@UEAAPEAXI@Z 00000001800186d0     Brackets.obj
 0001:000176d0       $unwind$??_GPluginCheckBoxBinding@@UEAAPEAXI@Z 00000001800186d0     Brackets.obj
 0001:000176d0       $unwind$??_GPluginEditFieldBinding@@UEAAPEAXI@Z 00000001800186d0     Brackets.obj
 0001:000176d0       $unwind$??_GPluginIntEditFieldBinding@@UEAAPEAXI@Z 00000001800186d0     Brackets.obj
 0001:000176d0       $unwind$??_GPluginRadioButtonBinding@@UEAAPEAXI@Z 00000001800186d0     Brackets.obj
 0001:000176d0       $unwind$??_GPluginUIntEditFieldBinding@@UEAAPEAXI@Z 00000001800186d0     Brackets.obj
 0001:000176d0       $unwind$?SaveValue@PluginCheckBoxBinding@@UEAAXPEAUFarDialogItem@@H@Z 00000001800186d0     Brackets.obj
 0001:000176d0       $unwind$?SaveValue@PluginEditFieldBinding@@UEAAXPEAUFarDialogItem@@H@Z 00000001800186d0     Brackets.obj
 0001:000176d0       $unwind$?SaveValue@PluginIntEditFieldBinding@@UEAAXPEAUFarDialogItem@@H@Z 00000001800186d0     Brackets.obj
 0001:000176d0       $unwind$?SaveValue@PluginUIntEditFieldBinding@@UEAAXPEAUFarDialogItem@@H@Z 00000001800186d0     Brackets.obj
 0001:000176d0       $unwind$GetPluginInfoW     00000001800186d0     Brackets.obj
 0001:000176d0       $unwind$__raise_securityfailure 00000001800186d0     LIBCMT:gs_report.obj
 0001:000176d0       $unwind$??2@YAPEAX_K@Z     00000001800186d0     LIBCMT:new_scalar.obj
 0001:000176d0       $unwind$??_Gtype_info@@UEAAPEAXI@Z 00000001800186d0     LIBCMT:std_type_info_static.obj
 0001:000176d0       $unwind$??0bad_alloc@std@@QEAA@AEBV01@@Z 00000001800186d0     LIBCMT:throw_bad_alloc.obj
 0001:000176d0       $unwind$??0bad_array_new_length@std@@QEAA@AEBV01@@Z 00000001800186d0     LIBCMT:throw_bad_alloc.obj
 0001:000176d0       $unwind$??0exception@std@@QEAA@AEBV01@@Z 00000001800186d0     LIBCMT:throw_bad_alloc.obj
 0001:000176d0       $unwind$__scrt_initialize_crt 00000001800186d0     LIBCMT:utility.obj
 0001:000176d0       $unwind$__scrt_initialize_onexit_tables 00000001800186d0     LIBCMT:utility.obj
 0001:000176d0       $unwind$__scrt_release_startup_lock 00000001800186d0     LIBCMT:utility.obj
 0001:000176d0       $unwind$__scrt_uninitialize_crt 00000001800186d0     LIBCMT:utility.obj
 0001:000176d0       $unwind$__vcrt_uninitialize_locks 00000001800186d0     libvcruntime:locks.obj
 0001:000176d0       $unwind$__vcrt_freeptd     00000001800186d0     libvcruntime:per_thread_data.obj
 0001:000176d0       $unwind$__std_exception_destroy 00000001800186d0     libvcruntime:std_exception.obj
 0001:000176d0       $unwind$__std_type_info_destroy_list 00000001800186d0     libvcruntime:std_type_info.obj
 0001:000176d0       $unwind$__vcrt_FlsAlloc    00000001800186d0     libvcruntime:winapi_downlevel.obj
 0001:000176d0       $unwind$__vcrt_FlsFree     00000001800186d0     libvcruntime:winapi_downlevel.obj
 0001:000176d0       $unwind$__vcrt_FlsGetValue 00000001800186d0     libvcruntime:winapi_downlevel.obj
 0001:000176d0       $unwind$_calloc_base       00000001800186d0     libucrt:calloc_base.obj
 0001:000176d0       $unwind$_malloc_base       00000001800186d0     libucrt:malloc_base.obj
 0001:000176d0       $unwind$_callnewh          00000001800186d0     libucrt:new_handler.obj
 0001:000176d0       $unwind$initialize_pointers 00000001800186d0     libucrt:initialization.obj
 0001:000176d0       $unwind$uninitialize_allocated_memory 00000001800186d0     libucrt:initialization.obj
 0001:000176d0       $unwind$__acrt_initialize_locks 00000001800186d0     libucrt:locks.obj
 0001:000176d0       $unwind$__acrt_uninitialize_locks 00000001800186d0     libucrt:locks.obj
 0001:000176d0       $unwind$__acrt_freeptd     00000001800186d0     libucrt:per_thread_data.obj
 0001:000176d0       $unwind$__acrt_getptd_head 00000001800186d0     libucrt:per_thread_data.obj
 0001:000176d0       $unwind$__acrt_get_process_end_policy 00000001800186d0     libucrt:win_policies.obj
 0001:000176d0       $unwind$__acrt_AppPolicyGetProcessTerminationMethodInternal 00000001800186d0     libucrt:winapi_thunks.obj
 0001:000176d0       $unwind$__acrt_FlsAlloc    00000001800186d0     libucrt:winapi_thunks.obj
 0001:000176d0       $unwind$__acrt_FlsFree     00000001800186d0     libucrt:winapi_thunks.obj
 0001:000176d0       $unwind$__acrt_FlsGetValue 00000001800186d0     libucrt:winapi_thunks.obj
 0001:000176d0       $unwind$__acrt_uninitialize_winapi_thunks 00000001800186d0     libucrt:winapi_thunks.obj
 0001:000176d0       $unwind$__acrt_update_locale_info 00000001800186d0     libucrt:locale_update.obj
 0001:000176d0       $unwind$__acrt_update_multibyte_info 00000001800186d0     libucrt:locale_update.obj
 0001:000176d0       $unwind$__acrt_allocate_buffer_for_argv 00000001800186d0     libucrt:argv_parsing.obj
 0001:000176d0       $unwind$?exit_or_terminate_process@@YAXI@Z 00000001800186d0     libucrt:exit.obj
 0001:000176d0       $unwind$?try_cor_exit_process@@YAXI@Z 00000001800186d0     libucrt:exit.obj
 0001:000176d0       $unwind$__acrt_uninitialize_stdio 00000001800186d0     libucrt:_file.obj
 0001:000176d0       $unwind$__acrt_stdio_free_buffer_nolock 00000001800186d0     libucrt:_freebuf.obj
 0001:000176d0       $unwind$_fflush_nolock     00000001800186d0     libucrt:fflush.obj
 0001:000176d0       $unwind$strcpy_s           00000001800186d0     libucrt:strcpy_s.obj
 0001:000176d0       $unwind$_clrfp             00000001800186d0     libucrt:fpctrl.obj
 0001:000176d0       $unwind$_set_statfp        00000001800186d0     libucrt:fpctrl.obj
 0001:000176d8       $unwind$OpenW              00000001800186d8     Brackets.obj
 0001:000176f0       $unwind$SetStartupInfoW    00000001800186f0     Brackets.obj
 0001:00017704       $unwind$??_G?$DialogBuilderBase@UFarDialogItem@@@@MEAAPEAXI@Z 0000000180018704     Brackets.obj
 0001:00017704       $unwind$??_GPluginDialogBuilder@@UEAAPEAXI@Z 0000000180018704     Brackets.obj
 0001:00017704       $unwind$?CreateRadioButtonBinding@PluginDialogBuilder@@MEAAPEAU?$DialogItemBinding@UFarDialogItem@@@@PEAH@Z 0000000180018704     Brackets.obj
 0001:00017704       $unwind$?SaveValue@PluginRadioButtonBinding@@UEAAXPEAUFarDialogItem@@H@Z 0000000180018704     Brackets.obj
 0001:00017704       $unwind$_RTC_Initialize    0000000180018704     LIBCMT:initsect.obj
 0001:00017704       $unwind$_RTC_Terminate     0000000180018704     LIBCMT:initsect.obj
 0001:00017704       $unwind$??_Gbad_alloc@std@@UEAAPEAXI@Z 0000000180018704     LIBCMT:throw_bad_alloc.obj
 0001:00017704       $unwind$??_Gbad_array_new_length@std@@UEAAPEAXI@Z 0000000180018704     LIBCMT:throw_bad_alloc.obj
 0001:00017704       $unwind$??_Gexception@std@@UEAAPEAXI@Z 0000000180018704     LIBCMT:throw_bad_alloc.obj
 0001:00017704       $unwind$__vcrt_FlsSetValue 0000000180018704     libvcruntime:winapi_downlevel.obj
 0001:00017704       $unwind$??$common_initialize_environment_nolock@D@@YAHXZ 0000000180018704     libucrt:environment_initialization.obj
 0001:00017704       $unwind$_realloc_base      0000000180018704     libucrt:realloc_base.obj
 0001:00017704       $unwind$?replace_current_thread_locale_nolock@@YAXQEAU__acrt_ptd@@QEAU__crt_locale_data@@@Z 0000000180018704     libucrt:per_thread_data.obj
 0001:00017704       $unwind$__acrt_execute_uninitializers 0000000180018704     libucrt:shared_initialization.obj
 0001:00017704       $unwind$__acrt_FlsSetValue 0000000180018704     libucrt:winapi_thunks.obj
 0001:00017704       $unwind$__acrt_LocaleNameToLCID 0000000180018704     libucrt:winapi_thunks.obj
 0001:00017704       $unwind$_updatetlocinfoEx_nolock 0000000180018704     libucrt:locale_refcounting.obj
 0001:00017704       $unwind$_close_nolock      0000000180018704     libucrt:close.obj
 0001:00017704       $unwind$__acrt_uninitialize_lowio 0000000180018704     libucrt:ioinit.obj
 0001:00017704       $unwind$__acrt_errno_map_os_error 0000000180018704     libucrt:errno.obj
 0001:00017704       $unwind$_initterm_e        0000000180018704     libucrt:initterm.obj
 0001:00017704       $unwind$_fclose_nolock     0000000180018704     libucrt:fclose.obj
 0001:00017704       $unwind$strncpy_s          0000000180018704     libucrt:strncpy_s.obj
 0001:00017710       $unwind$?AddDialogItem@?$DialogBuilderBase@UFarDialogItem@@@@IEAAPEAUFarDialogItem@@W4FARDIALOGITEMTYPES@@PEB_W@Z 0000000180018710     Brackets.obj
 0001:00017710       $unwind$?AddIntEditField@PluginDialogBuilder@@UEAAPEAUFarDialogItem@@PEAHH@Z 0000000180018710     Brackets.obj
 0001:00017710       $unwind$?AddUIntEditField@PluginDialogBuilder@@UEAAPEAUFarDialogItem@@PEAIH@Z 0000000180018710     Brackets.obj
 0001:00017728       $unwind$?UpdateBorderSize@?$DialogBuilderBase@UFarDialogItem@@@@IEAAXXZ 0000000180018728     Brackets.obj
 0001:00017738       $chain$1$?UpdateBorderSize@?$DialogBuilderBase@UFarDialogItem@@@@IEAAXXZ 0000000180018738     Brackets.obj
 0001:00017750       $chain$2$?UpdateBorderSize@?$DialogBuilderBase@UFarDialogItem@@@@IEAAXXZ 0000000180018750     Brackets.obj
 0001:00017764       $chain$3$?UpdateBorderSize@?$DialogBuilderBase@UFarDialogItem@@@@IEAAXXZ 0000000180018764     Brackets.obj
 0001:00017774       $chain$4$?UpdateBorderSize@?$DialogBuilderBase@UFarDialogItem@@@@IEAAXXZ 0000000180018774     Brackets.obj
 0001:00017784       $unwind$??1?$DialogBuilderBase@UFarDialogItem@@@@MEAA@XZ 0000000180018784     Brackets.obj
 0001:00017790       $chain$0$??1?$DialogBuilderBase@UFarDialogItem@@@@MEAA@XZ 0000000180018790     Brackets.obj
 0001:000177a4       $chain$1$??1?$DialogBuilderBase@UFarDialogItem@@@@MEAA@XZ 00000001800187a4     Brackets.obj
 0001:000177b4       $unwind$?AddButtons@?$DialogBuilderBase@UFarDialogItem@@@@QEAAXHPEBHHH@Z 00000001800187b4     Brackets.obj
 0001:000177c0       $chain$4$?AddButtons@?$DialogBuilderBase@UFarDialogItem@@@@QEAAXHPEBHHH@Z 00000001800187c0     Brackets.obj
 0001:000177e4       $chain$5$?AddButtons@?$DialogBuilderBase@UFarDialogItem@@@@QEAAXHPEBHHH@Z 00000001800187e4     Brackets.obj
 0001:000177f4       $unwind$?DoShowDialog@PluginDialogBuilder@@MEAA_JXZ 00000001800187f4     Brackets.obj
 0001:00017800       $unwind$?CreateCheckBoxBinding@PluginDialogBuilder@@MEAAPEAU?$DialogItemBinding@UFarDialogItem@@@@PEAHH@Z 0000000180018800     Brackets.obj
 0001:00017800       $unwind$_DllMainCRTStartup 0000000180018800     LIBCMT:dll_dllmain.obj
 0001:00017800       $unwind$__vcrt_getptd_noexit 0000000180018800     libvcruntime:per_thread_data.obj
 0001:00017800       $unwind$__vcrt_InitializeCriticalSectionEx 0000000180018800     libvcruntime:winapi_downlevel.obj
 0001:00017800       $unwind$__acrt_getptd      0000000180018800     libucrt:per_thread_data.obj
 0001:00017800       $unwind$__acrt_getptd_noexit 0000000180018800     libucrt:per_thread_data.obj
 0001:00017800       $unwind$__acrt_execute_initializers 0000000180018800     libucrt:shared_initialization.obj
 0001:00017800       $unwind$__acrt_InitializeCriticalSectionEx 0000000180018800     libucrt:winapi_thunks.obj
 0001:00017800       $unwind$?free_crt_array_internal@@YAXQEAPEBX_K@Z 0000000180018800     libucrt:inittime.obj
 0001:00017800       $unwind$??$common_lseek_nolock@_J@@YA_JH_JH@Z 0000000180018800     libucrt:lseek.obj
 0001:00017800       $unwind$__acrt_stdio_flush_nolock 0000000180018800     libucrt:fflush.obj
 0001:00017800       $unwind$??0_LocaleUpdate@@QEAA@QEAU__crt_locale_pointers@@@Z 0000000180018800     libucrt:output.obj
 0001:00017800       $unwind$_exception_enabled 0000000180018800     libucrt:libm_error.obj
 0001:00017810       $unwind$?Config@@YAHXZ     0000000180018810     Brackets.obj
 0001:00017830       $unwind$?ShowMenu@@YAHH@Z  0000000180018830     Brackets.obj
 0001:00017844       $unwind$?dllmain_crt_process_attach@@YAHQEAUHINSTANCE__@@QEAX@Z 0000000180018844     LIBCMT:dll_dllmain.obj
 0001:00017880       $unwind$?fin$0@?0??dllmain_crt_process_attach@@YAHQEAUHINSTANCE__@@QEAX@Z@4HA 0000000180018880     LIBCMT:dll_dllmain.obj
 0001:00017880       $unwind$?fin$0@?0??dllmain_crt_process_detach@@YAH_N@Z@4HA 0000000180018880     LIBCMT:dll_dllmain.obj
 0001:00017880       $unwind$?fin$1@?0??dllmain_crt_process_detach@@YAH_N@Z@4HA 0000000180018880     LIBCMT:dll_dllmain.obj
 0001:00017880       $unwind$_IsNonwritableInCurrentImage$filt$0 0000000180018880     LIBCMT:pesect.obj
 0001:00017880       $unwind$_query_new_handler$fin$0 0000000180018880     libucrt:new_handler.obj
 0001:00017880       $unwind$?fin$0@?0???$?RV<lambda_0ae27a3a962d80f24befdcbee591983d>@@AEAV<lambda_8d0ee55de4b1038c4002e0adecdf1839>@@V<lambda_dc504788e8f1664fe9b84e20bfb512f2>@@@?$__crt_seh_guarded_call@X@@QEAAX$$QEAV<lambda_0ae27a3a962d80f24befdcbee591983d>@@AEAV<lambda_8d0ee55de4b1038c4002e0adecdf1839>@@$$QEAV<lambda_dc504788e8f1664fe9b84e20bfb512f2>@@@Z@4HA 0000000180018880     libucrt:per_thread_data.obj
 0001:00017880       $unwind$?fin$0@?0???$?RV<lambda_2d41944a1d46af3157314b8a01080d33>@@AEAV<lambda_8f455de75cd7d7f24b4096f044d8b9e6>@@V<lambda_aa500f224e6afead328df44964fe2772>@@@?$__crt_seh_guarded_call@X@@QEAAX$$QEAV<lambda_2d41944a1d46af3157314b8a01080d33>@@AEAV<lambda_8f455de75cd7d7f24b4096f044d8b9e6>@@$$QEAV<lambda_aa500f224e6afead328df44964fe2772>@@@Z@4HA 0000000180018880     libucrt:per_thread_data.obj
 0001:00017880       $unwind$?fin$0@?0???$?RV<lambda_aa87e3671a710a21b5dc78c0bdf72e11>@@AEAV<lambda_92619d2358a28f41a33ba319515a20b9>@@V<lambda_6992ecaafeb10aed2b74cb1fae11a551>@@@?$__crt_seh_guarded_call@X@@QEAAX$$QEAV<lambda_aa87e3671a710a21b5dc78c0bdf72e11>@@AEAV<lambda_92619d2358a28f41a33ba319515a20b9>@@$$QEAV<lambda_6992ecaafeb10aed2b74cb1fae11a551>@@@Z@4HA 0000000180018880     libucrt:per_thread_data.obj
 0001:00017880       $unwind$?fin$0@?0???$?RV<lambda_f2e299630e499de9f9a165e60fcd3db5>@@AEAV<lambda_2ae9d31cdba2644fcbeaf08da7c24588>@@V<lambda_40d01ff24d0e7b3814fdbdcee8eab3c7>@@@?$__crt_seh_guarded_call@X@@QEAAX$$QEAV<lambda_f2e299630e499de9f9a165e60fcd3db5>@@AEAV<lambda_2ae9d31cdba2644fcbeaf08da7c24588>@@$$QEAV<lambda_40d01ff24d0e7b3814fdbdcee8eab3c7>@@@Z@4HA 0000000180018880     libucrt:per_thread_data.obj
 0001:00017880       $unwind$__acrt_update_thread_locale_data$fin$0 0000000180018880     libucrt:locale_refcounting.obj
 0001:00017880       $unwind$?fin$0@?0???$?RV<lambda_410d79af7f07d98d83a3f525b3859a53>@@AEAV<lambda_3e16ef9562a7dcce91392c22ab16ea36>@@V<lambda_38119f0e861e05405d8a144b9b982f0a>@@@?$__crt_seh_guarded_call@X@@QEAAX$$QEAV<lambda_410d79af7f07d98d83a3f525b3859a53>@@AEAV<lambda_3e16ef9562a7dcce91392c22ab16ea36>@@$$QEAV<lambda_38119f0e861e05405d8a144b9b982f0a>@@@Z@4HA 0000000180018880     libucrt:wsetlocale.obj
 0001:00017880       $unwind$?fin$0@?0???$?RV<lambda_751a882b2c74d4b022dec766aa51a29a>@@AEAV<lambda_628dfdc04ba53c8bfc02c9951375f3f5>@@V<lambda_f6c7be5f7998530c34de24c7437d6b54>@@@?$__crt_seh_guarded_call@H@@QEAAH$$QEAV<lambda_751a882b2c74d4b022dec766aa51a29a>@@AEAV<lambda_628dfdc04ba53c8bfc02c9951375f3f5>@@$$QEAV<lambda_f6c7be5f7998530c34de24c7437d6b54>@@@Z@4HA 0000000180018880     libucrt:close.obj
 0001:00017880       $unwind$?fin$0@?0???$?RV<lambda_a37b2b86f63e897a80ea819b0eb08c01>@@AEAV<lambda_38ce7e780aa69e748d6df282ebc68efe>@@V<lambda_99fb1378e971ab6e7edea83e3a7a83a2>@@@?$__crt_seh_guarded_call@H@@QEAAH$$QEAV<lambda_a37b2b86f63e897a80ea819b0eb08c01>@@AEAV<lambda_38ce7e780aa69e748d6df282ebc68efe>@@$$QEAV<lambda_99fb1378e971ab6e7edea83e3a7a83a2>@@@Z@4HA 0000000180018880     libucrt:commit.obj
 0001:00017880       $unwind$__acrt_initialize_lowio$fin$0 0000000180018880     libucrt:ioinit.obj
 0001:00017880       $unwind$__acrt_lowio_ensure_fh_exists$fin$0 0000000180018880     libucrt:osfinfo.obj
 0001:00017880       $unwind$_write$fin$0       0000000180018880     libucrt:write.obj
 0001:00017880       $unwind$?fin$0@?0???$?RV<lambda_efdfa57d1f175319df784efa44bb7b81>@@AEAV<lambda_5f0a4c1567f8adc6734073e5d1e1b35c>@@V<lambda_2e8a7d3640ea6ccb4c2413664c2db6fd>@@@?$__crt_seh_guarded_call@X@@QEAAX$$QEAV<lambda_efdfa57d1f175319df784efa44bb7b81>@@AEAV<lambda_5f0a4c1567f8adc6734073e5d1e1b35c>@@$$QEAV<lambda_2e8a7d3640ea6ccb4c2413664c2db6fd>@@@Z@4HA 0000000180018880     libucrt:mbctype.obj
 0001:00017880       $unwind$?fin$0@?0??update_thread_multibyte_data_internal@@YAPEAU__crt_multibyte_data@@QEAU__acrt_ptd@@QEAPEAU1@@Z@4HA 0000000180018880     libucrt:mbctype.obj
 0001:00017880       $unwind$?fin$0@?0???$?RV<lambda_450d765d439847d4c735a33c368b5fc0>@@AEAV<lambda_44731a7d0e6d81c3e6aa82d741081786>@@V<lambda_601a2a7da3b7a96e9554ac7215c4b07c>@@@?$__crt_seh_guarded_call@P6AXH@Z@@QEAAP6AXH@Z$$QEAV<lambda_450d765d439847d4c735a33c368b5fc0>@@AEAV<lambda_44731a7d0e6d81c3e6aa82d741081786>@@$$QEAV<lambda_601a2a7da3b7a96e9554ac7215c4b07c>@@@Z@4HA 0000000180018880     libucrt:signal.obj
 0001:00017880       $unwind$raise$fin$0        0000000180018880     libucrt:signal.obj
 0001:00017880       $unwind$?filt$0@?0???R<lambda_6e4b09c48022b2350581041d5f6b0c4c>@@QEBA@XZ@4HA 0000000180018880     libucrt:exit.obj
 0001:00017880       $unwind$?fin$0@?0???$?RV<lambda_d80eeec6fff315bfe5c115232f3240e3>@@AEAV<lambda_6e4b09c48022b2350581041d5f6b0c4c>@@V<lambda_2358e3775559c9db80273638284d5e45>@@@?$__crt_seh_guarded_call@X@@QEAAX$$QEAV<lambda_d80eeec6fff315bfe5c115232f3240e3>@@AEAV<lambda_6e4b09c48022b2350581041d5f6b0c4c>@@$$QEAV<lambda_2358e3775559c9db80273638284d5e45>@@@Z@4HA 0000000180018880     libucrt:exit.obj
 0001:00017880       $unwind$?fin$0@?0???$?RV<lambda_7777bce6b2f8c936911f934f8298dc43>@@AEAV<lambda_f03950bc5685219e0bcd2087efbe011e>@@V<lambda_3883c3dff614d5e0c5f61bb1ac94921c>@@@?$__crt_seh_guarded_call@H@@QEAAH$$QEAV<lambda_7777bce6b2f8c936911f934f8298dc43>@@AEAV<lambda_f03950bc5685219e0bcd2087efbe011e>@@$$QEAV<lambda_3883c3dff614d5e0c5f61bb1ac94921c>@@@Z@4HA 0000000180018880     libucrt:onexit.obj
 0001:00017880       $unwind$_fcloseall$fin$0   0000000180018880     libucrt:closeall.obj
 0001:00017880       $unwind$fclose$fin$0       0000000180018880     libucrt:fclose.obj
 0001:00017880       $unwind$?fin$0@?0???$?RV<lambda_842d9ff0dc9ef11c61343bbaebe7f885>@@AEAV<lambda_c5860995281e5c4ce005b3de8f5874ee>@@V<lambda_d90129c13df834fdcbf8d2b88dafcf2d>@@@?$__crt_seh_guarded_call@X@@QEAAX$$QEAV<lambda_842d9ff0dc9ef11c61343bbaebe7f885>@@AEAV<lambda_c5860995281e5c4ce005b3de8f5874ee>@@$$QEAV<lambda_d90129c13df834fdcbf8d2b88dafcf2d>@@@Z@4HA 0000000180018880     libucrt:fflush.obj
 0001:00017880       $unwind$?fin$0@?0???$?RV<lambda_886d6c58226a84441f68b9f2b8217b83>@@AEAV<lambda_ab61a845afdef5b7c387490eaf3616ee>@@V<lambda_f7f22ab5edc0698d5f6905b0d3f44752>@@@?$__crt_seh_guarded_call@X@@QEAAX$$QEAV<lambda_886d6c58226a84441f68b9f2b8217b83>@@AEAV<lambda_ab61a845afdef5b7c387490eaf3616ee>@@$$QEAV<lambda_f7f22ab5edc0698d5f6905b0d3f44752>@@@Z@4HA 0000000180018880     libucrt:fflush.obj
 0001:00017880       $unwind$_ctrlfp$filt$0     0000000180018880     libucrt:fpctrl.obj
 0001:00017888       $unwind$?dllmain_crt_process_detach@@YAH_N@Z 0000000180018888     LIBCMT:dll_dllmain.obj
 0001:000178dc       $unwind$?dllmain_dispatch@@YAHQEAUHINSTANCE__@@KQEAX@Z 00000001800188dc     LIBCMT:dll_dllmain.obj
 0001:00017904       $unwind$?filt$0@?0??dllmain_dispatch@@YAHQEAUHINSTANCE__@@KQEAX@Z@4HA 0000000180018904     LIBCMT:dll_dllmain.obj
 0001:0001790c       $unwind$?__scrt_throw_std_bad_alloc@@YAXXZ 000000018001890c     LIBCMT:throw_bad_alloc.obj
 0001:0001790c       $unwind$?__scrt_throw_std_bad_array_new_length@@YAXXZ 000000018001890c     LIBCMT:throw_bad_alloc.obj
 0001:0001790c       $unwind$_raise_exc         000000018001890c     libucrt:fpexcept.obj
 0001:00017914       $unwind$__security_init_cookie 0000000180018914     LIBCMT:gs_support.obj
 0001:00017920       $unwind$__scrt_is_nonwritable_in_current_image 0000000180018920     LIBCMT:utility.obj
 0001:00017940       $unwind$__scrt_is_nonwritable_in_current_image$filt$0 0000000180018940     LIBCMT:utility.obj
 0001:00017948       $unwind$__scrt_dllmain_exception_filter 0000000180018948     LIBCMT:utility.obj
 0001:00017948       $unwind$_recalloc_base     0000000180018948     libucrt:recalloc.obj
 0001:00017948       $unwind$__acrt_free_locale 0000000180018948     libucrt:locale_refcounting.obj
 0001:00017948       $unwind$__acrt_lowio_create_handle_array 0000000180018948     libucrt:osfinfo.obj
 0001:00017948       $unwind$?setSBCS@@YAXPEAU__crt_multibyte_data@@@Z 0000000180018948     libucrt:mbctype.obj
 0001:00017948       $unwind$_seh_filter_exe    0000000180018948     libucrt:exception_filter.obj
 0001:00017948       $unwind$_initterm          0000000180018948     libucrt:initterm.obj
 0001:0001795c       $unwind$__scrt_fastfail    000000018001895c     LIBCMT:utility_desktop.obj
 0001:0001796c       $unwind$__isa_available_init 000000018001896c     LIBCMT:cpu_disp.obj
 0001:00017980       $xdatasym                  0000000180018980     LIBCMT:guard_dispatch.obj
 0001:00017988       $xdatasym                  0000000180018988     libvcruntime:memset.obj
 0001:00017998       $unwind$__C_specific_handler 0000000180018998     libvcruntime:riscchandler.obj
 0001:000179b4       $unwind$__std_exception_copy 00000001800189b4     libvcruntime:std_exception.obj
 0001:000179b4       $unwind$_free_osfhnd       00000001800189b4     libucrt:osfinfo.obj
 0001:000179c8       $unwind$_CxxThrowException 00000001800189c8     libvcruntime:throw.obj
 0001:000179d8       $unwind$__DestructExceptionObject 00000001800189d8     libvcruntime:ehhelpers.obj
 0001:000179f8       $unwind$__DestructExceptionObject$filt$0 00000001800189f8     libvcruntime:ehhelpers.obj
 0001:00017a08       $xdatasym                  0000000180018a08     libvcruntime:notify.obj
 0001:00017a18       $xdatasym                  0000000180018a18     libvcruntime:memcpy.obj
 0001:00017a28       $unwind$?try_get_function@@YAPEAXW4function_id@?A0x81a78551@@QEBDQEBW4module_id@2@2@Z 0000000180018a28     libvcruntime:winapi_downlevel.obj
 0001:00017a28       $unwind$?try_get_function@@YAPEAXW4function_id@?A0x391cf84c@@QEBDQEBW4module_id@2@2@Z 0000000180018a28     libucrt:winapi_thunks.obj
 0001:00017a48       $xdatasym                  0000000180018a48     libvcruntime:handlers.obj
 0001:00017a68       $unwind$_query_new_handler 0000000180018a68     libucrt:new_handler.obj
 0001:00017a88       $unwind$?common_exit@@YAXHW4_crt_exit_cleanup_mode@@W4_crt_exit_return_mode@@@Z 0000000180018a88     libucrt:exit.obj
 0001:00017a94       $unwind$??R<lambda_6e4b09c48022b2350581041d5f6b0c4c>@@QEBA@XZ 0000000180018a94     libucrt:exit.obj
 0001:00017ab4       $unwind$??$?RV<lambda_d80eeec6fff315bfe5c115232f3240e3>@@AEAV<lambda_6e4b09c48022b2350581041d5f6b0c4c>@@V<lambda_2358e3775559c9db80273638284d5e45>@@@?$__crt_seh_guarded_call@X@@QEAAX$$QEAV<lambda_d80eeec6fff315bfe5c115232f3240e3>@@AEAV<lambda_6e4b09c48022b2350581041d5f6b0c4c>@@$$QEAV<lambda_2358e3775559c9db80273638284d5e45>@@@Z 0000000180018ab4     libucrt:exit.obj
 0001:00017ad8       $unwind$_configure_narrow_argv 0000000180018ad8     libucrt:argv_parsing.obj
 0001:00017aec       $unwind$??$parse_command_line@D@@YAXPEADPEAPEAD0PEA_K2@Z 0000000180018aec     libucrt:argv_parsing.obj
 0001:00017b08       $unwind$??$free_environment@D@@YAXQEAPEAD@Z 0000000180018b08     libucrt:environment_initialization.obj
 0001:00017b08       $unwind$??$free_environment@_W@@YAXQEAPEA_W@Z 0000000180018b08     libucrt:environment_initialization.obj
 0001:00017b14       $unwind$??$create_environment@D@@YAQEAPEADQEAD@Z 0000000180018b14     libucrt:environment_initialization.obj
 0001:00017b2c       $unwind$_execute_onexit_table 0000000180018b2c     libucrt:onexit.obj
 0001:00017b34       $unwind$__acrt_DownlevelLocaleNameToLCID 0000000180018b34     libucrt:lcidtoname_downlevel.obj
 0001:00017b34       $unwind$??R<lambda_f03950bc5685219e0bcd2087efbe011e>@@QEBAHXZ 0000000180018b34     libucrt:onexit.obj
 0001:00017b4c       $unwind$??$?RV<lambda_7777bce6b2f8c936911f934f8298dc43>@@AEAV<lambda_f03950bc5685219e0bcd2087efbe011e>@@V<lambda_3883c3dff614d5e0c5f61bb1ac94921c>@@@?$__crt_seh_guarded_call@H@@QEAAH$$QEAV<lambda_7777bce6b2f8c936911f934f8298dc43>@@AEAV<lambda_f03950bc5685219e0bcd2087efbe011e>@@$$QEAV<lambda_3883c3dff614d5e0c5f61bb1ac94921c>@@@Z 0000000180018b4c     libucrt:onexit.obj
 0001:00017b70       $unwind$terminate          0000000180018b70     libucrt:terminate.obj
 0001:00017b90       $xdatasym                  0000000180018b90     libucrt:strncmp.obj
 0001:00017b94       $unwind$_free_base         0000000180018b94     libucrt:free_base.obj
 0001:00017b94       $unwind$?destroy_fls@@YAXPEAX@Z 0000000180018b94     libucrt:per_thread_data.obj
 0001:00017b94       $unwind$__acrt_locale_free_numeric 0000000180018b94     libucrt:initnum.obj
 0001:00017b94       $unwind$__acrt_locale_free_lc_time_if_unreferenced 0000000180018b94     libucrt:locale_refcounting.obj
 0001:00017b9c       $unwind$?construct_ptd_array@@YAXQEAU__acrt_ptd@@@Z 0000000180018b9c     libucrt:per_thread_data.obj
 0001:00017ba4       $unwind$?destroy_ptd_array@@YAXQEAU__acrt_ptd@@@Z 0000000180018ba4     libucrt:per_thread_data.obj
 0001:00017bac       $unwind$??$?RV<lambda_0ae27a3a962d80f24befdcbee591983d>@@AEAV<lambda_8d0ee55de4b1038c4002e0adecdf1839>@@V<lambda_dc504788e8f1664fe9b84e20bfb512f2>@@@?$__crt_seh_guarded_call@X@@QEAAX$$QEAV<lambda_0ae27a3a962d80f24befdcbee591983d>@@AEAV<lambda_8d0ee55de4b1038c4002e0adecdf1839>@@$$QEAV<lambda_dc504788e8f1664fe9b84e20bfb512f2>@@@Z 0000000180018bac     libucrt:per_thread_data.obj
 0001:00017bd0       $unwind$??$?RV<lambda_aa87e3671a710a21b5dc78c0bdf72e11>@@AEAV<lambda_92619d2358a28f41a33ba319515a20b9>@@V<lambda_6992ecaafeb10aed2b74cb1fae11a551>@@@?$__crt_seh_guarded_call@X@@QEAAX$$QEAV<lambda_aa87e3671a710a21b5dc78c0bdf72e11>@@AEAV<lambda_92619d2358a28f41a33ba319515a20b9>@@$$QEAV<lambda_6992ecaafeb10aed2b74cb1fae11a551>@@@Z 0000000180018bd0     libucrt:per_thread_data.obj
 0001:00017bf4       $unwind$??$?RV<lambda_f2e299630e499de9f9a165e60fcd3db5>@@AEAV<lambda_2ae9d31cdba2644fcbeaf08da7c24588>@@V<lambda_40d01ff24d0e7b3814fdbdcee8eab3c7>@@@?$__crt_seh_guarded_call@X@@QEAAX$$QEAV<lambda_f2e299630e499de9f9a165e60fcd3db5>@@AEAV<lambda_2ae9d31cdba2644fcbeaf08da7c24588>@@$$QEAV<lambda_40d01ff24d0e7b3814fdbdcee8eab3c7>@@@Z 0000000180018bf4     libucrt:per_thread_data.obj
 0001:00017c18       $unwind$??$?RV<lambda_2d41944a1d46af3157314b8a01080d33>@@AEAV<lambda_8f455de75cd7d7f24b4096f044d8b9e6>@@V<lambda_aa500f224e6afead328df44964fe2772>@@@?$__crt_seh_guarded_call@X@@QEAAX$$QEAV<lambda_2d41944a1d46af3157314b8a01080d33>@@AEAV<lambda_8f455de75cd7d7f24b4096f044d8b9e6>@@$$QEAV<lambda_aa500f224e6afead328df44964fe2772>@@@Z 0000000180018c18     libucrt:per_thread_data.obj
 0001:00017c3c       $unwind$_invalid_parameter_noinfo 0000000180018c3c     libucrt:invalid_parameter.obj
 0001:00017c3c       $unwind$_log10_special     0000000180018c3c     libucrt:log_special.obj
 0001:00017c44       $unwind$__acrt_call_reportfault 0000000180018c44     libucrt:invalid_parameter.obj
 0001:00017c64       $unwind$_invalid_parameter 0000000180018c64     libucrt:invalid_parameter.obj
 0001:00017c78       $unwind$??$__acrt_mbs_to_wcs_cp@U__crt_win32_buffer_internal_dynamic_resizing@@@@YAHQEBDAEAV?$__crt_win32_buffer@_WU__crt_win32_buffer_internal_dynamic_resizing@@@@I@Z 0000000180018c78     libucrt:argv_wildcards.obj
 0001:00017c90       $unwind$__dcrt_get_narrow_environment_from_os 0000000180018c90     libucrt:get_environment_from_os.obj
 0001:00017c90       $unwind$??$__acrt_wcs_to_mbs_cp@U__crt_win32_buffer_internal_dynamic_resizing@@@@YAHQEB_WAEAV?$__crt_win32_buffer@DU__crt_win32_buffer_internal_dynamic_resizing@@@@I@Z 0000000180018c90     libucrt:argv_wildcards.obj
 0001:00017ca8       $unwind$??$common_expand_argv_wildcards@D@@YAHQEAPEADQEAPEAPEAD@Z 0000000180018ca8     libucrt:argv_wildcards.obj
 0001:00017cc0       $unwind$??$copy_and_add_argument_to_buffer@D@@YAHQEBD0_KAEAV?$argument_list@D@?A0x5f5c8891@@@Z 0000000180018cc0     libucrt:argv_wildcards.obj
 0001:00017cdc       $unwind$??$expand_argument_wildcards@D@@YAHQEAD0AEAV?$argument_list@D@?A0x5f5c8891@@@Z 0000000180018cdc     libucrt:argv_wildcards.obj
 0001:00017d00       $unwind$__acrt_GetModuleFileNameA 0000000180018d00     libucrt:getmodulefilenamea.obj
 0001:00017d1c       $unwind$__dcrt_write_console 0000000180018d1c     libucrt:initcon.obj
 0001:00017d1c       $unwind$??$__acrt_wcs_to_mbs_cp@U__crt_win32_buffer_no_resizing@@@@YAHQEB_WAEAV?$__crt_win32_buffer@DU__crt_win32_buffer_no_resizing@@@@I@Z 0000000180018d1c     libucrt:getmodulefilenamea.obj
 0001:00017d30       $unwind$_setmbcp_nolock    0000000180018d30     libucrt:mbctype.obj
 0001:00017d50       $unwind$__dcrt_lowio_ensure_console_output_initialized 0000000180018d50     libucrt:initcon.obj
 0001:00017d50       $unwind$_isleadbyte_l      0000000180018d50     libucrt:_wctype.obj
 0001:00017d50       $unwind$?getSystemCP@@YAHH@Z 0000000180018d50     libucrt:mbctype.obj
 0001:00017d58       $unwind$?update_thread_multibyte_data_internal@@YAPEAU__crt_multibyte_data@@QEAU__acrt_ptd@@QEAPEAU1@@Z 0000000180018d58     libucrt:mbctype.obj
 0001:00017d80       $unwind$?setmbcp_internal@@YAHH_NQEAU__acrt_ptd@@QEAPEAU__crt_multibyte_data@@@Z 0000000180018d80     libucrt:mbctype.obj
 0001:00017d90       $unwind$?setSBUpLow@@YAXPEAU__crt_multibyte_data@@@Z 0000000180018d90     libucrt:mbctype.obj
 0001:00017dac       $unwind$??$?RV<lambda_efdfa57d1f175319df784efa44bb7b81>@@AEAV<lambda_5f0a4c1567f8adc6734073e5d1e1b35c>@@V<lambda_2e8a7d3640ea6ccb4c2413664c2db6fd>@@@?$__crt_seh_guarded_call@X@@QEAAX$$QEAV<lambda_efdfa57d1f175319df784efa44bb7b81>@@AEAV<lambda_5f0a4c1567f8adc6734073e5d1e1b35c>@@$$QEAV<lambda_2e8a7d3640ea6ccb4c2413664c2db6fd>@@@Z 0000000180018dac     libucrt:mbctype.obj
 0001:00017dd0       $unwind$?x_ismbbtype_l@@YAHPEAU__crt_locale_pointers@@IHH@Z 0000000180018dd0     libucrt:ismbbyte.obj
 0001:00017de0       $unwind$__GSHandlerCheckCommon 0000000180018de0     LIBCMT:gshandler.obj
 0001:00017de0       $unwind$__acrt_WideCharToMultiByte 0000000180018de0     libucrt:widechartomultibyte.obj
 0001:00017de8       $unwind$__acrt_initialize_winapi_thunks 0000000180018de8     libucrt:winapi_thunks.obj
 0001:00017df0       $unwind$_mbtowc_l          0000000180018df0     libucrt:mbtowc.obj
 0001:00017df0       $unwind$__acrt_LCMapStringEx 0000000180018df0     libucrt:winapi_thunks.obj
 0001:00017e04       $unwind$__acrt_initialize_lowio 0000000180018e04     libucrt:ioinit.obj
 0001:00017e24       $unwind$?initialize_inherited_file_handles_nolock@@YAXXZ 0000000180018e24     libucrt:ioinit.obj
 0001:00017e40       $unwind$?initialize_stdio_handles_nolock@@YAXXZ 0000000180018e40     libucrt:ioinit.obj
 0001:00017e40       $unwind$__acrt_initialize_stdio 0000000180018e40     libucrt:_file.obj
 0001:00017e58       $unwind$__acrt_uninitialize_locale 0000000180018e58     libucrt:wsetlocale.obj
 0001:00017e58       $unwind$__acrt_get_sigabrt_handler 0000000180018e58     libucrt:signal.obj
 0001:00017e60       $unwind$raise              0000000180018e60     libucrt:signal.obj
 0001:00017e9c       $unwind$??$?RV<lambda_450d765d439847d4c735a33c368b5fc0>@@AEAV<lambda_44731a7d0e6d81c3e6aa82d741081786>@@V<lambda_601a2a7da3b7a96e9554ac7215c4b07c>@@@?$__crt_seh_guarded_call@P6AXH@Z@@QEAAP6AXH@Z$$QEAV<lambda_450d765d439847d4c735a33c368b5fc0>@@AEAV<lambda_44731a7d0e6d81c3e6aa82d741081786>@@$$QEAV<lambda_601a2a7da3b7a96e9554ac7215c4b07c>@@@Z 0000000180018e9c     libucrt:signal.obj
 0001:00017ec0       $unwind$?common_flush_all@@YAH_N@Z 0000000180018ec0     libucrt:fflush.obj
 0001:00017ec8       $unwind$??$?RV<lambda_842d9ff0dc9ef11c61343bbaebe7f885>@@AEAV<lambda_c5860995281e5c4ce005b3de8f5874ee>@@V<lambda_d90129c13df834fdcbf8d2b88dafcf2d>@@@?$__crt_seh_guarded_call@X@@QEAAX$$QEAV<lambda_842d9ff0dc9ef11c61343bbaebe7f885>@@AEAV<lambda_c5860995281e5c4ce005b3de8f5874ee>@@$$QEAV<lambda_d90129c13df834fdcbf8d2b88dafcf2d>@@@Z 0000000180018ec8     libucrt:fflush.obj
 0001:00017eec       $unwind$??$?RV<lambda_886d6c58226a84441f68b9f2b8217b83>@@AEAV<lambda_ab61a845afdef5b7c387490eaf3616ee>@@V<lambda_f7f22ab5edc0698d5f6905b0d3f44752>@@@?$__crt_seh_guarded_call@X@@QEAAX$$QEAV<lambda_886d6c58226a84441f68b9f2b8217b83>@@AEAV<lambda_ab61a845afdef5b7c387490eaf3616ee>@@$$QEAV<lambda_f7f22ab5edc0698d5f6905b0d3f44752>@@@Z 0000000180018eec     libucrt:fflush.obj
 0001:00017f14       $unwind$??$?RV<lambda_410d79af7f07d98d83a3f525b3859a53>@@AEAV<lambda_3e16ef9562a7dcce91392c22ab16ea36>@@V<lambda_38119f0e861e05405d8a144b9b982f0a>@@@?$__crt_seh_guarded_call@X@@QEAAX$$QEAV<lambda_410d79af7f07d98d83a3f525b3859a53>@@AEAV<lambda_3e16ef9562a7dcce91392c22ab16ea36>@@$$QEAV<lambda_38119f0e861e05405d8a144b9b982f0a>@@@Z 0000000180018f14     libucrt:wsetlocale.obj
 0001:00017f3c       $unwind$__acrt_update_thread_locale_data 0000000180018f3c     libucrt:locale_refcounting.obj
 0001:00017f60       $unwind$qsort              0000000180018f60     libucrt:qsort.obj
 0001:00017f78       $chain$4$qsort             0000000180018f78     libucrt:qsort.obj
 0001:00017f9c       $chain$5$qsort             0000000180018f9c     libucrt:qsort.obj
 0001:00017fac       $unwind$strpbrk            0000000180018fac     libucrt:strpbrk.obj
 0001:00017fbc       $unwind$fallbackMethod     0000000180018fbc     libucrt:strpbrk.obj
 0001:00017fcc       $unwind$_mbsdec_l          0000000180018fcc     libucrt:mbsdec.obj
 0001:00017fd8       $unwind$__acrt_GetStringTypeA 0000000180018fd8     libucrt:getstringtypea.obj
 0001:00018000       $unwind$__acrt_LCMapStringA 0000000180019000     libucrt:lcmapstringa.obj
 0001:00018010       $unwind$?__acrt_LCMapStringA_stat@@YAHPEAU__crt_locale_pointers@@PEB_WKPEBDHPEADHHH@Z 0000000180019010     libucrt:lcmapstringa.obj
 0001:00018038       $unwind$__acrt_lowio_destroy_handle_array 0000000180019038     libucrt:osfinfo.obj
 0001:00018048       $unwind$__acrt_lowio_ensure_fh_exists 0000000180019048     libucrt:osfinfo.obj
 0001:00018074       $unwind$_close             0000000180019074     libucrt:close.obj
 0001:00018074       $unwind$_commit            0000000180019074     libucrt:commit.obj
 0001:0001807c       $unwind$??$?RV<lambda_a37b2b86f63e897a80ea819b0eb08c01>@@AEAV<lambda_38ce7e780aa69e748d6df282ebc68efe>@@V<lambda_99fb1378e971ab6e7edea83e3a7a83a2>@@@?$__crt_seh_guarded_call@H@@QEAAH$$QEAV<lambda_a37b2b86f63e897a80ea819b0eb08c01>@@AEAV<lambda_38ce7e780aa69e748d6df282ebc68efe>@@$$QEAV<lambda_99fb1378e971ab6e7edea83e3a7a83a2>@@@Z 000000018001907c     libucrt:commit.obj
 0001:000180a0       $unwind$_write             00000001800190a0     libucrt:write.obj
 0001:000180d0       $unwind$_write_nolock      00000001800190d0     libucrt:write.obj
 0001:000180e8       $unwind$?write_double_translated_ansi_nolock@@YA?AUwrite_result@?A0x17268360@@HQEBDI@Z 00000001800190e8     libucrt:write.obj
 0001:0001810c       $unwind$?write_text_ansi_nolock@@YA?AUwrite_result@?A0x17268360@@HQEBDI@Z 000000018001910c     libucrt:write.obj
 0001:0001810c       $unwind$?write_text_utf16le_nolock@@YA?AUwrite_result@?A0x17268360@@HQEBDI@Z 000000018001910c     libucrt:write.obj
 0001:0001812c       $unwind$?write_text_utf8_nolock@@YA?AUwrite_result@?A0x17268360@@HQEBDI@Z 000000018001912c     libucrt:write.obj
 0001:00018150       $unwind$_fcloseall         0000000180019150     libucrt:closeall.obj
 0001:00018174       $unwind$?__mbrtowc_utf8@__crt_mbstring@@YA_KPEA_WPEBD_KPEAU_Mbstatet@@@Z 0000000180019174     libucrt:mbrtowc.obj
 0001:0001817c       $unwind$?__mbsrtowcs_utf8@__crt_mbstring@@YA_KPEA_WPEAPEBD_KPEAU_Mbstatet@@@Z 000000018001917c     libucrt:mbrtowc.obj
 0001:00018194       $unwind$__acrt_locale_free_monetary 0000000180019194     libucrt:initmon.obj
 0001:0001819c       $unwind$__acrt_locale_free_time 000000018001919c     libucrt:inittime.obj
 0001:000181ac       $unwind$_putwch_nolock     00000001800191ac     libucrt:putwch.obj
 0001:000181b4       $unwind$fclose             00000001800191b4     libucrt:fclose.obj
 0001:000181d8       $unwind$?__mbrtoc32_utf8@__crt_mbstring@@YA_KPEA_UPEBD_KPEAU_Mbstatet@@@Z 00000001800191d8     libucrt:mbrtoc32.obj
 0001:000181f8       $xdatasym                  00000001800191f8     libucrt:log10.obj
 0001:00018204       $unwind$??$?RV<lambda_751a882b2c74d4b022dec766aa51a29a>@@AEAV<lambda_628dfdc04ba53c8bfc02c9951375f3f5>@@V<lambda_f6c7be5f7998530c34de24c7437d6b54>@@@?$__crt_seh_guarded_call@H@@QEAAH$$QEAV<lambda_751a882b2c74d4b022dec766aa51a29a>@@AEAV<lambda_628dfdc04ba53c8bfc02c9951375f3f5>@@$$QEAV<lambda_f6c7be5f7998530c34de24c7437d6b54>@@@Z 0000000180019204     libucrt:close.obj
 0001:00018228       $unwind$_call_matherr      0000000180019228     libucrt:libm_error.obj
 0001:00018230       $unwind$_handle_error      0000000180019230     libucrt:libm_error.obj
 0001:00018250       $unwind$__acrt_initialize_fma3 0000000180019250     libucrt:fma3_available.obj
 0001:00018258       $unwind$_log_special_common 0000000180019258     libucrt:log_special.obj
 0001:00018268       $xdatasym                  0000000180019268     libucrt:fpsr.obj
 0001:00018270       $unwind$_raise_exc_ex      0000000180019270     libucrt:fpexcept.obj
 0001:00018284       $unwind$_ctrlfp            0000000180019284     libucrt:fpctrl.obj
 0001:000182ac       $unwind$_IsNonwritableInCurrentImage 00000001800192ac     LIBCMT:pesect.obj
 0001:000182d0       $xdatasym                  00000001800192d0     LIBCMT:amdsecgs.obj
 0001:000182d4       $unwind$__report_securityfailure 00000001800192d4     LIBCMT:gs_report.obj
 0001:000182dc       $unwind$__report_gsfailure 00000001800192dc     LIBCMT:gs_report.obj
 0001:000182e4       $unwind$capture_current_context 00000001800192e4     LIBCMT:gs_report.obj
 0001:000182f0       $unwind$capture_previous_context 00000001800192f0     LIBCMT:gs_report.obj
 0001:00018300       $xdatasym                  0000000180019300     libvcruntime:memcmp.obj
 0001:00018400       .edata                     0000000180019400     Brackets.exp
 0001:00018428       rgpv                       0000000180019428     Brackets.exp
 0001:0001843c       rgszName                   000000018001943c     Brackets.exp
 0001:00018450       rgwOrd                     0000000180019450     Brackets.exp
 0001:0001845a       szName                     000000018001945a     Brackets.exp
 0001:00018467       $N00001                    0000000180019467     Brackets.exp
 0001:00018472       $N00002                    0000000180019472     Brackets.exp
 0001:00018481       $N00003                    0000000180019481     Brackets.exp
 0001:00018490       $N00004                    0000000180019490     Brackets.exp
 0001:00018496       $N00005                    0000000180019496     Brackets.exp
 0002:00000000       ?HelpTopic@?1??ShowMenu@@YAHH@Z@4PAPEB_WA 000000018001a000     Brackets.obj
 0002:00000010       ?CmdName@?BB@??OpenW@@9@4PAU<unnamed-type-CmdName>@?BB@??1@YAPEAXPEBUOpenInfo@@@Z@A 000000018001a010     Brackets.obj
 0002:000000a0       ?__vcrt_flsindex@@3KA      000000018001a0a0     libvcruntime:per_thread_data.obj
 0002:000000c0       ?__acrt_flsindex@@3KA      000000018001a0c0     libucrt:per_thread_data.obj
 0002:000000c4       ?errno_no_memory@@3HA      000000018001a0c4     libucrt:errno.obj
 0002:000000c8       ?doserrno_no_memory@@3KA   000000018001a0c8     libucrt:errno.obj
 0002:00000300       _mbctypes                  000000018001a300     libucrt:mbctype.obj
 0002:00000410       _mbcasemaps                000000018001a410     libucrt:mbctype.obj
 0002:00000510       ?__rgctypeflag@@3PADA      000000018001a510     libucrt:mbctype.obj
 0002:00000520       ?__rgcode_page_info@@3PAUcode_page_info@@A 000000018001a520     libucrt:mbctype.obj
 0002:00000a30       ?__dcrt_lowio_console_output_handle@@3PEAXEA 000000018001aa30     libucrt:initcon.obj
 0002:00000a40       ?dazSupported@?1??_ctrlfp@@9@9 000000018001aa40     libucrt:fpctrl.obj
 0002:00000b00       ?Opt@@3UOptions@@A         000000018001ab00     Brackets.obj
 0002:00000bc0       ?Info@@3UPluginStartupInfo@@A 000000018001abc0     Brackets.obj
 0002:00000cd8       ?PluginMenuStrings@?1??GetPluginInfoW@@9@4PAPEB_WA 000000018001acd8     Brackets.obj
 0002:00000ce0       ?__proc_attached@@3HA      000000018001ace0     LIBCMT:dll_dllmain.obj
 0002:00000d20       ?is_initialized_as_dll@@3_NA 000000018001ad20     LIBCMT:utility.obj
 0002:00000d21       ?module_local_atexit_table_initialized@@3_NA 000000018001ad21     LIBCMT:utility.obj
 0002:00000d28       ?module_local_atexit_table@@3U_onexit_table_t@@A 000000018001ad28     LIBCMT:utility.obj
 0002:00000d40       ?module_local_at_quick_exit_table@@3U_onexit_table_t@@A 000000018001ad40     LIBCMT:utility.obj
 0002:00000da8       ?heap@@3V_HeapManager@@A   000000018001ada8     libvcruntime:undname.obj
 0002:00000dd0       ?__vcrt_startup_thread_ptd@@3U__vcrt_ptd@@A 000000018001add0     libvcruntime:per_thread_data.obj
 0002:00000e50       __vcrt_lock_table          000000018001ae50     libvcruntime:locks.obj
 0002:00000e78       __vcrt_locks_initialized   000000018001ae78     libvcruntime:locks.obj
 0002:00000e80       ?module_handles@@3PAPEAUHINSTANCE__@@A 000000018001ae80     libvcruntime:winapi_downlevel.obj
 0002:00000e98       ?function_pointers@@3PAPEAXA 000000018001ae98     libvcruntime:winapi_downlevel.obj
 0002:00000ec8       ?__acrt_new_handler@@3V?$dual_state_global@P6AH_K@Z@__crt_state_management@@A 000000018001aec8     libucrt:new_handler.obj
 0002:00000ed0       ?c_termination_complete@@3JA 000000018001aed0     libucrt:exit.obj
 0002:00000ed8       ?thread_local_exit_callback_func@@3P6AXPEAXK0@ZEA 000000018001aed8     libucrt:exit.obj
 0002:00000ef0       ?program_name@?1???$common_configure_argv@D@@YAHW4_crt_argv_mode@@@Z@4PADA 000000018001aef0     libucrt:argv_parsing.obj
 0002:00001050       ?__acrt_lock_table@@3PAU_RTL_CRITICAL_SECTION@@A 000000018001b050     libucrt:locks.obj
 0002:00001280       ?__acrt_locks_initialized@@3IA 000000018001b280     libucrt:locks.obj
 0002:00001288       ?__acrt_invalid_parameter_handler@@3V?$dual_state_global@P6AXPEB_W00I_K@Z@__crt_state_management@@A 000000018001b288     libucrt:invalid_parameter.obj
 0002:000012a8       ?fSystemSet@@3HA           000000018001b2a8     libucrt:mbctype.obj
 0002:000012ac       ?initialized@?1??__acrt_initialize_multibyte@@9@4_NA 000000018001b2ac     libucrt:mbctype.obj
 0002:000012e0       ?module_handles@@3PAPEAUHINSTANCE__@@A 000000018001b2e0     libucrt:winapi_thunks.obj
 0002:00001380       ?encoded_function_pointers@@3PAPEAXA 000000018001b380     libucrt:winapi_thunks.obj
 0002:000018a8       ?ctrlc_action@@3V?$dual_state_global@P6AXH@Z@__crt_state_management@@A 000000018001b8a8     libucrt:signal.obj
 0002:000018b0       ?ctrlbreak_action@@3V?$dual_state_global@P6AXH@Z@__crt_state_management@@A 000000018001b8b0     libucrt:signal.obj
 0002:000018b8       ?abort_action@@3V?$dual_state_global@P6AXH@Z@__crt_state_management@@A 000000018001b8b8     libucrt:signal.obj
 0002:000018c0       ?term_action@@3V?$dual_state_global@P6AXH@Z@__crt_state_management@@A 000000018001b8c0     libucrt:signal.obj
 0002:000018c8       ?user_matherr@@3V?$dual_state_global@P6AHPEAU_exception@@@Z@__crt_state_management@@A 000000018001b8c8     libucrt:matherr.obj
 0002:000018f8       ?internal_state@?1??_mbtowc_l@@9@4U_Mbstatet@@A 000000018001b8f8     libucrt:mbtowc.obj
 0002:00001904       ?__acrt_global_new_mode@@3V?$dual_state_global@J@__crt_state_management@@A 000000018001b904     libucrt:new_mode.obj
 0002:00001910       ?__acrt_app_type@@3W4_crt_app_type@@A 000000018001b910     libucrt:report_runtime_error.obj
 0002:00001918       ?internal_pst@?1??__mbrtoc32_utf8@__crt_mbstring@@YA_KPEA_UPEBD_KPEAU_Mbstatet@@@Z@4U3@A 000000018001b918     libucrt:mbrtoc32.obj
 0002:00001930       GS_ExceptionRecord         000000018001b930     LIBCMT:gs_report.obj
 0002:000019d0       GS_ContextRecord           000000018001b9d0     LIBCMT:gs_report.obj
 0003:0000000c       $pdata$ConfigureW          000000018001c00c     Brackets.obj
 0003:00000018       $pdata$GetGlobalInfoW      000000018001c018     Brackets.obj
 0003:00000024       $pdata$GetPluginInfoW      000000018001c024     Brackets.obj
 0003:00000030       $pdata$OpenW               000000018001c030     Brackets.obj
 0003:0000003c       $pdata$SetStartupInfoW     000000018001c03c     Brackets.obj
 0003:00000048       $pdata$??_G?$DialogItemBinding@UFarDialogItem@@@@UEAAPEAXI@Z 000000018001c048     Brackets.obj
 0003:00000054       $pdata$?SaveValue@PluginCheckBoxBinding@@UEAAXPEAUFarDialogItem@@H@Z 000000018001c054     Brackets.obj
 0003:00000060       $pdata$??_GPluginCheckBoxBinding@@UEAAPEAXI@Z 000000018001c060     Brackets.obj
 0003:00000060       $pdata$??_GPluginEditFieldBinding@@UEAAPEAXI@Z 000000018001c060     Brackets.obj
 0003:0000006c       $pdata$?SaveValue@PluginRadioButtonBinding@@UEAAXPEAUFarDialogItem@@H@Z 000000018001c06c     Brackets.obj
 0003:00000078       $pdata$??_GPluginRadioButtonBinding@@UEAAPEAXI@Z 000000018001c078     Brackets.obj
 0003:00000084       $pdata$?SaveValue@PluginEditFieldBinding@@UEAAXPEAUFarDialogItem@@H@Z 000000018001c084     Brackets.obj
 0003:00000090       $pdata$?SaveValue@PluginIntEditFieldBinding@@UEAAXPEAUFarDialogItem@@H@Z 000000018001c090     Brackets.obj
 0003:0000009c       $pdata$??_GPluginIntEditFieldBinding@@UEAAPEAXI@Z 000000018001c09c     Brackets.obj
 0003:0000009c       $pdata$??_GPluginUIntEditFieldBinding@@UEAAPEAXI@Z 000000018001c09c     Brackets.obj
 0003:000000a8       $pdata$?SaveValue@PluginUIntEditFieldBinding@@UEAAXPEAUFarDialogItem@@H@Z 000000018001c0a8     Brackets.obj
 0003:000000b4       $pdata$?AddDialogItem@?$DialogBuilderBase@UFarDialogItem@@@@IEAAPEAUFarDialogItem@@W4FARDIALOGITEMTYPES@@PEB_W@Z 000000018001c0b4     Brackets.obj
 0003:000000c0       $pdata$?UpdateBorderSize@?$DialogBuilderBase@UFarDialogItem@@@@IEAAXXZ 000000018001c0c0     Brackets.obj
 0003:000000cc       $pdata$1$?UpdateBorderSize@?$DialogBuilderBase@UFarDialogItem@@@@IEAAXXZ 000000018001c0cc     Brackets.obj
 0003:000000d8       $pdata$2$?UpdateBorderSize@?$DialogBuilderBase@UFarDialogItem@@@@IEAAXXZ 000000018001c0d8     Brackets.obj
 0003:000000e4       $pdata$3$?UpdateBorderSize@?$DialogBuilderBase@UFarDialogItem@@@@IEAAXXZ 000000018001c0e4     Brackets.obj
 0003:000000f0       $pdata$4$?UpdateBorderSize@?$DialogBuilderBase@UFarDialogItem@@@@IEAAXXZ 000000018001c0f0     Brackets.obj
 0003:000000fc       $pdata$??1?$DialogBuilderBase@UFarDialogItem@@@@MEAA@XZ 000000018001c0fc     Brackets.obj
 0003:00000108       $pdata$0$??1?$DialogBuilderBase@UFarDialogItem@@@@MEAA@XZ 000000018001c108     Brackets.obj
 0003:00000114       $pdata$1$??1?$DialogBuilderBase@UFarDialogItem@@@@MEAA@XZ 000000018001c114     Brackets.obj
 0003:00000120       $pdata$?AddButtons@?$DialogBuilderBase@UFarDialogItem@@@@QEAAXHPEBHHH@Z 000000018001c120     Brackets.obj
 0003:0000012c       $pdata$4$?AddButtons@?$DialogBuilderBase@UFarDialogItem@@@@QEAAXHPEBHHH@Z 000000018001c12c     Brackets.obj
 0003:00000138       $pdata$5$?AddButtons@?$DialogBuilderBase@UFarDialogItem@@@@QEAAXHPEBHHH@Z 000000018001c138     Brackets.obj
 0003:00000144       $pdata$??_G?$DialogBuilderBase@UFarDialogItem@@@@MEAAPEAXI@Z 000000018001c144     Brackets.obj
 0003:00000150       $pdata$?DoShowDialog@PluginDialogBuilder@@MEAA_JXZ 000000018001c150     Brackets.obj
 0003:0000015c       $pdata$?CreateCheckBoxBinding@PluginDialogBuilder@@MEAAPEAU?$DialogItemBinding@UFarDialogItem@@@@PEAHH@Z 000000018001c15c     Brackets.obj
 0003:00000168       $pdata$?CreateRadioButtonBinding@PluginDialogBuilder@@MEAAPEAU?$DialogItemBinding@UFarDialogItem@@@@PEAH@Z 000000018001c168     Brackets.obj
 0003:00000174       $pdata$?AddIntEditField@PluginDialogBuilder@@UEAAPEAUFarDialogItem@@PEAHH@Z 000000018001c174     Brackets.obj
 0003:00000180       $pdata$?AddUIntEditField@PluginDialogBuilder@@UEAAPEAUFarDialogItem@@PEAIH@Z 000000018001c180     Brackets.obj
 0003:0000018c       $pdata$??_GPluginDialogBuilder@@UEAAPEAXI@Z 000000018001c18c     Brackets.obj
 0003:00000198       $pdata$?Config@@YAHXZ      000000018001c198     Brackets.obj
 0003:000001a4       $pdata$?ShowMenu@@YAHH@Z   000000018001c1a4     Brackets.obj
 0003:000001b0       $pdata$??2@YAPEAX_K@Z      000000018001c1b0     LIBCMT:new_scalar.obj
 0003:000001bc       $pdata$?dllmain_crt_process_attach@@YAHQEAUHINSTANCE__@@QEAX@Z 000000018001c1bc     LIBCMT:dll_dllmain.obj
 0003:000001c8       $pdata$?fin$0@?0??dllmain_crt_process_attach@@YAHQEAUHINSTANCE__@@QEAX@Z@4HA 000000018001c1c8     LIBCMT:dll_dllmain.obj
 0003:000001d4       $pdata$?dllmain_crt_process_detach@@YAH_N@Z 000000018001c1d4     LIBCMT:dll_dllmain.obj
 0003:000001e0       $pdata$?fin$0@?0??dllmain_crt_process_detach@@YAH_N@Z@4HA 000000018001c1e0     LIBCMT:dll_dllmain.obj
 0003:000001ec       $pdata$?fin$1@?0??dllmain_crt_process_detach@@YAH_N@Z@4HA 000000018001c1ec     LIBCMT:dll_dllmain.obj
 0003:000001f8       $pdata$?dllmain_crt_dispatch@@YAHQEAUHINSTANCE__@@KQEAX@Z 000000018001c1f8     LIBCMT:dll_dllmain.obj
 0003:00000204       $pdata$?dllmain_dispatch@@YAHQEAUHINSTANCE__@@KQEAX@Z 000000018001c204     LIBCMT:dll_dllmain.obj
 0003:00000210       $pdata$?filt$0@?0??dllmain_dispatch@@YAHQEAUHINSTANCE__@@KQEAX@Z@4HA 000000018001c210     LIBCMT:dll_dllmain.obj
 0003:0000021c       $pdata$_DllMainCRTStartup  000000018001c21c     LIBCMT:dll_dllmain.obj
 0003:00000228       $pdata$??0exception@std@@QEAA@AEBV01@@Z 000000018001c228     LIBCMT:throw_bad_alloc.obj
 0003:00000234       $pdata$??_Gbad_alloc@std@@UEAAPEAXI@Z 000000018001c234     LIBCMT:throw_bad_alloc.obj
 0003:00000234       $pdata$??_Gbad_array_new_length@std@@UEAAPEAXI@Z 000000018001c234     LIBCMT:throw_bad_alloc.obj
 0003:00000234       $pdata$??_Gexception@std@@UEAAPEAXI@Z 000000018001c234     LIBCMT:throw_bad_alloc.obj
 0003:00000240       $pdata$??0bad_alloc@std@@QEAA@AEBV01@@Z 000000018001c240     LIBCMT:throw_bad_alloc.obj
 0003:0000024c       $pdata$??0bad_array_new_length@std@@QEAA@AEBV01@@Z 000000018001c24c     LIBCMT:throw_bad_alloc.obj
 0003:00000258       $pdata$?__scrt_throw_std_bad_alloc@@YAXXZ 000000018001c258     LIBCMT:throw_bad_alloc.obj
 0003:00000264       $pdata$?__scrt_throw_std_bad_array_new_length@@YAXXZ 000000018001c264     LIBCMT:throw_bad_alloc.obj
 0003:00000270       $pdata$__security_init_cookie 000000018001c270     LIBCMT:gs_support.obj
 0003:0000027c       $pdata$__scrt_initialize_default_local_stdio_options 000000018001c27c     LIBCMT:default_local_stdio_options.obj
 0003:00000288       $pdata$__scrt_is_nonwritable_in_current_image 000000018001c288     LIBCMT:utility.obj
 0003:00000294       $pdata$__scrt_is_nonwritable_in_current_image$filt$0 000000018001c294     LIBCMT:utility.obj
 0003:000002a0       $pdata$__scrt_acquire_startup_lock 000000018001c2a0     LIBCMT:utility.obj
 0003:000002ac       $pdata$__scrt_release_startup_lock 000000018001c2ac     LIBCMT:utility.obj
 0003:000002b8       $pdata$__scrt_initialize_crt 000000018001c2b8     LIBCMT:utility.obj
 0003:000002c4       $pdata$__scrt_uninitialize_crt 000000018001c2c4     LIBCMT:utility.obj
 0003:000002d0       $pdata$__scrt_initialize_onexit_tables 000000018001c2d0     LIBCMT:utility.obj
 0003:000002dc       $pdata$__scrt_dllmain_exception_filter 000000018001c2dc     LIBCMT:utility.obj
 0003:000002e8       $pdata$__scrt_dllmain_before_initialize_c 000000018001c2e8     LIBCMT:utility.obj
 0003:000002f4       $pdata$__scrt_dllmain_after_initialize_c 000000018001c2f4     LIBCMT:utility.obj
 0003:00000300       $pdata$__scrt_dllmain_uninitialize_c 000000018001c300     LIBCMT:utility.obj
 0003:0000030c       $pdata$__scrt_dllmain_uninitialize_critical 000000018001c30c     LIBCMT:utility.obj
 0003:00000318       $pdata$__scrt_dllmain_crt_thread_attach 000000018001c318     LIBCMT:utility.obj
 0003:00000324       $pdata$__scrt_dllmain_crt_thread_detach 000000018001c324     LIBCMT:utility.obj
 0003:00000330       $pdata$__scrt_fastfail     000000018001c330     LIBCMT:utility_desktop.obj
 0003:0000033c       $pdata$_RTC_Initialize     000000018001c33c     LIBCMT:initsect.obj
 0003:00000348       $pdata$_RTC_Terminate      000000018001c348     LIBCMT:initsect.obj
 0003:00000354       $pdata$??_Gtype_info@@UEAAPEAXI@Z 000000018001c354     LIBCMT:std_type_info_static.obj
 0003:00000360       $pdata$__isa_available_init 000000018001c360     LIBCMT:cpu_disp.obj
 0003:00000390       $pdata$__C_specific_handler 000000018001c390     libvcruntime:riscchandler.obj
 0003:0000039c       $pdata$__std_exception_copy 000000018001c39c     libvcruntime:std_exception.obj
 0003:000003a8       $pdata$__std_exception_destroy 000000018001c3a8     libvcruntime:std_exception.obj
 0003:000003b4       $pdata$_CxxThrowException  000000018001c3b4     libvcruntime:throw.obj
 0003:000003c0       $pdata$__std_type_info_destroy_list 000000018001c3c0     libvcruntime:std_type_info.obj
 0003:000003cc       $pdata$__vcrt_initialize   000000018001c3cc     libvcruntime:initialization.obj
 0003:000003d8       $pdata$__vcrt_uninitialize 000000018001c3d8     libvcruntime:initialization.obj
 0003:000003e4       $pdata$__vcrt_uninitialize_critical 000000018001c3e4     libvcruntime:initialization.obj
 0003:000003f0       $pdata$__vcrt_thread_attach 000000018001c3f0     libvcruntime:initialization.obj
 0003:000003fc       $pdata$__vcrt_thread_detach 000000018001c3fc     libvcruntime:initialization.obj
 0003:00000408       $pdata$__DestructExceptionObject 000000018001c408     libvcruntime:ehhelpers.obj
 0003:00000414       $pdata$__DestructExceptionObject$filt$0 000000018001c414     libvcruntime:ehhelpers.obj
 0003:00000444       $pdata$__vcrt_initialize_ptd 000000018001c444     libvcruntime:per_thread_data.obj
 0003:00000450       $pdata$__vcrt_uninitialize_ptd 000000018001c450     libvcruntime:per_thread_data.obj
 0003:0000045c       $pdata$__vcrt_getptd       000000018001c45c     libvcruntime:per_thread_data.obj
 0003:00000468       $pdata$__vcrt_getptd_noexit 000000018001c468     libvcruntime:per_thread_data.obj
 0003:00000474       $pdata$__vcrt_freeptd      000000018001c474     libvcruntime:per_thread_data.obj
 0003:00000480       $pdata$__vcrt_freefls      000000018001c480     libvcruntime:per_thread_data.obj
 0003:0000048c       $pdata$__vcrt_initialize_locks 000000018001c48c     libvcruntime:locks.obj
 0003:00000498       $pdata$__vcrt_uninitialize_locks 000000018001c498     libvcruntime:locks.obj
 0003:000004bc       $pdata$__vcrt_FlsAlloc     000000018001c4bc     libvcruntime:winapi_downlevel.obj
 0003:000004c8       $pdata$__vcrt_FlsFree      000000018001c4c8     libvcruntime:winapi_downlevel.obj
 0003:000004d4       $pdata$__vcrt_FlsGetValue  000000018001c4d4     libvcruntime:winapi_downlevel.obj
 0003:000004e0       $pdata$__vcrt_FlsSetValue  000000018001c4e0     libvcruntime:winapi_downlevel.obj
 0003:000004ec       $pdata$__vcrt_InitializeCriticalSectionEx 000000018001c4ec     libvcruntime:winapi_downlevel.obj
 0003:000004f8       $pdata$?try_get_function@@YAPEAXW4function_id@?A0x81a78551@@QEBDQEBW4module_id@2@2@Z 000000018001c4f8     libvcruntime:winapi_downlevel.obj
 0003:00000534       $pdata$_callnewh           000000018001c534     libucrt:new_handler.obj
 0003:00000540       $pdata$_query_new_handler  000000018001c540     libucrt:new_handler.obj
 0003:0000054c       $pdata$_query_new_handler$fin$0 000000018001c54c     libucrt:new_handler.obj
 0003:00000558       $pdata$_initterm           000000018001c558     libucrt:initterm.obj
 0003:00000564       $pdata$_initterm_e         000000018001c564     libucrt:initterm.obj
 0003:00000570       $pdata$_seh_filter_exe     000000018001c570     libucrt:exception_filter.obj
 0003:0000057c       $pdata$?try_cor_exit_process@@YAXI@Z 000000018001c57c     libucrt:exit.obj
 0003:00000588       $pdata$?exit_or_terminate_process@@YAXI@Z 000000018001c588     libucrt:exit.obj
 0003:00000594       $pdata$?common_exit@@YAXHW4_crt_exit_cleanup_mode@@W4_crt_exit_return_mode@@@Z 000000018001c594     libucrt:exit.obj
 0003:000005a0       $pdata$??R<lambda_6e4b09c48022b2350581041d5f6b0c4c>@@QEBA@XZ 000000018001c5a0     libucrt:exit.obj
 0003:000005ac       $pdata$?filt$0@?0???R<lambda_6e4b09c48022b2350581041d5f6b0c4c>@@QEBA@XZ@4HA 000000018001c5ac     libucrt:exit.obj
 0003:000005b8       $pdata$??$?RV<lambda_d80eeec6fff315bfe5c115232f3240e3>@@AEAV<lambda_6e4b09c48022b2350581041d5f6b0c4c>@@V<lambda_2358e3775559c9db80273638284d5e45>@@@?$__crt_seh_guarded_call@X@@QEAAX$$QEAV<lambda_d80eeec6fff315bfe5c115232f3240e3>@@AEAV<lambda_6e4b09c48022b2350581041d5f6b0c4c>@@$$QEAV<lambda_2358e3775559c9db80273638284d5e45>@@@Z 000000018001c5b8     libucrt:exit.obj
 0003:000005c4       $pdata$?fin$0@?0???$?RV<lambda_0ae27a3a962d80f24befdcbee591983d>@@AEAV<lambda_8d0ee55de4b1038c4002e0adecdf1839>@@V<lambda_dc504788e8f1664fe9b84e20bfb512f2>@@@?$__crt_seh_guarded_call@X@@QEAAX$$QEAV<lambda_0ae27a3a962d80f24befdcbee591983d>@@AEAV<lambda_8d0ee55de4b1038c4002e0adecdf1839>@@$$QEAV<lambda_dc504788e8f1664fe9b84e20bfb512f2>@@@Z@4HA 000000018001c5c4     libucrt:per_thread_data.obj
 0003:000005c4       $pdata$?fin$0@?0???$?RV<lambda_2d41944a1d46af3157314b8a01080d33>@@AEAV<lambda_8f455de75cd7d7f24b4096f044d8b9e6>@@V<lambda_aa500f224e6afead328df44964fe2772>@@@?$__crt_seh_guarded_call@X@@QEAAX$$QEAV<lambda_2d41944a1d46af3157314b8a01080d33>@@AEAV<lambda_8f455de75cd7d7f24b4096f044d8b9e6>@@$$QEAV<lambda_aa500f224e6afead328df44964fe2772>@@@Z@4HA 000000018001c5c4     libucrt:per_thread_data.obj
 0003:000005c4       $pdata$?fin$0@?0???$?RV<lambda_aa87e3671a710a21b5dc78c0bdf72e11>@@AEAV<lambda_92619d2358a28f41a33ba319515a20b9>@@V<lambda_6992ecaafeb10aed2b74cb1fae11a551>@@@?$__crt_seh_guarded_call@X@@QEAAX$$QEAV<lambda_aa87e3671a710a21b5dc78c0bdf72e11>@@AEAV<lambda_92619d2358a28f41a33ba319515a20b9>@@$$QEAV<lambda_6992ecaafeb10aed2b74cb1fae11a551>@@@Z@4HA 000000018001c5c4     libucrt:per_thread_data.obj
 0003:000005c4       $pdata$?fin$0@?0???$?RV<lambda_f2e299630e499de9f9a165e60fcd3db5>@@AEAV<lambda_2ae9d31cdba2644fcbeaf08da7c24588>@@V<lambda_40d01ff24d0e7b3814fdbdcee8eab3c7>@@@?$__crt_seh_guarded_call@X@@QEAAX$$QEAV<lambda_f2e299630e499de9f9a165e60fcd3db5>@@AEAV<lambda_2ae9d31cdba2644fcbeaf08da7c24588>@@$$QEAV<lambda_40d01ff24d0e7b3814fdbdcee8eab3c7>@@@Z@4HA 000000018001c5c4     libucrt:per_thread_data.obj
 0003:000005c4       $pdata$?fin$0@?0???$?RV<lambda_efdfa57d1f175319df784efa44bb7b81>@@AEAV<lambda_5f0a4c1567f8adc6734073e5d1e1b35c>@@V<lambda_2e8a7d3640ea6ccb4c2413664c2db6fd>@@@?$__crt_seh_guarded_call@X@@QEAAX$$QEAV<lambda_efdfa57d1f175319df784efa44bb7b81>@@AEAV<lambda_5f0a4c1567f8adc6734073e5d1e1b35c>@@$$QEAV<lambda_2e8a7d3640ea6ccb4c2413664c2db6fd>@@@Z@4HA 000000018001c5c4     libucrt:mbctype.obj
 0003:000005c4       $pdata$?fin$0@?0???$?RV<lambda_450d765d439847d4c735a33c368b5fc0>@@AEAV<lambda_44731a7d0e6d81c3e6aa82d741081786>@@V<lambda_601a2a7da3b7a96e9554ac7215c4b07c>@@@?$__crt_seh_guarded_call@P6AXH@Z@@QEAAP6AXH@Z$$QEAV<lambda_450d765d439847d4c735a33c368b5fc0>@@AEAV<lambda_44731a7d0e6d81c3e6aa82d741081786>@@$$QEAV<lambda_601a2a7da3b7a96e9554ac7215c4b07c>@@@Z@4HA 000000018001c5c4     libucrt:signal.obj
 0003:000005c4       $pdata$?fin$0@?0???$?RV<lambda_d80eeec6fff315bfe5c115232f3240e3>@@AEAV<lambda_6e4b09c48022b2350581041d5f6b0c4c>@@V<lambda_2358e3775559c9db80273638284d5e45>@@@?$__crt_seh_guarded_call@X@@QEAAX$$QEAV<lambda_d80eeec6fff315bfe5c115232f3240e3>@@AEAV<lambda_6e4b09c48022b2350581041d5f6b0c4c>@@$$QEAV<lambda_2358e3775559c9db80273638284d5e45>@@@Z@4HA 000000018001c5c4     libucrt:exit.obj
 0003:000005c4       $pdata$?fin$0@?0???$?RV<lambda_7777bce6b2f8c936911f934f8298dc43>@@AEAV<lambda_f03950bc5685219e0bcd2087efbe011e>@@V<lambda_3883c3dff614d5e0c5f61bb1ac94921c>@@@?$__crt_seh_guarded_call@H@@QEAAH$$QEAV<lambda_7777bce6b2f8c936911f934f8298dc43>@@AEAV<lambda_f03950bc5685219e0bcd2087efbe011e>@@$$QEAV<lambda_3883c3dff614d5e0c5f61bb1ac94921c>@@@Z@4HA 000000018001c5c4     libucrt:onexit.obj
 0003:000005d0       $pdata$_configure_narrow_argv 000000018001c5d0     libucrt:argv_parsing.obj
 0003:000005dc       $pdata$__acrt_allocate_buffer_for_argv 000000018001c5dc     libucrt:argv_parsing.obj
 0003:000005e8       $pdata$??$parse_command_line@D@@YAXPEADPEAPEAD0PEA_K2@Z 000000018001c5e8     libucrt:argv_parsing.obj
 0003:000005f4       $pdata$__dcrt_uninitialize_environments_nolock 000000018001c5f4     libucrt:environment_initialization.obj
 0003:00000600       $pdata$??$common_initialize_environment_nolock@D@@YAHXZ 000000018001c600     libucrt:environment_initialization.obj
 0003:0000060c       $pdata$??$uninitialize_environment_internal@D@@YAXAEAPEAPEAD@Z 000000018001c60c     libucrt:environment_initialization.obj
 0003:00000618       $pdata$??$uninitialize_environment_internal@_W@@YAXAEAPEAPEA_W@Z 000000018001c618     libucrt:environment_initialization.obj
 0003:00000624       $pdata$??$free_environment@D@@YAXQEAPEAD@Z 000000018001c624     libucrt:environment_initialization.obj
 0003:00000624       $pdata$??$free_environment@_W@@YAXQEAPEA_W@Z 000000018001c624     libucrt:environment_initialization.obj
 0003:00000630       $pdata$??$create_environment@D@@YAQEAPEADQEAD@Z 000000018001c630     libucrt:environment_initialization.obj
 0003:0000063c       $pdata$_execute_onexit_table 000000018001c63c     libucrt:onexit.obj
 0003:00000648       $pdata$??R<lambda_f03950bc5685219e0bcd2087efbe011e>@@QEBAHXZ 000000018001c648     libucrt:onexit.obj
 0003:00000654       $pdata$??$?RV<lambda_7777bce6b2f8c936911f934f8298dc43>@@AEAV<lambda_f03950bc5685219e0bcd2087efbe011e>@@V<lambda_3883c3dff614d5e0c5f61bb1ac94921c>@@@?$__crt_seh_guarded_call@H@@QEAAH$$QEAV<lambda_7777bce6b2f8c936911f934f8298dc43>@@AEAV<lambda_f03950bc5685219e0bcd2087efbe011e>@@$$QEAV<lambda_3883c3dff614d5e0c5f61bb1ac94921c>@@@Z 000000018001c654     libucrt:onexit.obj
 0003:00000660       $pdata$__acrt_uninitialize 000000018001c660     libucrt:initialization.obj
 0003:0000066c       $pdata$__acrt_uninitialize_critical 000000018001c66c     libucrt:initialization.obj
 0003:00000678       $pdata$__acrt_thread_attach 000000018001c678     libucrt:initialization.obj
 0003:00000684       $pdata$__acrt_thread_detach 000000018001c684     libucrt:initialization.obj
 0003:00000690       $pdata$initialize_c        000000018001c690     libucrt:initialization.obj
 0003:0000069c       $pdata$uninitialize_environment 000000018001c69c     libucrt:initialization.obj
 0003:000006a8       $pdata$initialize_pointers 000000018001c6a8     libucrt:initialization.obj
 0003:000006b4       $pdata$uninitialize_allocated_memory 000000018001c6b4     libucrt:initialization.obj
 0003:000006c0       $pdata$uninitialize_allocated_io_buffers 000000018001c6c0     libucrt:initialization.obj
 0003:000006cc       $pdata$terminate           000000018001c6cc     libucrt:terminate.obj
 0003:000006d8       $pdata$strcpy_s            000000018001c6d8     libucrt:strcpy_s.obj
 0003:000006e4       $pdata$abort               000000018001c6e4     libucrt:abort.obj
 0003:000006f0       $pdata$??0_LocaleUpdate@@QEAA@QEAU__crt_locale_pointers@@@Z 000000018001c6f0     libucrt:output.obj
 0003:00000708       $pdata$__acrt_initialize_locks 000000018001c708     libucrt:locks.obj
 0003:00000714       $pdata$__acrt_uninitialize_locks 000000018001c714     libucrt:locks.obj
 0003:00000720       $pdata$_malloc_base        000000018001c720     libucrt:malloc_base.obj
 0003:0000072c       $pdata$_free_base          000000018001c72c     libucrt:free_base.obj
 0003:00000738       $pdata$__acrt_initialize_ptd 000000018001c738     libucrt:per_thread_data.obj
 0003:00000744       $pdata$__acrt_uninitialize_ptd 000000018001c744     libucrt:per_thread_data.obj
 0003:00000750       $pdata$__acrt_getptd       000000018001c750     libucrt:per_thread_data.obj
 0003:0000075c       $pdata$__acrt_getptd_head  000000018001c75c     libucrt:per_thread_data.obj
 0003:00000768       $pdata$__acrt_getptd_noexit 000000018001c768     libucrt:per_thread_data.obj
 0003:00000774       $pdata$__acrt_freeptd      000000018001c774     libucrt:per_thread_data.obj
 0003:00000780       $pdata$?destroy_fls@@YAXPEAX@Z 000000018001c780     libucrt:per_thread_data.obj
 0003:0000078c       $pdata$?replace_current_thread_locale_nolock@@YAXQEAU__acrt_ptd@@QEAU__crt_locale_data@@@Z 000000018001c78c     libucrt:per_thread_data.obj
 0003:00000798       $pdata$?construct_ptd_array@@YAXQEAU__acrt_ptd@@@Z 000000018001c798     libucrt:per_thread_data.obj
 0003:000007a4       $pdata$?destroy_ptd_array@@YAXQEAU__acrt_ptd@@@Z 000000018001c7a4     libucrt:per_thread_data.obj
 0003:000007b0       $pdata$??$?RV<lambda_0ae27a3a962d80f24befdcbee591983d>@@AEAV<lambda_8d0ee55de4b1038c4002e0adecdf1839>@@V<lambda_dc504788e8f1664fe9b84e20bfb512f2>@@@?$__crt_seh_guarded_call@X@@QEAAX$$QEAV<lambda_0ae27a3a962d80f24befdcbee591983d>@@AEAV<lambda_8d0ee55de4b1038c4002e0adecdf1839>@@$$QEAV<lambda_dc504788e8f1664fe9b84e20bfb512f2>@@@Z 000000018001c7b0     libucrt:per_thread_data.obj
 0003:000007bc       $pdata$??$?RV<lambda_aa87e3671a710a21b5dc78c0bdf72e11>@@AEAV<lambda_92619d2358a28f41a33ba319515a20b9>@@V<lambda_6992ecaafeb10aed2b74cb1fae11a551>@@@?$__crt_seh_guarded_call@X@@QEAAX$$QEAV<lambda_aa87e3671a710a21b5dc78c0bdf72e11>@@AEAV<lambda_92619d2358a28f41a33ba319515a20b9>@@$$QEAV<lambda_6992ecaafeb10aed2b74cb1fae11a551>@@@Z 000000018001c7bc     libucrt:per_thread_data.obj
 0003:000007c8       $pdata$??$?RV<lambda_f2e299630e499de9f9a165e60fcd3db5>@@AEAV<lambda_2ae9d31cdba2644fcbeaf08da7c24588>@@V<lambda_40d01ff24d0e7b3814fdbdcee8eab3c7>@@@?$__crt_seh_guarded_call@X@@QEAAX$$QEAV<lambda_f2e299630e499de9f9a165e60fcd3db5>@@AEAV<lambda_2ae9d31cdba2644fcbeaf08da7c24588>@@$$QEAV<lambda_40d01ff24d0e7b3814fdbdcee8eab3c7>@@@Z 000000018001c7c8     libucrt:per_thread_data.obj
 0003:000007d4       $pdata$??$?RV<lambda_2d41944a1d46af3157314b8a01080d33>@@AEAV<lambda_8f455de75cd7d7f24b4096f044d8b9e6>@@V<lambda_aa500f224e6afead328df44964fe2772>@@@?$__crt_seh_guarded_call@X@@QEAAX$$QEAV<lambda_2d41944a1d46af3157314b8a01080d33>@@AEAV<lambda_8f455de75cd7d7f24b4096f044d8b9e6>@@$$QEAV<lambda_aa500f224e6afead328df44964fe2772>@@@Z 000000018001c7d4     libucrt:per_thread_data.obj
 0003:000007e0       $pdata$__acrt_get_process_end_policy 000000018001c7e0     libucrt:win_policies.obj
 0003:000007ec       $pdata$_invalid_parameter_noinfo 000000018001c7ec     libucrt:invalid_parameter.obj
 0003:000007f8       $pdata$_invoke_watson      000000018001c7f8     libucrt:invalid_parameter.obj
 0003:00000804       $pdata$__acrt_call_reportfault 000000018001c804     libucrt:invalid_parameter.obj
 0003:00000810       $pdata$_invalid_parameter  000000018001c810     libucrt:invalid_parameter.obj
 0003:0000081c       $pdata$_errno              000000018001c81c     libucrt:errno.obj
 0003:00000828       $pdata$__doserrno          000000018001c828     libucrt:errno.obj
 0003:00000834       $pdata$__acrt_errno_map_os_error 000000018001c834     libucrt:errno.obj
 0003:00000840       $pdata$_calloc_base        000000018001c840     libucrt:calloc_base.obj
 0003:0000084c       $pdata$??$__acrt_mbs_to_wcs_cp@U__crt_win32_buffer_internal_dynamic_resizing@@@@YAHQEBDAEAV?$__crt_win32_buffer@_WU__crt_win32_buffer_internal_dynamic_resizing@@@@I@Z 000000018001c84c     libucrt:argv_wildcards.obj
 0003:00000858       $pdata$??$__acrt_wcs_to_mbs_cp@U__crt_win32_buffer_internal_dynamic_resizing@@@@YAHQEB_WAEAV?$__crt_win32_buffer@DU__crt_win32_buffer_internal_dynamic_resizing@@@@I@Z 000000018001c858     libucrt:argv_wildcards.obj
 0003:00000864       $pdata$??$common_expand_argv_wildcards@D@@YAHQEAPEADQEAPEAPEAD@Z 000000018001c864     libucrt:argv_wildcards.obj
 0003:00000870       $pdata$??$copy_and_add_argument_to_buffer@D@@YAHQEBD0_KAEAV?$argument_list@D@?A0x5f5c8891@@@Z 000000018001c870     libucrt:argv_wildcards.obj
 0003:0000087c       $pdata$??$expand_argument_wildcards@D@@YAHQEAD0AEAV?$argument_list@D@?A0x5f5c8891@@@Z 000000018001c87c     libucrt:argv_wildcards.obj
 0003:00000888       $pdata$__acrt_GetModuleFileNameA 000000018001c888     libucrt:getmodulefilenamea.obj
 0003:00000894       $pdata$??$__acrt_wcs_to_mbs_cp@U__crt_win32_buffer_no_resizing@@@@YAHQEB_WAEAV?$__crt_win32_buffer@DU__crt_win32_buffer_no_resizing@@@@I@Z 000000018001c894     libucrt:getmodulefilenamea.obj
 0003:000008a0       $pdata$__acrt_update_thread_multibyte_data 000000018001c8a0     libucrt:mbctype.obj
 0003:000008ac       $pdata$__acrt_initialize_multibyte 000000018001c8ac     libucrt:mbctype.obj
 0003:000008b8       $pdata$_setmbcp_nolock     000000018001c8b8     libucrt:mbctype.obj
 0003:000008c4       $pdata$?getSystemCP@@YAHH@Z 000000018001c8c4     libucrt:mbctype.obj
 0003:000008d0       $pdata$?setSBCS@@YAXPEAU__crt_multibyte_data@@@Z 000000018001c8d0     libucrt:mbctype.obj
 0003:000008dc       $pdata$?update_thread_multibyte_data_internal@@YAPEAU__crt_multibyte_data@@QEAU__acrt_ptd@@QEAPEAU1@@Z 000000018001c8dc     libucrt:mbctype.obj
 0003:000008e8       $pdata$?fin$0@?0??update_thread_multibyte_data_internal@@YAPEAU__crt_multibyte_data@@QEAU__acrt_ptd@@QEAPEAU1@@Z@4HA 000000018001c8e8     libucrt:mbctype.obj
 0003:000008f4       $pdata$?setmbcp_internal@@YAHH_NQEAU__acrt_ptd@@QEAPEAU__crt_multibyte_data@@@Z 000000018001c8f4     libucrt:mbctype.obj
 0003:00000900       $pdata$?setSBUpLow@@YAXPEAU__crt_multibyte_data@@@Z 000000018001c900     libucrt:mbctype.obj
 0003:0000090c       $pdata$??$?RV<lambda_efdfa57d1f175319df784efa44bb7b81>@@AEAV<lambda_5f0a4c1567f8adc6734073e5d1e1b35c>@@V<lambda_2e8a7d3640ea6ccb4c2413664c2db6fd>@@@?$__crt_seh_guarded_call@X@@QEAAX$$QEAV<lambda_efdfa57d1f175319df784efa44bb7b81>@@AEAV<lambda_5f0a4c1567f8adc6734073e5d1e1b35c>@@$$QEAV<lambda_2e8a7d3640ea6ccb4c2413664c2db6fd>@@@Z 000000018001c90c     libucrt:mbctype.obj
 0003:00000918       $pdata$?x_ismbbtype_l@@YAHPEAU__crt_locale_pointers@@IHH@Z 000000018001c918     libucrt:ismbbyte.obj
 0003:00000924       $pdata$__acrt_initialize_command_line 000000018001c924     libucrt:argv_data.obj
 0003:00000930       $pdata$__acrt_WideCharToMultiByte 000000018001c930     libucrt:widechartomultibyte.obj
 0003:0000093c       $pdata$__dcrt_get_narrow_environment_from_os 000000018001c93c     libucrt:get_environment_from_os.obj
 0003:00000948       $pdata$_recalloc_base      000000018001c948     libucrt:recalloc.obj
 0003:00000954       $pdata$__acrt_initialize_winapi_thunks 000000018001c954     libucrt:winapi_thunks.obj
 0003:00000960       $pdata$__acrt_uninitialize_winapi_thunks 000000018001c960     libucrt:winapi_thunks.obj
 0003:0000096c       $pdata$__acrt_AreFileApisANSI 000000018001c96c     libucrt:winapi_thunks.obj
 0003:00000978       $pdata$__acrt_FlsAlloc     000000018001c978     libucrt:winapi_thunks.obj
 0003:00000984       $pdata$__acrt_FlsFree      000000018001c984     libucrt:winapi_thunks.obj
 0003:00000990       $pdata$__acrt_FlsGetValue  000000018001c990     libucrt:winapi_thunks.obj
 0003:0000099c       $pdata$__acrt_FlsSetValue  000000018001c99c     libucrt:winapi_thunks.obj
 0003:000009a8       $pdata$__acrt_InitializeCriticalSectionEx 000000018001c9a8     libucrt:winapi_thunks.obj
 0003:000009b4       $pdata$__acrt_LCMapStringEx 000000018001c9b4     libucrt:winapi_thunks.obj
 0003:000009c0       $pdata$__acrt_LocaleNameToLCID 000000018001c9c0     libucrt:winapi_thunks.obj
 0003:000009cc       $pdata$__acrt_AppPolicyGetProcessTerminationMethodInternal 000000018001c9cc     libucrt:winapi_thunks.obj
 0003:000009d8       $pdata$?try_get_function@@YAPEAXW4function_id@?A0x391cf84c@@QEBDQEBW4module_id@2@2@Z 000000018001c9d8     libucrt:winapi_thunks.obj
 0003:000009e4       $pdata$__acrt_initialize_heap 000000018001c9e4     libucrt:heap_handle.obj
 0003:000009f0       $pdata$__acrt_initialize_lowio 000000018001c9f0     libucrt:ioinit.obj
 0003:000009fc       $pdata$__acrt_initialize_lowio$fin$0 000000018001c9fc     libucrt:ioinit.obj
 0003:000009fc       $pdata$__acrt_lowio_ensure_fh_exists$fin$0 000000018001c9fc     libucrt:osfinfo.obj
 0003:00000a08       $pdata$__acrt_uninitialize_lowio 000000018001ca08     libucrt:ioinit.obj
 0003:00000a14       $pdata$?initialize_inherited_file_handles_nolock@@YAXXZ 000000018001ca14     libucrt:ioinit.obj
 0003:00000a20       $pdata$?initialize_stdio_handles_nolock@@YAXXZ 000000018001ca20     libucrt:ioinit.obj
 0003:00000a2c       $pdata$__acrt_execute_initializers 000000018001ca2c     libucrt:shared_initialization.obj
 0003:00000a38       $pdata$__acrt_execute_uninitializers 000000018001ca38     libucrt:shared_initialization.obj
 0003:00000a44       $pdata$__acrt_get_sigabrt_handler 000000018001ca44     libucrt:signal.obj
 0003:00000a50       $pdata$raise               000000018001ca50     libucrt:signal.obj
 0003:00000a5c       $pdata$raise$fin$0         000000018001ca5c     libucrt:signal.obj
 0003:00000a68       $pdata$??$?RV<lambda_450d765d439847d4c735a33c368b5fc0>@@AEAV<lambda_44731a7d0e6d81c3e6aa82d741081786>@@V<lambda_601a2a7da3b7a96e9554ac7215c4b07c>@@@?$__crt_seh_guarded_call@P6AXH@Z@@QEAAP6AXH@Z$$QEAV<lambda_450d765d439847d4c735a33c368b5fc0>@@AEAV<lambda_44731a7d0e6d81c3e6aa82d741081786>@@$$QEAV<lambda_601a2a7da3b7a96e9554ac7215c4b07c>@@@Z 000000018001ca68     libucrt:signal.obj
 0003:00000a74       $pdata$_fflush_nolock      000000018001ca74     libucrt:fflush.obj
 0003:00000a80       $pdata$__acrt_stdio_flush_nolock 000000018001ca80     libucrt:fflush.obj
 0003:00000a8c       $pdata$?common_flush_all@@YAH_N@Z 000000018001ca8c     libucrt:fflush.obj
 0003:00000a98       $pdata$??$?RV<lambda_842d9ff0dc9ef11c61343bbaebe7f885>@@AEAV<lambda_c5860995281e5c4ce005b3de8f5874ee>@@V<lambda_d90129c13df834fdcbf8d2b88dafcf2d>@@@?$__crt_seh_guarded_call@X@@QEAAX$$QEAV<lambda_842d9ff0dc9ef11c61343bbaebe7f885>@@AEAV<lambda_c5860995281e5c4ce005b3de8f5874ee>@@$$QEAV<lambda_d90129c13df834fdcbf8d2b88dafcf2d>@@@Z 000000018001ca98     libucrt:fflush.obj
 0003:00000aa4       $pdata$?fin$0@?0???$?RV<lambda_842d9ff0dc9ef11c61343bbaebe7f885>@@AEAV<lambda_c5860995281e5c4ce005b3de8f5874ee>@@V<lambda_d90129c13df834fdcbf8d2b88dafcf2d>@@@?$__crt_seh_guarded_call@X@@QEAAX$$QEAV<lambda_842d9ff0dc9ef11c61343bbaebe7f885>@@AEAV<lambda_c5860995281e5c4ce005b3de8f5874ee>@@$$QEAV<lambda_d90129c13df834fdcbf8d2b88dafcf2d>@@@Z@4HA 000000018001caa4     libucrt:fflush.obj
 0003:00000ab0       $pdata$??$?RV<lambda_886d6c58226a84441f68b9f2b8217b83>@@AEAV<lambda_ab61a845afdef5b7c387490eaf3616ee>@@V<lambda_f7f22ab5edc0698d5f6905b0d3f44752>@@@?$__crt_seh_guarded_call@X@@QEAAX$$QEAV<lambda_886d6c58226a84441f68b9f2b8217b83>@@AEAV<lambda_ab61a845afdef5b7c387490eaf3616ee>@@$$QEAV<lambda_f7f22ab5edc0698d5f6905b0d3f44752>@@@Z 000000018001cab0     libucrt:fflush.obj
 0003:00000abc       $pdata$?fin$0@?0???$?RV<lambda_886d6c58226a84441f68b9f2b8217b83>@@AEAV<lambda_ab61a845afdef5b7c387490eaf3616ee>@@V<lambda_f7f22ab5edc0698d5f6905b0d3f44752>@@@?$__crt_seh_guarded_call@X@@QEAAX$$QEAV<lambda_886d6c58226a84441f68b9f2b8217b83>@@AEAV<lambda_ab61a845afdef5b7c387490eaf3616ee>@@$$QEAV<lambda_f7f22ab5edc0698d5f6905b0d3f44752>@@@Z@4HA 000000018001cabc     libucrt:fflush.obj
 0003:00000ac8       $pdata$__acrt_initialize_stdio 000000018001cac8     libucrt:_file.obj
 0003:00000ad4       $pdata$__acrt_uninitialize_stdio 000000018001cad4     libucrt:_file.obj
 0003:00000ae0       $pdata$_mbtowc_l           000000018001cae0     libucrt:mbtowc.obj
 0003:00000aec       $pdata$__acrt_update_locale_info 000000018001caec     libucrt:locale_update.obj
 0003:00000af8       $pdata$__acrt_update_multibyte_info 000000018001caf8     libucrt:locale_update.obj
 0003:00000b04       $pdata$_fileno             000000018001cb04     libucrt:fileno.obj
 0003:00000b10       $pdata$__acrt_uninitialize_locale 000000018001cb10     libucrt:wsetlocale.obj
 0003:00000b1c       $pdata$??$?RV<lambda_410d79af7f07d98d83a3f525b3859a53>@@AEAV<lambda_3e16ef9562a7dcce91392c22ab16ea36>@@V<lambda_38119f0e861e05405d8a144b9b982f0a>@@@?$__crt_seh_guarded_call@X@@QEAAX$$QEAV<lambda_410d79af7f07d98d83a3f525b3859a53>@@AEAV<lambda_3e16ef9562a7dcce91392c22ab16ea36>@@$$QEAV<lambda_38119f0e861e05405d8a144b9b982f0a>@@@Z 000000018001cb1c     libucrt:wsetlocale.obj
 0003:00000b28       $pdata$?fin$0@?0???$?RV<lambda_410d79af7f07d98d83a3f525b3859a53>@@AEAV<lambda_3e16ef9562a7dcce91392c22ab16ea36>@@V<lambda_38119f0e861e05405d8a144b9b982f0a>@@@?$__crt_seh_guarded_call@X@@QEAAX$$QEAV<lambda_410d79af7f07d98d83a3f525b3859a53>@@AEAV<lambda_3e16ef9562a7dcce91392c22ab16ea36>@@$$QEAV<lambda_38119f0e861e05405d8a144b9b982f0a>@@@Z@4HA 000000018001cb28     libucrt:wsetlocale.obj
 0003:00000b34       $pdata$__pctype_func       000000018001cb34     libucrt:ctype.obj
 0003:00000b40       $pdata$__acrt_release_locale_ref 000000018001cb40     libucrt:locale_refcounting.obj
 0003:00000b4c       $pdata$__acrt_free_locale  000000018001cb4c     libucrt:locale_refcounting.obj
 0003:00000b58       $pdata$__acrt_locale_free_lc_time_if_unreferenced 000000018001cb58     libucrt:locale_refcounting.obj
 0003:00000b64       $pdata$__acrt_update_thread_locale_data 000000018001cb64     libucrt:locale_refcounting.obj
 0003:00000b70       $pdata$__acrt_update_thread_locale_data$fin$0 000000018001cb70     libucrt:locale_refcounting.obj
 0003:00000b7c       $pdata$_updatetlocinfoEx_nolock 000000018001cb7c     libucrt:locale_refcounting.obj
 0003:00000b88       $pdata$qsort               000000018001cb88     libucrt:qsort.obj
 0003:00000b94       $pdata$4$qsort             000000018001cb94     libucrt:qsort.obj
 0003:00000ba0       $pdata$5$qsort             000000018001cba0     libucrt:qsort.obj
 0003:00000bac       $pdata$strncpy_s           000000018001cbac     libucrt:strncpy_s.obj
 0003:00000bb8       $pdata$strpbrk             000000018001cbb8     libucrt:strpbrk.obj
 0003:00000bc4       $pdata$fallbackMethod      000000018001cbc4     libucrt:strpbrk.obj
 0003:00000bd0       $pdata$_mbsdec_l           000000018001cbd0     libucrt:mbsdec.obj
 0003:00000bdc       $pdata$__acrt_GetStringTypeA 000000018001cbdc     libucrt:getstringtypea.obj
 0003:00000be8       $pdata$__acrt_LCMapStringA 000000018001cbe8     libucrt:lcmapstringa.obj
 0003:00000bf4       $pdata$?__acrt_LCMapStringA_stat@@YAHPEAU__crt_locale_pointers@@PEB_WKPEBDHPEADHHH@Z 000000018001cbf4     libucrt:lcmapstringa.obj
 0003:00000c00       $pdata$?initialize_multibyte@@YAHXZ 000000018001cc00     libucrt:multibyte_initializer.obj
 0003:00000c0c       $pdata$_msize_base         000000018001cc0c     libucrt:msize.obj
 0003:00000c18       $pdata$_realloc_base       000000018001cc18     libucrt:realloc_base.obj
 0003:00000c24       $pdata$__acrt_DownlevelLocaleNameToLCID 000000018001cc24     libucrt:lcidtoname_downlevel.obj
 0003:00000c30       $pdata$_get_osfhandle      000000018001cc30     libucrt:osfinfo.obj
 0003:00000c3c       $pdata$_free_osfhnd        000000018001cc3c     libucrt:osfinfo.obj
 0003:00000c48       $pdata$__acrt_lowio_create_handle_array 000000018001cc48     libucrt:osfinfo.obj
 0003:00000c54       $pdata$__acrt_lowio_destroy_handle_array 000000018001cc54     libucrt:osfinfo.obj
 0003:00000c60       $pdata$__acrt_lowio_ensure_fh_exists 000000018001cc60     libucrt:osfinfo.obj
 0003:00000c6c       $pdata$_commit             000000018001cc6c     libucrt:commit.obj
 0003:00000c78       $pdata$??$?RV<lambda_a37b2b86f63e897a80ea819b0eb08c01>@@AEAV<lambda_38ce7e780aa69e748d6df282ebc68efe>@@V<lambda_99fb1378e971ab6e7edea83e3a7a83a2>@@@?$__crt_seh_guarded_call@H@@QEAAH$$QEAV<lambda_a37b2b86f63e897a80ea819b0eb08c01>@@AEAV<lambda_38ce7e780aa69e748d6df282ebc68efe>@@$$QEAV<lambda_99fb1378e971ab6e7edea83e3a7a83a2>@@@Z 000000018001cc78     libucrt:commit.obj
 0003:00000c84       $pdata$?fin$0@?0???$?RV<lambda_751a882b2c74d4b022dec766aa51a29a>@@AEAV<lambda_628dfdc04ba53c8bfc02c9951375f3f5>@@V<lambda_f6c7be5f7998530c34de24c7437d6b54>@@@?$__crt_seh_guarded_call@H@@QEAAH$$QEAV<lambda_751a882b2c74d4b022dec766aa51a29a>@@AEAV<lambda_628dfdc04ba53c8bfc02c9951375f3f5>@@$$QEAV<lambda_f6c7be5f7998530c34de24c7437d6b54>@@@Z@4HA 000000018001cc84     libucrt:close.obj
 0003:00000c84       $pdata$?fin$0@?0???$?RV<lambda_a37b2b86f63e897a80ea819b0eb08c01>@@AEAV<lambda_38ce7e780aa69e748d6df282ebc68efe>@@V<lambda_99fb1378e971ab6e7edea83e3a7a83a2>@@@?$__crt_seh_guarded_call@H@@QEAAH$$QEAV<lambda_a37b2b86f63e897a80ea819b0eb08c01>@@AEAV<lambda_38ce7e780aa69e748d6df282ebc68efe>@@$$QEAV<lambda_99fb1378e971ab6e7edea83e3a7a83a2>@@@Z@4HA 000000018001cc84     libucrt:commit.obj
 0003:00000c90       $pdata$_write              000000018001cc90     libucrt:write.obj
 0003:00000c9c       $pdata$_write$fin$0        000000018001cc9c     libucrt:write.obj
 0003:00000ca8       $pdata$_write_nolock       000000018001cca8     libucrt:write.obj
 0003:00000cb4       $pdata$?write_double_translated_ansi_nolock@@YA?AUwrite_result@?A0x17268360@@HQEBDI@Z 000000018001ccb4     libucrt:write.obj
 0003:00000cc0       $pdata$?write_text_ansi_nolock@@YA?AUwrite_result@?A0x17268360@@HQEBDI@Z 000000018001ccc0     libucrt:write.obj
 0003:00000ccc       $pdata$?write_text_utf16le_nolock@@YA?AUwrite_result@?A0x17268360@@HQEBDI@Z 000000018001cccc     libucrt:write.obj
 0003:00000cd8       $pdata$?write_text_utf8_nolock@@YA?AUwrite_result@?A0x17268360@@HQEBDI@Z 000000018001ccd8     libucrt:write.obj
 0003:00000ce4       $pdata$_fcloseall          000000018001cce4     libucrt:closeall.obj
 0003:00000cf0       $pdata$_fcloseall$fin$0    000000018001ccf0     libucrt:closeall.obj
 0003:00000cfc       $pdata$__acrt_stdio_free_buffer_nolock 000000018001ccfc     libucrt:_freebuf.obj
 0003:00000d08       $pdata$_isatty             000000018001cd08     libucrt:isatty.obj
 0003:00000d14       $pdata$_isleadbyte_l       000000018001cd14     libucrt:_wctype.obj
 0003:00000d20       $pdata$?__mbrtowc_utf8@__crt_mbstring@@YA_KPEA_WPEBD_KPEAU_Mbstatet@@@Z 000000018001cd20     libucrt:mbrtowc.obj
 0003:00000d2c       $pdata$?__mbsrtowcs_utf8@__crt_mbstring@@YA_KPEA_WPEAPEBD_KPEAU_Mbstatet@@@Z 000000018001cd2c     libucrt:mbrtowc.obj
 0003:00000d38       $pdata$__acrt_locale_free_monetary 000000018001cd38     libucrt:initmon.obj
 0003:00000d44       $pdata$__acrt_locale_free_numeric 000000018001cd44     libucrt:initnum.obj
 0003:00000d50       $pdata$__acrt_locale_free_time 000000018001cd50     libucrt:inittime.obj
 0003:00000d5c       $pdata$?free_crt_array_internal@@YAXQEAPEBX_K@Z 000000018001cd5c     libucrt:inittime.obj
 0003:00000d68       $pdata$??$common_lseek_nolock@_J@@YA_JH_JH@Z 000000018001cd68     libucrt:lseek.obj
 0003:00000d74       $pdata$_putwch_nolock      000000018001cd74     libucrt:putwch.obj
 0003:00000d80       $pdata$fclose              000000018001cd80     libucrt:fclose.obj
 0003:00000d8c       $pdata$fclose$fin$0        000000018001cd8c     libucrt:fclose.obj
 0003:00000d98       $pdata$_fclose_nolock      000000018001cd98     libucrt:fclose.obj
 0003:00000da4       $pdata$?__mbrtoc32_utf8@__crt_mbstring@@YA_KPEA_UPEBD_KPEAU_Mbstatet@@@Z 000000018001cda4     libucrt:mbrtoc32.obj
 0003:00000dbc       $pdata$__dcrt_lowio_ensure_console_output_initialized 000000018001cdbc     libucrt:initcon.obj
 0003:00000dc8       $pdata$__dcrt_write_console 000000018001cdc8     libucrt:initcon.obj
 0003:00000dd4       $pdata$__dcrt_terminate_console_output 000000018001cdd4     libucrt:initcon.obj
 0003:00000de0       $pdata$_close              000000018001cde0     libucrt:close.obj
 0003:00000dec       $pdata$_close_nolock       000000018001cdec     libucrt:close.obj
 0003:00000df8       $pdata$??$?RV<lambda_751a882b2c74d4b022dec766aa51a29a>@@AEAV<lambda_628dfdc04ba53c8bfc02c9951375f3f5>@@V<lambda_f6c7be5f7998530c34de24c7437d6b54>@@@?$__crt_seh_guarded_call@H@@QEAAH$$QEAV<lambda_751a882b2c74d4b022dec766aa51a29a>@@AEAV<lambda_628dfdc04ba53c8bfc02c9951375f3f5>@@$$QEAV<lambda_f6c7be5f7998530c34de24c7437d6b54>@@@Z 000000018001cdf8     libucrt:close.obj
 0003:00000e04       $pdata$_call_matherr       000000018001ce04     libucrt:libm_error.obj
 0003:00000e10       $pdata$_exception_enabled  000000018001ce10     libucrt:libm_error.obj
 0003:00000e1c       $pdata$_handle_error       000000018001ce1c     libucrt:libm_error.obj
 0003:00000e28       $pdata$__acrt_initialize_fma3 000000018001ce28     libucrt:fma3_available.obj
 0003:00000e34       $pdata$_log_special_common 000000018001ce34     libucrt:log_special.obj
 0003:00000e40       $pdata$_log10_special      000000018001ce40     libucrt:log_special.obj
 0003:00000e58       $pdata$_set_errno_from_matherr 000000018001ce58     libucrt:fpexcept.obj
 0003:00000e64       $pdata$_raise_exc          000000018001ce64     libucrt:fpexcept.obj
 0003:00000e70       $pdata$_raise_exc_ex       000000018001ce70     libucrt:fpexcept.obj
 0003:00000e7c       $pdata$_clrfp              000000018001ce7c     libucrt:fpctrl.obj
 0003:00000e88       $pdata$_ctrlfp             000000018001ce88     libucrt:fpctrl.obj
 0003:00000e94       $pdata$_ctrlfp$filt$0      000000018001ce94     libucrt:fpctrl.obj
 0003:00000ea0       $pdata$_statfp             000000018001cea0     libucrt:fpctrl.obj
 0003:00000eac       $pdata$_set_statfp         000000018001ceac     libucrt:fpctrl.obj
 0003:00000eb8       $pdata$_IsNonwritableInCurrentImage 000000018001ceb8     LIBCMT:pesect.obj
 0003:00000ec4       $pdata$_IsNonwritableInCurrentImage$filt$0 000000018001cec4     LIBCMT:pesect.obj
 0003:00000ed0       $pdata$__GSHandlerCheckCommon 000000018001ced0     LIBCMT:gshandler.obj
 0003:00000edc       $pdata$__GSHandlerCheck    000000018001cedc     LIBCMT:gshandler.obj
 0003:00000ef4       $pdata$__report_securityfailure 000000018001cef4     LIBCMT:gs_report.obj
 0003:00000f00       $pdata$__report_rangecheckfailure 000000018001cf00     LIBCMT:gs_report.obj
 0003:00000f0c       $pdata$__report_gsfailure  000000018001cf0c     LIBCMT:gs_report.obj
 0003:00000f18       $pdata$capture_current_context 000000018001cf18     LIBCMT:gs_report.obj
 0003:00000f24       $pdata$capture_previous_context 000000018001cf24     LIBCMT:gs_report.obj
 0003:00000f30       $pdata$__raise_securityfailure 000000018001cf30     LIBCMT:gs_report.obj
 0004:00000504       .idata$6                   000000018001d504     kernel32:KERNEL32.dll
 0004:00000520       .idata$6                   000000018001d520     user32:USER32.dll
 0005:00000000       MsetTab                    000000018001e000     libvcruntime:memset.obj
 0005:00000050       MoveSmall                  000000018001e050     libvcruntime:memcpy.obj
 0006:00000060       $R000000                   000000018001f060     Brackets.res
